:020000040800F2
:1000000000500020B1230008612400082D360008AC
:100010006124000861240008612400080000000039
:100020000000000000000000000000006124000843
:100030006124000800000000612400084155000808
:10004000612400086124000861240008612400087C
:10005000612400086124000861240008612400086C
:10006000612400086124000861240008612400085C
:100070006124000861240008555400086124000828
:10008000612400086124000861240008612400083C
:10009000612400086124000861240008612400082C
:1000A00061240008612400086124000885230008F9
:1000B0009123000899230008A52300083D4C00085F
:1000C000BD4F0008414C0008B94F000861240008EA
:1000D0006124000889540008C55400086124000800
:1000E0006124000861240008612400080000000069
:1000F0000000000000000000000000000000000000
:0C01000000000000000000005FF808F1A3
:1001100010B5054C237833B9044810B10448AFF347
:1001200000800121217010BD9C050020000000000E
:100130005011010808B5064B1BB106480649AFF33C
:1001400000800648016811B1054A02B1904708BD18
:100150000000000050110108A00500209C050020AF
:100160000000000081F0004102E000BF83F0004386
:1001700030B54FEA41044FEA430594EA050F08BF42
:1001800090EA020F1FBF54EA000C55EA020C7FEA06
:10019000645C7FEA655C00F0E2804FEA5454D4EB83
:1001A0005555B8BF6D420CDD2C4480EA020281EA4D
:1001B000030382EA000083EA010180EA020281EA85
:1001C0000303362D88BF30BD11F0004F4FEA0131D7
:1001D0004FF4801C4CEA113102D0404261EB4101E6
:1001E00013F0004F4FEA03334CEA133302D052426C
:1001F00063EB430394EA050F00F0A780A4F1010428
:10020000D5F1200E0DDB02FA0EFC22FA05F2801861
:1002100041F1000103FA0EF2801843FA05F3594147
:100220000EE0A5F120050EF1200E012A03FA0EFCC6
:1002300028BF4CF0020C43FA05F3C01851EBE371F0
:1002400001F0004507D54FF0000EDCF1000C7EEB0D
:1002500000006EEB0101B1F5801F1BD3B1F5001F4B
:100260000CD349085FEA30004FEA3C0C04F101046A
:100270004FEA445212F5800F80F09A80BCF1004F93
:1002800008BF5FEA500C50F1000041EB045141EA15
:10029000050130BD5FEA4C0C404141EB010111F416
:1002A000801FA4F10104E9D191F0000F04BF0146C1
:1002B0000020B1FA81F308BF2033A3F10B03B3F19F
:1002C00020020CDA0C3208DD02F1140CC2F10C022F
:1002D00001FA0CF021FA02F10CE002F11402D8BF8D
:1002E000C2F1200C01FA02F120FA0CFCDCBF41EA59
:1002F0000C019040E41AA2BF01EB0451294330BD28
:100300006FEA04041F3C1CDA0C340EDC04F1140404
:10031000C4F1200220FA04F001FA02F340EA0300DB
:1003200021FA04F345EA030130BDC4F10C04C4F121
:10033000200220FA02F001FA04F340EA0300294601
:1003400030BD21FA04F0294630BD94F0000F83F44B
:10035000801306BF81F480110134013D4EE77FEA2E
:10036000645C18BF7FEA655C29D094EA050F08BF7A
:1003700090EA020F05D054EA000C04BF194610465B
:1003800030BD91EA030F1EBF0021002030BD5FEA9F
:10039000545C05D14000494128BF41F0004130BDC7
:1003A00014F580043CBF01F5801130BD01F000451B
:1003B00045F0FE4141F470014FF0000030BD7FEA8E
:1003C000645C1ABF194610467FEA655C1CBF0B4689
:1003D000024650EA013406BF52EA033591EA030FA0
:1003E00041F4002130BD00BF90F0000F04BF002198
:1003F000704730B54FF4806404F132044FF00005CB
:100400004FF0000150E700BF90F0000F04BF002143
:10041000704730B54FF4806404F1320410F00045A9
:1004200048BF40424FF000013EE700BF42004FEAA4
:10043000E2014FEA31014FEA02701FBF12F07F4321
:1004400093F07F4F81F06051704792F0000F14BF1E
:1004500093F07F4F704730B54FF4607401F0004562
:1004600021F0004120E700BF50EA010208BF7047B9
:1004700030B54FF000050AE050EA010208BF7047AE
:1004800030B511F0004502D5404261EB41014FF417
:10049000806404F132045FEA915C3FF4DCAE4FF01B
:1004A00003025FEADC0C18BF03325FEADC0C18BF02
:1004B000033202EBDC02C2F1200300FA03FC20FA53
:1004C00002F001FA03FE40EA0E0021FA02F11444A0
:1004D000C1E600BF70B54FF0FF0C4CF4E06C1CEAB5
:1004E00011541DBF1CEA135594EA0C0F95EA0C0F2A
:1004F00000F0DEF82C4481EA030621EA4C5123EA9D
:100500004C5350EA013518BF52EA033541F48011CB
:1005100043F4801338D0A0FB02CE4FF00005E1FB7E
:1005200002E506F00042E0FB03E54FF00006E1FBC8
:1005300003569CF0000F18BF4EF0010EA4F1FF040B
:10054000B6F5007F64F5407404D25FEA4E0E6D414B
:1005500046EB060642EAC62141EA55514FEAC5205C
:1005600040EA5E504FEACE2EB4F1FD0C88BFBCF5D8
:10057000E06F1ED8BEF1004F08BF5FEA500E50F189
:10058000000041EB045170BD06F0004646EA01014F
:1005900040EA020081EA0301B4EB5C04C2BFD4EB81
:1005A0000C0541EA045170BD41F480114FF0000E7A
:1005B000013C00F3AB8014F1360FDEBF002001F0E8
:1005C000004170BDC4F10004203C35DA0C341BDC62
:1005D00004F11404C4F1200500FA05F320FA04F034
:1005E00001FA05F240EA020001F0004221F0004168
:1005F00010EBD37021FA04F642EB06015EEA430EDB
:1006000008BF20EAD37070BDC4F10C04C4F120050A
:1006100000FA04F320FA05F001FA04F240EA0200BD
:1006200001F0004110EBD37041F100015EEA430E8E
:1006300008BF20EAD37070BDC4F1200500FA05F2AE
:100640004EEA020E20FA04F301FA05F243EA02032D
:1006500021FA04F001F0004121FA04F220EA02003C
:1006600000EBD3705EEA430E08BF20EAD37070BD82
:1006700094F0000F0FD101F00046400041EB010162
:1006800011F4801F08BF013CF7D041EA060195F044
:10069000000F18BF704703F00046520043EB0303FE
:1006A00013F4801F08BF013DF7D043EA06037047EB
:1006B00094EA0C0F0CEA135518BF95EA0C0F0CD0F6
:1006C00050EA410618BF52EA4306D1D181EA03013C
:1006D00001F000414FF0000070BD50EA410606BF36
:1006E0001046194652EA430619D094EA0C0F02D17B
:1006F00050EA013613D195EA0C0F05D152EA0336C0
:100700001CBF104619460AD181EA030101F00041DD
:1007100041F0FE4141F470014FF0000070BD41F026
:10072000FE4141F4780170BD70B54FF0FF0C4CF400
:10073000E06C1CEA11541DBF1CEA135594EA0C0F1F
:1007400095EA0C0F00F0A7F8A4EB050481EA030E6C
:1007500052EA03354FEA013100F088804FEA033353
:100760004FF0805545EA131343EA12634FEA022221
:1007700045EA111545EA10654FEA00260EF00041E2
:100780009D4208BF964244F1FD0404F5407402D234
:100790005B084FEA3202B61A65EB03055B084FEAC5
:1007A00032024FF480104FF4002CB6EB020E75EBC2
:1007B000030E22BFB61A754640EA0C005B084FEAEA
:1007C0003202B6EB020E75EB030E22BFB61A754667
:1007D00040EA5C005B084FEA3202B6EB020E75EBB2
:1007E000030E22BFB61A754640EA9C005B084FEA2A
:1007F0003202B6EB020E75EB030E22BFB61A754637
:1008000040EADC0055EA060E18D04FEA051545EA25
:1008100016754FEA06164FEAC30343EA52734FEACE
:10082000C2025FEA1C1CC0D111F4801F0BD141EA47
:1008300000014FF000004FF0004CB6E711F4801FAC
:1008400004BF01430020B4F1FD0C88BFBCF5E06F8C
:100850003FF6AFAEB5EB030C04BFB6EB020C5FEA9C
:10086000500C50F1000041EB045170BD0EF0004EF1
:100870004EEA113114EB5C04C2BFD4EB0C0541EA23
:10088000045170BD41F480114FF0000E013C90E620
:1008900045EA060E8DE60CEA135594EA0C0F08BFE4
:1008A00095EA0C0F3FF43BAF94EA0C0F0AD150EAE3
:1008B00001347FF434AF95EA0C0F7FF425AF104676
:1008C00019462CE795EA0C0F06D152EA03353FF49E
:1008D000FDAE1046194622E750EA410618BF52EA1B
:1008E00043067FF4C5AE50EA41047FF40DAF52EAEF
:1008F00043057FF4EBAE12E74FEA4102B2F1E04369
:1009000024BFB3F5001CDCF1FE5C0DD901F0004CF6
:100910004FEAC0024CEA5070B2F1004F40EB830046
:1009200008BF20F00100704711F0804F21D113F172
:100930003872BCBF01F00040704741F480114FEAAB
:100940005252C2F11802C2F1200C10FA0CF320FA34
:1009500002F018BF40F001004FEAC1234FEAD32351
:1009600003FA0CFC40EA0C0023FA02F34FEA4303BB
:10097000CCE77FEA625307D150EA01331EBF4FF044
:10098000FE4040F44000704701F0004040F0FE405F
:1009900040F40000704700BF80F0004002E000BF5C
:1009A00081F0004142001FBF5FEA410392EA030F5A
:1009B0007FEA226C7FEA236C6AD04FEA1262D2EBA4
:1009C0001363C1BFD218414048404140B8BF5B42A9
:1009D000192B88BF704710F0004F40F4000020F042
:1009E0007F4018BF404211F0004F41F4000121F058
:1009F0007F4118BF494292EA030F3FD0A2F10102A2
:100A000041FA03FC10EB0C00C3F1200301FA03F1DF
:100A100000F0004302D5494260EB4000B0F5000F02
:100A200013D3B0F1807F06D340084FEA310102F1C1
:100A30000102FE2A51D2B1F1004F40EBC25008BF73
:100A400020F0010040EA03007047490040EB00003D
:100A500010F4000FA2F10102EDD1B0FA80FCACF16C
:100A6000080CB2EB0C0200FA0CF0AABF00EBC2506B
:100A700052421843BCBFD0401843704792F0000F59
:100A800081F4000106BF80F400000132013BB5E7AC
:100A90004FEA41037FEA226C18BF7FEA236C21D022
:100AA00092EA030F04D092F0000F08BF0846704787
:100AB00090EA010F1CBF0020704712F07F4F04D155
:100AC000400028BF40F00040704712F100723CBF68
:100AD00000F50000704700F0004343F0FE4040F492
:100AE000000070477FEA226216BF08467FEA236350
:100AF0000146420206BF5FEA412390EA010F40F43B
:100B0000800070474FF0000304E000BF10F0004386
:100B100048BF40425FEA000C08BF704743F096436D
:100B200001464FF000001CE050EA010208BF704788
:100B30004FF000030AE000BF50EA010208BF70470F
:100B400011F0004302D5404261EB41015FEA010C24
:100B500002BF84460146002043F0B64308BFA3F11C
:100B60008053A3F50003BCFA8CF2083AA3EBC253FE
:100B700010DB01FA02FC634400FA02FCC2F120021D
:100B8000BCF1004F20FA02F243EB020008BF20F054
:100B90000100704702F1200201FA02FCC2F12002BA
:100BA00050EA4C0021FA02F243EB020008BF20EAAF
:100BB000DC7070474FF0FF0C1CEAD0521EBF1CEADD
:100BC000D15392EA0C0F93EA0C0F6FD01A4480EACB
:100BD000010C400218BF5FEA41211ED04FF00063B4
:100BE00043EA501043EA5111A0FB01310CF00040E0
:100BF000B1F5000F3EBF490041EAD3715B0040EA06
:100C0000010062F17F02FD2A1DD8B3F1004F40EBD5
:100C1000C25008BF20F00100704790F0000F0CF0A8
:100C2000004C08BF49024CEA502040EA51207F3A6C
:100C3000C2BFD2F1FF0340EAC250704740F4000047
:100C40004FF00003013A5DDC12F1190FDCBF00F038
:100C500000407047C2F10002410021FA02F1C2F1E6
:100C6000200200FA02FC5FEA310040F1000053EA82
:100C70004C0308BF20EADC70704792F0000F00F0D0
:100C8000004C02BF400010F4000F013AF9D040EAD6
:100C90000C0093F0000F01F0004C02BF490011F46A
:100CA000000F013BF9D041EA0C018FE70CEAD15368
:100CB00092EA0C0F18BF93EA0C0F0AD030F0004CE8
:100CC00018BF31F0004CD8D180EA010000F000409C
:100CD000704790F0000F17BF90F0004F084691F05A
:100CE000000F91F0004F14D092EA0C0F01D1420294
:100CF0000FD193EA0C0F03D14B0218BF084608D15D
:100D000080EA010000F0004040F0FE4040F40000A6
:100D1000704740F0FE4040F4400070474FF0FF0C39
:100D20001CEAD0521EBF1CEAD15392EA0C0F93EA80
:100D30000C0F69D0A2EB030280EA010C49024FEAD2
:100D4000402037D04FF0805343EA111143EA10138B
:100D50000CF000408B4238BF5B0042F17D024FF443
:100D6000000C8B4224BF5B1A40EA0C00B3EB510F1E
:100D700024BFA3EB510340EA5C00B3EB910F24BF07
:100D8000A3EB910340EA9C00B3EBD10F24BFA3EB8C
:100D9000D10340EADC001B0118BF5FEA1C1CE0D154
:100DA000FD2A3FF650AF8B4240EBC25008BF20F007
:100DB000010070470CF0004C4CEA50207F32C2BF5B
:100DC000D2F1FF0340EAC250704740F400004FF0F8
:100DD0000003013A37E792F0000F00F0004C02BF29
:100DE000400010F4000F013AF9D040EA0C0093F0F3
:100DF000000F01F0004C02BF490011F4000F013B4D
:100E0000F9D041EA0C0195E70CEAD15392EA0C0FB4
:100E100008D142027FF47DAF93EA0C0F7FF470AFEC
:100E2000084676E793EA0C0F04D14B023FF44CAF2F
:100E300008466EE730F0004C18BF31F0004CCAD1C4
:100E400030F000427FF45CAF31F000437FF43CAF00
:100E50005FE700BF4FF0FF3C06E000BF4FF0010C22
:100E600002E000BF4FF0010C4DF804CD4FEA400204
:100E70004FEA41037FEA226C18BF7FEA236C11D04E
:100E800001B052EA530C18BF90EA010F58BFB2EB01
:100E9000030088BFC81738BF6FEAE17018BF40F081
:100EA000010070477FEA226C02D15FEA402C05D135
:100EB0007FEA236CE4D15FEA412CE1D05DF8040BBA
:100EC000704700BF844608466146FFE70FB5FFF74D
:100ED000C9FF002848BF10F1000F0FBD4DF808ED05
:100EE000FFF7F4FF0CBF012000205DF808FB00BFF6
:100EF0004DF808EDFFF7EAFF34BF012000205DF850
:100F000008FB00BF4DF808EDFFF7E0FF94BF01209C
:100F100000205DF808FB00BF4DF808EDFFF7D2FF99
:100F200094BF012000205DF808FB00BF4DF808EDDC
:100F3000FFF7C8FF34BF012000205DF808FB00BFA9
:100F40004FEA4002B2F1FE4F0FD34FF09E03B3EBD6
:100F500012620DD94FEA002343F0004310F0004F16
:100F600023FA02F018BF404270474FF0000070476C
:100F700012F1610F01D1420205D110F0004008BF0B
:100F80006FF0004070474FF00000704742000ED2F3
:100F9000B2F1FE4F0BD34FF09E03B3EB126209D4B4
:100FA0004FEA002343F0004323FA02F070474FF06A
:100FB0000000704712F1610F01D1420202D14FF0DF
:100FC000FF3070474FF00000704700BF2E4B2DE9F7
:100FD000F34105461878002838D0002426462746D5
:100FE000A0463221082253206B4603F0C3FE9DF831
:100FF00001109DF80000013400EB01239DF803105F
:101000009DF802001AB200EB01239DF805109DF82F
:101010000400E4B290441AB200EB01239DF80710DB
:10102000BF18202C1AB2164401F07F0001D000280E
:10103000D7D1164B98FBF4F897FBF4F796FBF4F630
:10104000A5F800806F80AE801C701AE03221062265
:101050006B46532003F08EFE9DF801209DF8001092
:101060009DF8030001EB02239DF802202B8002EB88
:1010700000219DF804309DF80500698003EB0022F3
:10108000AA80BDE8FC8100BFB8050020B90500209A
:1010900008B5134B53201B782D2108227BB103F098
:1010A0002DFF31210A22532003F028FF2C210C228E
:1010B000532003F023FF53203821902209E003F04E
:1010C0001DFF31210A22532003F018FF53202C2149
:1010D0000A2203F013FF034840F20912028008BD00
:1010E000B80500200C00002037B5104B05461A68E3
:1010F0000F480C46002182428DF8071001D10020D4
:1011000013E0532001220DF1070303F033FE002802
:10111000F5D09DF80710E529F1D12A780548064B4E
:10112000064920601A70616001203EBD4801002020
:10113000001BB70091100008B8050020CD0F000873
:1011400013B5022204461B2101AB682003F012FEF6
:101150009DF804209DF8053043EA022000F54E5129
:1011600010314FF48C7291FBF2F3233323801CBDBA
:1011700013B5062204461D216B46682003F0FAFDD4
:101180009DF800209DF8013043EA022001B20423BB
:1011900091FBF3F29DF802009DF80310228041EAD2
:1011A000002210B290FBF3F19DF805209DF8040099
:1011B000618042EA002108B290FBF3F3A3801CBDDA
:1011C00008B5192004F0EFF968201521002203F07A
:1011D00095FE10B9032004F057FA0C4B16211A782B
:1011E000682042F0180203F089FE172100226820CF
:1011F00003F084FE3D210122682003F07FFE682079
:101200003E210122BDE8084003F078BE0000002026
:1012100038B5054619200C4604F0C5F9682015219B
:10122000002203F06BFE18B3124B13481349144A03
:10123000622C2B606860A960EA60124B0FD004D862
:101240000A2C12D0142C0CD10DE0BC2C04D0B4F517
:10125000807F06D1002009E00120187038BD0220EF
:1012600004E0032002E0042000E0052018700120C3
:1012700038BD00BFC11100087111000841110008FC
:101280001844923100000020064B187820B1012844
:1012900006D14FF4805201E04FF4006202490A8007
:1012A000704700BFBA0500200C00002013B50622CD
:1012B000044643216B46682003F05CFD9DF8002046
:1012C0009DF8013043EA022001B2042391FBF3F2BE
:1012D0009DF802009DF80310228041EA002210B21E
:1012E00090FBF3F19DF805209DF80400618042EA2F
:1012F000002108B290FBF3F3A3801CBD13B50622B6
:1013000004463B216B46682003F034FD9DF8002025
:101310009DF801309DF8021043EA02209DF8032059
:10132000208042EA01239DF804009DF805106380A7
:1013300041EA0022A2801CBD07B5204A02204FF4DA
:101340000053ADF804308DF8070013681C480421E1
:1013500083428DF8061001D11A4803E01A498B42E6
:1013600003D11A4801A903F031FE6B2180226820C5
:1013700003F0C4FD052004F016F9192100226820AD
:1013800003F0BCFD6B210322682003F0B7FD372179
:101390000222682003F0B2FD0D4A1A21682012785B
:1013A00003F0ACFD1B211822682003F0A7FD682084
:1013B0001C21102203F0A2FD0EBD00BF4801002039
:1013C00000127A00000C0140001BB7000010014021
:1013D000010000202DE9FF41064623200D4614465A
:1013E00004F0E1F86820752101220DF1070303F0F4
:1013F000C1FC00286DD09DF80780B8F1680F67D157
:1014000006210A4602AB404603F0B4FC9DF80B30BF
:101410009DF80D7003F0010107F001004A0042EA57
:1014200080079DF8090000F001031F4307D0012F3A
:10143000294801D1002318E0022F0CD114E00C211F
:10144000012240460DF1070303F094FC9DF80710BC
:1014500011F00F0203D1052004F016F906E0042A6A
:101460001D4801D1077001E0012303701A481B4990
:1014700003781B4A31607260002B14BF6E216F210C
:10148000184A1948194B142C31722A606860EB60B5
:10149000174915D004D8052C16D00A2C0ED111E00E
:1014A000BC2C08D0B4F5807F03D0622C06D1022278
:1014B0000BE0002209E0012008700AE0032204E0AA
:1014C000042202E0052200E006220A70012000E06A
:1014D000002004B0BDE8F081BA05002089120008A0
:1014E000FD12000839130008AD12000819449231AA
:1014F0000100002013B506220446A8216B4668208F
:1015000003F038FC9DF800209DF8013043EA0220EA
:1015100001B2042391FBF3F29DF802009DF8031041
:10152000228041EA002210B290FBF3F19DF80520E1
:101530009DF80400618042EA002108B290FBF3F3B9
:10154000A3801CBD08B5642004F02DF86820232179
:10155000F02203F0D3FC10B9032004F095F8052025
:1015600004F021F8044B68201A78202142F00F0281
:10157000BDE8084003F0C2BCBB05002037B50546F6
:1015800019200C4604F00FF868200F2101220DF1FC
:10159000070303F0EFFB9DF80730D32B16D10C485F
:1015A0000C490D4A4E2C28606960EA600B4B07D04D
:1015B0005D2C09D0362C01D0002002E0402000E054
:1015C00080201870012002E0C020FAE700203EBD14
:1015D00045150008F5140008DDE9A731BB0500201A
:1015E0002DE9F041057890B000350646334818BF24
:1015F00001250AF0BBF800243148A542314B0CBF4D
:101600002146802106904FF400500CBF4FF0010896
:101610004FF002084FF4807205930A9120234FF493
:1016200080670E9005A925480B920D930C9707949F
:10163000CDF8208009940F940AF010F91F48012179
:101640000AF039F94FF46021012702911E486946DA
:1016500000948DF804508DF8057003948DF8108077
:1016600009F02AFA184804213A46032309F075FACA
:101670002DB1154831780222032309F06EFA124881
:10168000012109F046FA1048012109F039FA0E4803
:1016900009F048FA0C4809F04AFA0028FAD10A4839
:1016A00009F049FA084809F04BFA0028FAD106482F
:1016B000012109F049FA10B0BDE8F08108000240AC
:1016C000BC0500204C24014000240140024B33F8AB
:1016D000100080B2704700BFBC050020F8B5134B66
:1016E00005469B890E461446ECB116B116F8017BEF
:1016F00000E0FF270D48022109F0D8F90028F9D0B1
:101700000A48394609F0CDF90848012109F0CEF917
:101710000028F9D0054809F0C6F9C0B20DB105F8A6
:10172000010B013CE0E70120F8BD00BF003800409C
:101730002DE9F047012188B04FF4804009F012FFF5
:10174000374C01214FF4804009F024FF03214FF46E
:1017500020401823ADF800008DF80310204669469C
:101760008DF802304FF0040803F030FC2D4E4FF49A
:10177000804220466946ADF800204FF480554FF076
:10178000100A8DF8028003F021FC69462046ADF86E
:1017900000508DF802A003F019FC304609F024F93E
:1017A00007214FF4007000230222ADF81600ADF8B7
:1017B0001C104FF00109304603A94FF48277ADF8B1
:1017C0000C30ADF81030ADF81A30ADF81220ADF88D
:1017D0000E70ADF814901F46ADF818A009F036F958
:1017E0003046494609F051F99F238DF804308DF8B1
:1017F00005708DF806708DF807700DEB08014246F4
:10180000656102A8FFF76AFF25619DF80900B0F144
:10181000EF014A4252EB010008B0BDE8F08700BF7B
:10182000000C014000380040074BA1F57A7153F8D5
:101830002000838802684B434FF47A7093FBF0F1E9
:101840008BB21380704700BFC0060020024B53F8D4
:101850002000026811807047C00600202DE9F04F7B
:10186000DFF828814FEA001558F805408E468BB006
:1018700008EB0507114683469246204672460193BF
:1018800000F0CEFCB96807F108024FF0020C1823F3
:101890007868ADF8141005A98DF816308DF817C0CA
:1018A0000392CDF808C003F091FB0398364E0779F8
:1018B00006A809F09EFB70220198DDF808C0ADF87B
:1018C0001820012100234FF4807206EB0509ADF8C2
:1018D0001A10ADF81C30ADF81E00ADF820C0ADF800
:1018E00024200C2F2BD8DFE807F0072A2A2A102AF9
:1018F0002A2A192A2A2A2200204606A909F072FA61
:101900002046082109F0AAFB19E0204606A909F0A3
:10191000ADFA2046082109F0A9FB10E0204606A9EF
:1019200009F0E8FA2046082109F0AAFB07E0204662
:1019300006A909F021FB2046082109F0A9FB08EBC4
:101940000B118B7B1BB12046012109F070FB204657
:10195000012109F060FB0C2F10D8DFE807F0070F1A
:101960000F0F090F0F0F0B0F0F0F0D00343404E092
:10197000383402E03C3400E040347451A9F804A04B
:1019800048460BB0BDE8F08FD40500209CEA000863
:101990001F4A08B513881180C91A1E4889B240F63B
:1019A0008C22914203801C4B02D90020187008BD84
:1019B000A1F2EF2080B240F2DA5290421DD81B789B
:1019C000072B1AD81548032B20F81310144A09D8EE
:1019D00014480088884205D2012101FA03F31078E7
:1019E0000343137012780F2A07D10F480C4B02687B
:1019F0000021197011684B68984707480A4B027814
:101A0000511C0170186802681168884708BD00BF42
:101A1000B6060020C005002010070020C4050020E5
:101A2000C205002002000020901100207FB504466E
:101A300001A80D46164609F0E6FA00200123ADF88C
:101A40000A00ADF80C0001A92046ADF80450ADF82D
:101A50000660ADF8083009F057FB7FBD2DE9F7436C
:101A6000DFF858800501144E05EB0804A368894689
:101A7000761928210746B271606802228DF8061097
:101A800001A9ADF804308DF8072003F09FFA55F84E
:101A90000800217B0022FFF7C9FF204601224FF6F4
:101AA000FF7100F0DFFB204639464A4600F09AFB02
:101AB0003046BDE8FE8300BFD40500209CEA000844
:101AC00010B5144B00011B18DA795AB9012219819B
:101AD000DA71114B02221918097B1858BDE8104021
:101AE000FFF7A4BF1C8959810C4A091B9C7989B254
:101AF00022F8141000229981DA71074B1918097B1A
:101B00001858FFF793FF064802681368196888475A
:101B100010BD00BFD40500209CEA0008C4050020C9
:101B2000901100204B4B2DE9F0410446028A1960C8
:101B30004948A17965780280002914BF022700274F
:101B400005B10137454B002553F827707A5DFF2A10
:101B500002F00F0002F0F00308D122894048414909
:101B6000B2F5FA7F016070D8BDE8F081A17811B1BB
:101B7000811E012965D9E17811B1011F032960D9BE
:101B8000E17909B181425CD012F0300F03D02278A4
:101B9000002A08BF0023217931B1A27922B9A0F12E
:101BA0000801012998BF802362792AB1A17919B966
:101BB000021F032A98BF802303F01001CAB23AB172
:101BC00000222949FFF74AFF284B08221A7038E003
:101BD00003F02001CAB242B1244E25493278FFF702
:101BE0003DFF3078411C31702BE003F04001CAB258
:101BF00092B123891F4AB3F5FA7F94BF01210821CE
:101C00004A431D4EB2FBF3F39AB2A38996F80080C3
:101C1000FFF724FE194B0EE01B0612D56389154908
:101C2000174E91FBF3F292B2E389012196F80080FE
:101C3000FFF714FE134B43F8280008F1010886F85B
:101C4000008001350E2D81D187E70F4B0360BDE881
:101C5000F08100BF901100200200002058EA000827
:101C6000BC0600204D18000891190008B906002094
:101C7000C11A000840420F00B8060020C00600202C
:101C8000B4060020F00600202918000808B5044B0F
:101C90001A78824202D9034B1A68904708BD00BFE8
:101CA000B8060020BC060020044B1A78824204D9F2
:101CB000034B53F82000026811807047B4060020DF
:101CC000F0060020014B33F810007047C4050020D7
:101CD000704701717047426A806A131A594251EB8A
:101CE00003007047037913F001010BD0026AC36946
:101CF0009A4205D09CBFC0681218D01AC0B2704773
:101D00000020704708467047037910B513F00101B1
:101D100004460ED0FFF7E6FF60B1E3696269E1684F
:101D2000D05C4A1E934201D2013300E00023E361FC
:101D300010BD084610BD03799A070AD5436A826927
:101D4000D154416A03694A1CB2FBF3F103FB11222F
:101D50004262704790F842321BB1D1F1010138BFA5
:101D60000021D0F834014268836809B113617047DB
:101D70005361704707B5034699684822ADF80410CF
:101D80000223406801A98DF806208DF8073003F082
:101D90001DF90EBD58B50E4B044618680E46034695
:101DA000B3FBF2F1B1F5803F03D3012BF8D95B0807
:101DB000F6E7084A89B2B0FBF2F3DAB2204600F047
:101DC00051FA054A20463146BDE8584000F00ABAAB
:101DD0004C01002040420F004D2100087FB5044611
:101DE00001A80D46164609F00EF900200123ADF8B2
:101DF0000A00ADF80C0001A92046ADF80450ADF87A
:101E00000660ADF8083009F07FF97FBD38B50446AB
:101E10000D46002A0CBF02220022217B0068FFF73A
:101E2000DDFF034A20462946BDE8384000F0DAB914
:101E3000E11F000807B5034699681022ADF80410A9
:101E40000223406801A98DF806208DF8073003F0C1
:101E5000BDF80EBD00F134034FF48072436100F50C
:101E60009C710023C2600362C3618161026183626D
:101E7000436270472DE9F0411D46194B0E46032180
:101E800003600171044690460127FFF7E3FF00203D
:101E900084F83C0284F83902A4F84402A4F846020B
:101EA00084F83872D4F8340184F84252FFF7C2FF44
:101EB000206BFFF75FFF39462046FFF74BFF3220CC
:101EC00003F071FBD4F8340131464246FFF762FF5C
:101ED000206B31462A46BDE8F041FFF797BF00BFAF
:101EE00084EA000810B5084A044608480B46026315
:101EF0001032C0F8342100212246FFF7BBFF044B0B
:101F000001201C60187110BDDCEA0008941100204B
:101F100014070020034607490748084AC0F878120A
:101F200012681031C0F87C1300F512700121FFF720
:101F3000A1BF00BFFCEA0008941100201407002094
:101F4000C268036A511E8B4201D3002300E00133B3
:101F50000362704710B590F83C220446AAB9836A20
:101F6000416A994225D080692169C05C01338B4266
:101F7000A36228BFA26242000A2342F4007084F8E0
:101F80003D32A4F83E02012311E090F93D3273B1D5
:101F9000B0F83E124A08A0F83E2201F00101FFF716
:101FA000D9FE94F83D02431E84F83D3210BD84F8FA
:101FB0003C3210BD90F83B3210B583B990F83A32FC
:101FC00090F8392293420AD2012101FA03F1B0F8C4
:101FD000404201332143A0F84012DBB2F2E710BDCA
:101FE0002D4B10B54FF4127404FB00342079C10757
:101FF00051D594F8381221B3236B0021186809F0E9
:1020000051F894F83C1221B1B4F84402421CA4F8EF
:102010004422236B94F842221868197B002A14BFCB
:1020200002220022FFF7DAFE0020012184F83B1291
:1020300084F8390284F83A02A4F8400284F838029D
:1020400010BD94F83B222046012A04BF94F839229F
:1020500084F83A22FFF7AEFF94F83B02236B58B99D
:10206000012094F8422284F83B021868197B002A68
:1020700014BF022200220AE0002184F83B1294F8E7
:1020800042221868197B002A0CBF02220022BDE8F8
:102090001040FFF7A3BE10BD9411002090F83B1232
:1020A00000230122012980F8393280F838220CD12E
:1020B00080F83B32036B90F84222197B1868002AA3
:1020C0000CBF02220022FFF789BE70470279034647
:1020D000D20713D5B0F8402202F4007189B209B9D1
:1020E000D10705D4B3F84602421CA3F84622704734
:1020F0004169036A5208CA54FFF722BF704710B5FE
:1021000090F838320446002B1ED190F839124A1C40
:10211000D3B2092B80F8393203D1BDE81040FFF764
:1021200049BF0A2B10D190F83B0228B9B4F84012ED
:1021300041F00102A4F840222046FFF7C7FF2046E5
:10214000BDE81040FFF7AABF10BD0000064B10B558
:102150004FF4127404FB00342046FFF7FBFE2046C8
:10216000BDE81040FFF7CBBF9411002030B500242C
:102170000E4D55F82450854202D00134E4B2F7E701
:10218000A400E4B200200A4D2D5C8D4202D0451C13
:10219000E8B2F8E70019C0B20F2805D8054C04EBE7
:1021A000001083600171027330BD00BF7CEB00083A
:1021B0008CEB0008241600200C2912D8DFE801F06F
:1021C00007111111091111110B1111110D0002212B
:1021D00004E0042102E0082100E01021012208F0BF
:1021E00034BF704738B504460D461346217B00685E
:1021F0002A46FFF7BBFF2068217BBDE83840FFF788
:10220000DBBF07B58DF80400012000238DF8060020
:102210008DF8070001A88DF8053008F0F5FC0EBD1B
:102220007FB5044601A80D46164608F0D9FE0B4BB3
:102230000B485E4301680023B1FBF6F2013D561ED8
:10224000204601A9ADF80850ADF80460ADF80A3099
:10225000ADF8063008F07CFD7FBD00BF40420F00A6
:102260004C01002010B504460068FFF7D9FF206834
:10227000012108F0D0FE607BBDE81040FFF7C1BF30
:1022800000230C4A52F82320824202D05A1CD3B2B7
:10229000F7E79B00D8B20023074AD25C8A4202D0FB
:1022A0005A1CD3B2F8E71818044BC1B203EB011063
:1022B000704700BF7CEB00088CEB00082416002060
:1022C00070B5044600262E4BF55C95B902212046D8
:1022D00008F0C3FF01284FD12046022108F0C8FFB3
:1022E00029462046FFF7CCFF0546204608F0A8FF08
:1022F0003DE0042D12D12046294608F0AEFF01280A
:102300003AD12046294608F0B3FF29462046FFF778
:10231000B7FF0546204608F096FF28E0082D12D1A9
:102320002046294608F099FF012825D12046294654
:1023300008F09EFF29462046FFF7A2FF05462046EB
:1023400008F084FF13E00C2D16D11021204608F070
:1023500084FF012810D12046102108F089FF29466A
:102360002046FFF78DFF0546204608F072FFAA6859
:1023700001460AB1287B90470136042EA3D170BDD7
:102380008CEB00080148FFF79BBF00BF002C014009
:102390004FF08040FFF794BF0148FFF791BF00BFA7
:1023A000000400400148FFF78BBF00BF0008004059
:1023B0001D481E49026800608A4200F01F8000210B
:1023C00000F004B81A4B5B584350043119481A4BBB
:1023D00042189A42FFF4F6AF184A00F003B80023FF
:1023E00042F8043B164B9A42FFF4F9AF08F0DEF9CD
:1023F0000BF02CFA01F00AF8FFF7FEBF114E12485D
:1024000030601248016821F0706101604102016092
:102410000F4C182020600F490F4808600F48D0F873
:1024200000D0406800470000F04F0020EFBEADDE56
:1024300074110108000000209C0500209C0500206C
:10244000781D00201810024009000000040001401F
:10245000140C0140000C01404434434400F0FF1FC1
:10246000FFF7FEBF014B186802F0EBBD681D0020AE
:102470000149002000F074BE6524000810B5FEF785
:1024800045FB0A49FEF796FB0949FEF747FC094B55
:10249000044618680078FEF739FB01462046FEF72F
:1024A00089FBFEF773FD80B210BD00BF333353408C
:1024B00000F07F453007002038B50D4C002025780E
:1024C000FFF704F90B4A05F0070322F81300013562
:1024D000002325701846D15A02334018102B80B2C1
:1024E000F9D1C008FFF7CAFF034A107038BD00BF1A
:1024F0001C0700201E07002024170020074B084A55
:1025000019781088884207D3064B1A689078884259
:102510008CBF002001207047002070472417002046
:102520002617002030070020124B70B518602024B9
:1025300000250020FFF7CAF82D180A2003F033F811
:10254000013CF6D1C5F34F10FFF798FF094902236C
:102550000A6851784D006619B04203D30133062B47
:102560000C44F8D1044892780370534303490B801C
:1025700070BD00BF30070020040000202617002097
:102580002DE9F04F0446008885B048B9B4F902300F
:1025900043B9B4F90420D2F1010138BF002102E0AF
:1025A000002100E0014611F0010377D13D4D00B25A
:1025B0002B7000F005FD0646B4F9020000F000FDA6
:1025C0000546B4F9040000F0FBFC0446304609F06F
:1025D00095F90746304609F005FA8046284609F085
:1025E0008DF90646284609F0FDF90546204609F012
:1025F00085F98246204609F0F5F93946814650466C
:10260000FEF7D8FA394683464846FEF7D3FA5146D4
:1026100001904046FEF7CEFA494602904046FEF74A
:10262000C9FA314603905046FEF7C4FA1E4C49469B
:10263000206006F10040FEF7BDFA29466060A56003
:102640000298FEF7B7FA01460198FEF7ABF9294662
:10265000E0600398FEF7AEFA01465846FEF7A0F98F
:102660003146206108F10040FEF7A4FA2946606176
:102670005846FEF79FFA01460398FEF791F929465E
:10268000A0610198FEF796FA01460298FEF78AF9D2
:102690003946E0613046FEF78DFA206205B0BDE8AC
:1026A000F08F00BF05000020340700202DE9F8431B
:1026B0004D4B0C460168013A196080889880072AC2
:1026C00030D8DFE802F004080F14191E22261888FB
:1026D00020805A8803E0598821801A8852426280FB
:1026E0009A881EE01988484220805A88F6E759885F
:1026F000484220801A88F2E719884842208058888A
:102700000CE05A882280188808E0198821805A88AD
:1027100003E05988484220801A88504260809B8894
:102720005A42A280314B1A78002A5AD1B4F90000DB
:10273000FEF7ECF98046B4F90200FEF7E7F9074628
:10274000B4F90400FEF7E2F9294D0646296840462F
:10275000FEF730FAE96881463846FEF72BFA014663
:102760004846FEF71FF9A96981463046FEF722FA6E
:1027700001464846FEF716F909F0F4F8696820802A
:102780004046FEF717FA296981463846FEF712FAE5
:1027900001464846FEF706F9E96981463046FEF7EC
:1027A00009FA01464846FEF7FDF809F0DBF8A9688A
:1027B00060804046FEF7FEF9696980463846FEF7BC
:1027C000F9F901464046FEF7EDF8296A074630461A
:1027D000FEF7F0F901463846FEF7E4F809F0C2F8D2
:1027E000A080BDE8F88300BF580700200500002046
:1027F00034070020F8B5154C06462378274663B900
:1028000002F0C0FE124D2A683232904205D30123F5
:10281000237002F0B7FE2860F8BD3878A0B102F04E
:10282000B1FE0B4C2168731898420DD30748002263
:10283000027002F0A7FE074920600B780BB15A1E08
:102840000A70054901200870F8BD00BF5E0700202E
:1028500068070020610700206207002037B58DF867
:1028600005101F498DF807300B788DF8040002A879
:102870008DF80620C21812F8044C0D46443CE0B214
:102880000A2828D81749022B31F8104003D814B170
:102890002046FFF7AFFF2B78022B0BD9124D2D6886
:1028A00002F070FE021B954204D20D490F4B00202E
:1028B000087018700E4802780146012A00D074B9D9
:1028C000074B1878022801D8421C1A7000230B709D
:1028D00008490B7003E03224022BD9D9DBE73EBD57
:1028E0005F07002090EB00086807002061070020C8
:1028F000620700205E070020014B1860704700BF90
:102900009011002070B53D4B04465A7B3C4802B103
:10291000012202704FF4007000F052F9002828D014
:10292000384E394B316858780D68003018BF012097
:10293000AA68904748B13368344D1868012102698C
:102940002970904708B1022129702E4D2B68186814
:10295000C268904728B12C494B7813B92B4A022002
:10296000107029680B689869804710B127490022C8
:102970000A70202005F04EF960B12048244B827A7D
:102980000AB9C17A21B12048C27A0AB9012100E00E
:10299000002119701D4B1878022802D14C204E21BD
:1029A0001DE0012807D14D2153204C220B46BDE8E4
:1029B0007040FFF753BF164A1178012903D1532005
:1029C00001464E2206E00E4B1878012804D1532010
:1029D000014602464D23EAE724B153204D210A4621
:1029E0004423E4E70B4A117821B13220BDE870405E
:1029F000FFF700BF084B1C7070BD00BFF41C002027
:102A00006307002090110020E31C002060070020D5
:102A100064070020610700205E0700200E4B1A7833
:102A2000402A16D15888B0F5667F12D11979BE298F
:102A30000FD193F895230020EF2A0CD113F8011B36
:102A4000064A48409342F9D1D0F1010038BF002036
:102A5000704700207047704700F8010898FB010894
:102A600010B50C4C204605F089F90B4B2046B3F805
:102A7000D010B3F8D2201F3C05F09AF914F8B40B2B
:102A800001F07AF904F0B4F82046BDE8104000F0F7
:102A90006BBC00BF4B170020F817002010B5FFF7E4
:102AA000BDFF10B90A2002F0EFFD0E4C0E49204682
:102AB0004FF466720AF014FF94F89433022B02D993
:102AC000002084F8940394F89413CC2202FB014371
:102AD000064803F598710AF003FFBDE81040FFF7C0
:102AE000BFBF00BFF817002000F801082C17002016
:102AF00008B5FFF7D3FF0F2014210122BDE80840DD
:102B000007F03ABE08B5054BCC2202FB0030044961
:102B100000F598700AF0E4FE08BD00BFF817002029
:102B20002C170020224A38B5402313704FF46670EA
:102B30000023BE21EF245080117182F8954382F862
:102B400096331D461A4A985C0133B3F5667F85EAD1
:102B50000005F7D182F8965308F016FC04250024EE
:102B6000691E11F0FF0516D0342008F021FC114831
:102B700008F074FC0F4C04280BD10F4A2046A158D2
:102B800008F042FC0D4B04349C42F4D10428044666
:102B900001D00446E4E708F003FC042C02D1FFF75F
:102BA0003DFF20B90A20BDE8384002F06DBD38BDB8
:102BB000F817002000F80108F81FFE1798FB01081D
:102BC000034B996808420CBF00200120704700BFEA
:102BD000F8170020024B9A6810439860704700BFB6
:102BE000F81700202DE9F347B74AB84D106851682F
:102BF000B74C6B4603C34FF46672002128460AF0B7
:102C00001DFFCC22002120460AF018FF402003219E
:102C1000287002206971FFF7DDFFFA22A5F8F22083
:102C20002A236E22A5F8EE304FF4FA7085F80421BD
:102C30002B2340F24C42A5F8F60085F805312120FF
:102C400002F54873202185F80601A5F8163140F2F7
:102C50007E404FF47A7300274FF001094FF4167647
:102C600085F8F410A5F8142140F2DC5100F52F721C
:102C7000A5F8D00003F5CB70A5F8F060A5F8121107
:102C8000A5F8D22085F89473A5F8F870A5F8FA7025
:102C9000A5F8FC7085F8E27085F8E37085F8E470BB
:102CA000A5F8E670A5F8E870A5F8EA7085F8ED706B
:102CB00085F8EC9085F8077185F82C7185F82D71F1
:102CC00085F82E7185F8107185F8187185F81971DD
:102CD00085F81A91A5F8D430A5F8D6006C30A5F87F
:102CE000D8004FF4C870A5F8DE004FF41650322318
:102CF00040F2B452C5F8240140F6AC50A5F8DA20F1
:102D0000A5F8DC301A46A5F8E030A8814FF4E1338D
:102D10001E20C5F82031E07252232073552085F81B
:102D20002A31E07017230B204FF028086375A37534
:102D300060712D2314204FF0080E63732271A0716F
:102D400085F81C7185F81D7185F8287185F8297141
:102D5000AF7385F81B71277084F8018084F80280B6
:102D6000E775A7732776E773677684F810E06074D9
:102D70005020E076E1845A200421A3762072237546
:102D8000E077412384F82E10524853494FF00E0A41
:102D900084F82030514B84F807A04FF0640C4FF0BA
:102DA0000A0A4FF0780E84F8212060631522E1634F
:102DB0004B4805F5847184F83120A36384F812A090
:102DC00084F81CC084F8098084F80AE084F81E9016
:102DD00084F8237084F8247084F8257084F82270B5
:102DE0006785A785278584F82F8084F8308084F84C
:102DF000409005F01BF84FF44872C8204FF49663DA
:102E000040F2D9313E4684F86C7084F86D7084F8D5
:102E10006E8084F86F9084F87270A4F8702084F843
:102E2000B4A084F8B500A4F8B630A4F8B8104FF4F4
:102E30007F724FF4FA601DF80710A4F87420A0F513
:102E4000FA73FF220137A4F87600A4F8783084F8EA
:102E50007A1084F87B200834082FE8D11C4C01201C
:102E6000C823142184F8BA0084F8BB0084F8BC009D
:102E7000A4F8BE3084F8C01084F8C2001E2264207A
:102E80004FF49673282184F8C120A4F8C400A4F854
:102E9000C630A4F8C81000240C4A0023A01810342F
:102EA000C02C0361F8D100240E49CC2260180849D7
:102EB000CC340AF015FDB4F5197FF5D102B0BDE8A8
:102EC000F047FFF72FBE00BF34EA0008F8170020D4
:102ED0002C1700209A99193F3D0A773FF6287C3F2E
:102EE000A6EB00082819002008B5FFF797FD18B9D0
:102EF000BDE80840FFF776BE08BD0000024B9A68A7
:102F000022EA000098607047F8170020014B98688B
:102F1000704700BFF8170020884203DB8242B4BF2D
:102F200011460146084670470023036170472DE9AA
:102F3000F041066904460136012E0D46066105D1B1
:102F40000023616021608360BDE8F081D0F80080DB
:102F500008464146FDF724FD07463046FDF7D6FDFD
:102F600001463846FDF7DAFE01464046FDF71AFDF8
:102F70000646606031462846FDF712FD0146384698
:102F8000FDF718FEA168FDF70DFD2660E060A0606A
:102F9000BDE8F08110B504460069012807DD01385D
:102FA000FDF7B4FD0146E068FDF7B8FE10BD002056
:102FB00010BD08B5FFF7EEFFBDE8084008F0A0BD62
:102FC00008B5FDF721FA04A3D3E90023FDF782FA3F
:102FD000FDF792FC08BD00BF399D52A246DF913F2C
:102FE0002DE9F041069C06460F46002B0CBF4FF022
:102FF00020084FF03008204610F8013B0BB9154669
:1030000003E0002AFBDD013AF6E7002D04DD30463F
:103010004146B847013DF8E714F8011B11B13046AD
:10302000B847F9E7BDE8F0812DE9F04389B00646DD
:103030000F4603921C46039A134613F8011B039391
:10304000002900F08A80252901D0304683E0002045
:1030500004905578911C302D039105D19578033259
:1030600003924FF0010800E08046A5F13003D8B28A
:10307000092806D8284603A90A2204AB00F00CF957
:1030800005466C2D05D10399012211F8015B0391CE
:1030900000E00022642D2FD010D8582D3AD006D849
:1030A000002D5AD0252DC6D13046294653E0632D38
:1030B000C1D130462178251DB8474AE0752D0DD085
:1030C000782D27D0732DB6D1251D24683046009465
:1030D0003946049A0023FFF783FF3AE0251D206854
:1030E0000A2122B1002205AB00F060F802E005AB36
:1030F00000F08CF82C4623E005AD04F104092068AB
:10310000294612B100F077F801E000F0A4F84C462F
:10311000009517E004F104092068102142B1B5F1CF
:103120005804634253EB040205AB00F03FF806E09D
:10313000B5F158035A425A4105AB00F067F84C46C6
:1031400005A8009030463946049A4346FFF748FFE9
:1031500071E72C466FE7B8476DE709B0BDE8F0832B
:10316000024B196002490860704700BF6C070020DD
:10317000700700200FB407B5094904AB0868094976
:1031800053F8042B09680193FFF74EFF064B1868AC
:1031900001F076FF0028F9D0BDE80E4004B070477A
:1031A000700700206C070020681D0020F0B5012486
:1031B000B0FBF4F58D4201D34C43F9E70026C4B1CE
:1031C000B0FBF4F504FB1500B4FBF1F41EB9002DBF
:1031D00001DC002CF4D1092DEFB204DD002A0CBF74
:1031E0005725372500E03025ED1903F8015B01363E
:1031F000E5E71C70F0BD00280B4603DA2D224042A3
:1032000003F8012B0A210022FFF7D0BFF0B50124FB
:10321000B0FBF4F58D4201D34C43F9E70026C4B16D
:10322000B0FBF4F504FB1500B4FBF1F41EB9002D5E
:1032300001DC002CF4D1092DEFB204DD002A0CBF13
:103240005725372500E03025ED1903F8015B0136DD
:10325000E5E71C70F0BD00280B4603DA2D22404242
:1032600003F8012B0A210022FFF7D0BFA0F13003A1
:10327000DAB2092A01D818467047A0F16101052980
:1032800001D857387047A0F14103052B01D83738D2
:1032900070474FF0FF3070472DE9F8430D68044642
:1032A0000F469046994600262046FFF7DFFF00288C
:1032B00006DB404504DC08FB060615F8014BF3E786
:1032C0003D602046C9F80060BDE8F883014B00224C
:1032D0009A80704774070020034BB3F90400D0F1C3
:1032E000010038BF00207047740700200649074BD3
:1032F0000A68B3F90400137805214B439842D4BF00
:1033000000200120704700BF7C07002074070020C8
:1033100010B50446FFF7EAFF002814BF204600203E
:1033200000F0010010BD0000074B084A1968B2F90F
:1033300004004B780A78D118052251438842D4BF43
:1033400000200120704700BF7C0700207407002088
:10335000044B9A8811B2142901DD143A00E00022CE
:103360009A80704774070020024B002218600248C0
:10337000828070477C07002074070020034B0449BB
:103380001860044800220160C28070478007002056
:10339000B0EB00087407002008B502F091F9024B69
:1033A00000221A7008BD00BFE31C002010B5FFF713
:1033B0009DFFE0B1104B5C78201C18BF0120FFF787
:1033C000A7FF70B10D480E4B01680E484A8901688D
:1033D0001A805A809A804A88DA800B4BD888411C20
:1033E000D980FFF7A1FF00B90CB9FFF7D5FF064B55
:1033F0009A88501C988010BDE31C00208007002094
:10340000241D00207C0700207407002010B57A4C92
:1034100086B0A07B003018BF012002F0CFF8FFF784
:1034200027F8FFF761FDFFF739FB94F8073133B157
:10343000012B01D0092B02D18DF8003004E00021CE
:103440008DF8001084F807116846FEF7C9F86B483C
:10345000FFF796F8022004F0E7FB02F0F1FD664A60
:1034600054790E2C01D0082C01D1012000E000205D
:103470008DF80A004FF48070FFF7A2FB18B90820FE
:10348000FFF79EFB00E0012000F0010340208DF8D3
:103490000630FFF795FB8DF807000120FFF790FB42
:1034A0008DF805000820FFF78BFB80F001018DF8F7
:1034B000041003F015FA524A8DF8080092F8BC4047
:1034C0004FF47A72C4F380004B4C8DF80900B4F8C5
:1034D000DE30B4F8E0104FF48040ADF80C30ADF8B9
:1034E0000E10ADF81020FFF76BFB18B1B4F8DA003E
:1034F000ADF81000BDF80C30B3F5FA7F02D9002109
:10350000ADF810103E48B4F8122194F80741B0F815
:10351000B830012CADF81220ADF8143004D0092CCD
:1035200001D1072400E0002436488DF80B40FFF756
:1035300025FF354C2060FFF7DFF901A82168FEF771
:10354000F1FA3048216804F09FFB4FF48070FFF7D8
:1035500037FB40B10820FFF733FB20B9264991F82B
:103560001D0103F097FB0A24192002F01CF8192012
:1035700002F019F8621E12F0FF04F5D101F012F901
:1035800002F022F90220FFF71BFB10B11F48FEF7E3
:10359000CBFF1F4805F022FA4020FFF711FB50B186
:1035A000154CD4F8240194F82811FEF79BFC94F8EC
:1035B0002901FEF7AFFC4FF40060FFF701FB10B1EB
:1035C000144804F0EFFE01F0C3FF134B18600A48E3
:1035D0004179052903D1114C4FF4C8722280104B58
:1035E0004FF47A7018800F4A0F48C82101241180C7
:1035F000447300F0CFFBFCE7F8170020DE18002032
:103600002C1700200019002090110020FC18002029
:1036100018190020681D0020AC07002018080020A1
:10362000800800202C0C0020E31C002008B5034B70
:10363000B3F9D40002F020FEFEE700BFF817002027
:103640002DE9F04F794B0024B3F902A0B3F9000043
:1036500087B0BAF1000FB8BFCAF1000A0028B8BF9E
:1036600040428245B8BF82462546A046274605947B
:10367000A14626466E49CA7812B90B79002B40D074
:10368000022E3ED06B4B6C486849B0F8F620685E5D
:10369000E95EDFF8B4B101EB40005142FFF73CFCBA
:1036A000664A05EB0B0335F902C0B3F92A10CCEBDF
:1036B00000009BF8082000EB010902FB09F09BF8D1
:1036C0001C30642190FBF1F005226FF00401594396
:1036D0005A43CDF81090FFF71FFC594BDDF810C08E
:1036E000E258584981460CEB020042F210720493F2
:1036F000FFF712FC04999BF81230605058430013F6
:1037000005904B49CA781AB10B790BB9022E30D10A
:10371000464F4D48EF5F5021794306EB000B9BF875
:1037200001204A4BDFF83C8191FBF2F0E95E54F84E
:103730000820401A801846494FF47A520493FFF744
:10374000EBFB049B48F80400E95E0029B8BF49423E
:10375000B1F5207F02DD002048F8040058F804206D
:103760007D239BF80B1092FBF3FE01FB0EFC4FEA4E
:10377000AC182F480279A2B1022E12D00AFB07F131
:10378000CAF5FA7303FB09104FF4FA7190FBF1F2DA
:103790000AFB08F0DDF814B003FB0B0393FBF1F315
:1037A00008E0C3780BB1022E02D143463A4601E04D
:1037B000059B4A462549DFF8B0C0695A16F80CB097
:1037C00008B20BFB00FB6FF04F0C9BFBFCFB934420
:1037D000204ACDF804B035F902C0A952CCEB000064
:1037E0001D4ADFF888C0029054F80C10A058401809
:1037F000029903904018A15844F80C100299A15066
:10380000164A0434B15C202201FB00F090FBF2F177
:103810005B1A134A9B44013625F802B00235032E89
:103820007FF428AF07B0BDE8F08F00BFC41B0020B5
:10383000E31C0020F4070020F81700203C0C0020B7
:1038400008080020F0D8FFFF2C1700205E0C002095
:1038500080C1FFFFBC070020A0070020121C002031
:10386000CC1B002088070020151C0020B00700207A
:103870002DE9F74F002425462646A246474BDA7825
:103880000AB91879C8B1022E19D0454B45484649A6
:10389000B0F8F6206F5EE85E514200EB4700FFF79C
:1038A0003BFB424A424F35F902A0EB19CAEB00013B
:1038B000B3F92A0001EB000A0BE0022E09D13C49C2
:1038C000394B91F82470B3F904201B3757437B110F
:1038D00016E03249364ACF7877B9334892F82370E8
:1038E0002B5E1B375F4309793B1149B1927C02FB88
:1038F0000AF703EB272303E0137A03FB0AF0031113
:103900002C48DFF8C8B0295EBBF800005F1A284BCE
:10391000784306EB030898F80120DFF8B4907A4367
:1039200098F80B104FEAE21C54F80920C31201FB6F
:103930000320214944F809004FF40012CDF804C0D7
:10394000FFF7EAFA1D4B4FF6FF72E158E750791A7C
:10395000BBF8007044F809003B09B2FBF3F74F4392
:10396000174A184B54F80290E158BF11A750494428
:1039700098F81520C9194A43DDF804C012490CEB28
:10398000603044F80390013600EB22236B5204347C
:103990000235032E7FF472AFBDE8FE8FE31C0020DA
:1039A000F4070020F8170020C41B00203C0C002066
:1039B0002C1700205E0C00200000E0FFE407002030
:1039C000FC070020C4070020CC1B0020F8070020C3
:1039D000880700200B4B0C481A8852B9817841B1F6
:1039E00042786AB9012141700848094B02881A805F
:1039F0007047437823B90220FF21012206F0BCBEA4
:103A0000704700BF80080020E31C00204E1C0020EF
:103A1000101C00202DE9F04FA94BAA4AB3F906006B
:103A2000D18C85B088420FDBB0F5FA6F92F8254053
:103A300007DA451A6C43A1F5FA6694FBF6F4643490
:103A400003E0C4F1640400E064249F4A9D4BB2F893
:103A5000127192F9EC2093F823100097574293F8D3
:103A60006C50019193F86D60B9B293F824300291D3
:103A7000002103930A46924FDDF8008031F907C018
:103A800040F2E637C8EB0C0303F2F31EBE4503D841
:103A9000002BB8BF5B4201E04FF4FA73022ADFF853
:103AA00034822CD025B1AB42CCBFC5EB030300233D
:103AB0006427DFF84CA293FBF7FE6FF0630B3AF834
:103AC0001E900BFB0E3B0EF1010E3AF91EA00FFAF1
:103AD00089FECEEB0A0E0EFB0BFE9EFBF7FEF144B9
:103AE00028F80190DDF8048003FB08FE774B9EFB6D
:103AF000F3F3DB199BB2634393FBF7F712E026B1B4
:103B0000B342CCBFC6EB03030023029F5F43A8F878
:103B10000470039F002BB8BF5B427B436B4F93FB4A
:103B2000F7F76437674B02EB030E9EF801906423AE
:103B300007FB09F898FBF3F9DFF8C88102F8089051
:103B40009EF80B909EF815E007FB09F807FB0EF7AF
:103B500098FBF3F9DFF8B08197FBF3F302F80890D4
:103B6000DDF800805A4FC445D35503DA594BCF5A7C
:103B70007F42CF5201320231032A7FF47CAF524C94
:103B80004FF4FA62B4F81411FFF7C6F9B4F81461EF
:103B90004FF47A75801B4543C6F5FA63B5FBF3F520
:103BA00064214D4895FBF1F36FF0630630F8132064
:103BB00006FB0355013330F9130013B2C01A454315
:103BC000464B444C95FBF1F1587A8A18E280002864
:103BD00038D0434F434D3E882988721A10B2FFF700
:103BE000EFF9074607F08AFE0646384607F0FAFE68
:103BF0000546B4F90200FCF789FF0746B4F9000056
:103C0000FCF784FF31468046FCF7D4FF2946814605
:103C10003846FCF7CFFF01464846FCF7C1FEFDF7EA
:103C20008FF9314620803846FCF7C4FF2946064606
:103C30004046FCF7BFFF01463046FCF7B3FEFDF7F8
:103C40007FF960800220FEF7BBFF90B12648062274
:103C50000378591CCBB20370B3FBF2F002FB1031B6
:103C600011F0FF0F05D1FEF727FCFEF747FC1F4BB5
:103C700018701E4A1078003018BF0120FEF742FE6F
:103C80001B490B882BB91B4A108838B904F066FB16
:103C900004E0022003F0BEFF0028F4D01649174AC2
:103CA00009681368C81A002832DB0C4B587B68BBC4
:103CB000987001F5F42303F59070106028E000BFC0
:103CC000241D00202C170020F81700200CFEFFFFF9
:103CD000121C0020C41B00200C1D0020E31C00202F
:103CE0004E1C0020101C002095070020D407002047
:103CF000180800208008002010080020D0070020AD
:103D0000481D0020151C0020081C0020012199706E
:103D100004F070FE124A117831B94FF40060FEF7DA
:103D20004FFF08B104F062FB202003F073FF78B16D
:103D30000C4B18680C4B1A68811A002908DB0B4AD7
:103D40001178042904D900F5123000F5F8721A60D0
:103D5000074B996809B10748884705B0BDE8F08F5F
:103D6000F810002010080020E00700200E1C0020A2
:103D70003C1C0020A41B00200128034B14BF034A55
:103D8000034A1A60704700BF08000020413600084F
:103D90007138000838B50820FEF712FF90B1A04B2B
:103DA00093F8100103280CD8DFE800F002020508A0
:103DB00004F082FA06E004F0CBF803E004F086F9A0
:103DC00000E000209749984A0B681168591A0029A9
:103DD00002DA002800F0A48203F59C4493482034C2
:103DE0009349146003F072FF4FF48040FEF7E8FE41
:103DF00020B1904D2B780BB901F062FC884A92F803
:103E00001B11B1B18C4CC81C34F910504FF47A72AC
:103E10000021A5F57A70FFF77FF8FCF777FE874958
:103E2000FCF77CFF8649FCF7C5FEFDF7AFF8854B34
:103E300018804FF40070FEF7C3FE20B1824A11686B
:103E400008684469A047764D0022B5F81401B5F81A
:103E50001641134678499B08555E8542C4BF63F0FE
:103E60007F03DBB2A542B8BF43F040030232082A09
:103E7000F0D17648764A047805469C4204D1107801
:103E8000F92803D8411C00E0002111704FF4804054
:103E90002B70FEF795FE68B1614D674BB5F81211B6
:103EA000B5F8DC20B3F90640881A844202DD8B188D
:103EB0009C420CDB4FF48040FEF782FEF8B95E4C6A
:103EC0005749B4F90650B1F81421954217DA614DFB
:103ED0006148624CB5F84210002303604360836080
:103EE0002360636059B1534A5D4B1078002800F09D
:103EF0007E821C78002C00F07A82FFF76BFD54491B
:103F00000A78142A40F0DD8055484478ECB1514AD3
:103F1000B2F842502DB94D4908785F2801D101F01F
:103F2000CFFB3F4C94F81831002B00F0CA80494A6F
:103F3000B2F84250002D40F0C480444908787D28F2
:103F400040F0BF8001F0BCFBBBE0404D2B78572B0D
:103F500018D1444C4FF47A724FF480702280FEF7EF
:103F60002FFE08B102F0F2FD042003F053FE10B161
:103F70003D490A250D80082003F04CFED8B93B4B83
:103F8000188018E00420FEF71BFEA0B129785A29FA
:103F900011D1374802781AB10470364B012009E07C
:103FA000354C364B257885F00101217009B102208E
:103FB00000E003201870254802785D2A00F01E8278
:103FC0005B2A00F01D825E2A00F01C822148B0F8B6
:103FD000422032B91D4C25786F2D02D1FFF7FAFC33
:103FE00015E00F49194B91F8180118B112B91A7858
:103FF0007E2AF3D01C78972C04D1214B4FF4C87043
:10400000188004E0A72C02D1154901258D730F4AB1
:104010001478BB2C36D10F4CA18D8D1C37E000BF1E
:10402000F817002010080020F007002000190020D9
:104030000A1D0020F41C0020241D002000007A44EA
:1040400000C07F440C1C002090110020D8070020E5
:10405000D90700202C17002088070020080800201E
:10406000E31C0020800800202C0C00204E1C0020A7
:10407000940700209C070020C20700206107002051
:1040800018080020B72C04D1904CA28D951EA58550
:104090000BE0BE2C03D18D4D6B8D981C04E0BD2C24
:1040A0000FD18A4D698D881E68858948002490F853
:1040B0009403FEF727FDFEF735FDFEF719FD854B4E
:1040C0001C700420FEF77CFD00282CD0824C237845
:1040D0008BB1824A557875B181497D4BB1F90600A3
:1040E000B3F81421904206DD7E4D2B781BB97E4932
:1040F0003220088023707B4C627C52B17B4D2A7841
:104100002AB97B4B187810B9774C322121800124D1
:1041100008E0774D2B7833B17048417819B9297090
:10412000744D01242C700023734C1A4634F8020F8E
:1041300040F2135501B2A942CCBF0025012505FA72
:1041400003F5A0F21550B0F5C77F8CBF0020012009
:104150002A435D1C00FA05F0024340F2A46081424C
:10416000D4BF00210121981C01FA00F103330A4356
:104170000C2B92B2DAD1002354485A4900EB430089
:10418000B0F8420002420CBF002001205854013315
:10419000152BF1D14A7822B1022003F03BFD68B91A
:1041A00015E04FF40070FEF70BFD80B1534908682D
:1041B0000368DA6890470028EED108E0474AD378D0
:1041C00043B94F4901200B604B60D07002E0434877
:1041D0000021C170434A414B917839B118790021CF
:1041E000D97020B9464A01211060506019713D4BC9
:1041F000187810B9394901220A70202003F00AFD0D
:10420000002852D0354BD87A1A46002848D03D496C
:104210000878042844D93348817A79B1DA79002AB8
:1042200043D139480121D9711A72384B011D1A70D6
:1042300002F088FD364A0220107036E0C27AD97149
:104240001AB322483349B0F8C820B1F90000002859
:10425000B8BF4042904218DAB1F902100029B8BF45
:104260004942914211DA187AF8B901241C72274B9D
:104270002949187029480A684B68011D026043608B
:1042800002F060FD224804700FE02048134B0178D3
:1042900000221A7249B90122027002F07BFC04E08C
:1042A0000023D37113721A4A13700E490B4B087B0B
:1042B00000B10120064A98725179082901D00E29CF
:1042C00052D1064B002058724EE000BF2C17002040
:1042D000F8170020D9070020C2070020E31C0020A7
:1042E000241D0020F41C0020D6070020FA0700201F
:1042F000940700209C0700202A1D00209011002018
:10430000080800200E1C0020D41B002006000020FE
:104310009D070020C41B0020F01B0020B41B0020C0
:1043200041480368042B1FD8DFE803F00305080B9E
:1043300017000122026001684B1C03600268511CD7
:104340000160394803685A1C02604FF48070FEF720
:1043500037FC10B102F090FD06E033480021016007
:104360004FF40050FEF72CFC01F0F2F82F4A3049D0
:1043700010608A892F4B1AB11968411A002951DB44
:104380008018186001F030FCFFF744FB01F0E0F802
:10439000294B264A196810601860421A2748284994
:1043A00090F872300A8053B12649CA780AB9087960
:1043B00028B1254B2549DA8808888118D980202022
:1043C00003F028FC40B11F4BD87908B91A7A1AB10A
:1043D000197B09B103F098FB1D4B1868804701F069
:1043E0005DFF01F0D9FEBDE8384001F031BF5D78D6
:1043F000002D3FF484AD01F063F980E5012402E073
:10440000022400E003240A4BE5B2691E83F89413EA
:10441000FEF788FBFEF742FB022028212A4606F021
:10442000ABF9D3E538BD00BF980700201008002085
:10443000F8170020DC070020AC0700202C17002014
:10444000F8070020E31C0020C41B00205C0C0020A7
:1044500008000020F8B5664B1D88002D40D00023D1
:104460001946B5F5C87F634A01D100205050624E0D
:1044700050589F5F5F4CC0195050604A00209853BD
:104480009E1802330431062BA6F8F800E9D1012D5D
:1044900022D121684FF4C87301F1C80191FBF3F1F7
:1044A000A2F8F8106168C83191FBF3F1A2F8FA1094
:1044B000A168C83191FBF3F3514909885B1A51494E
:1044C000A2F8FC304885888592F89403FEF71AFB21
:1044D000FEF728FBFEF70CFB45480288531E0380BD
:1044E0000420FEF76DFB00286FD047490A88322A66
:1044F00011D1424D454CB5F8F860B5F8FA00B5F861
:10450000FC30404926806080A3804D8D404C8E8DCC
:104510002580668001E0002A32D000231946322A25
:104520003C4801D100244450334D44585E5FA619E5
:104530004650324800245C531D1802330431062BC8
:104540002646A5F8F840EAD1012A16D1324B334964
:104550001A70334B0C70022119702C4B1988A0F87B
:10456000F81059889B88A0F8FA102949A0F8FC3067
:10457000244B0888498858859985234B013A1A802D
:104580002848017809B30022027022481B4B0468B6
:10459000322194FBF1F4A3F8F8404468806894FB5E
:1045A000F1F490FBF1F11648A3F8FA400088091ADB
:1045B0001448A3F8FC104285828593F89403FEF713
:1045C000A1FAFEF7AFFAFEF793FA0B4B0B4A1888E5
:1045D000B2F8F810401A1880B2F8FA105888B2F8F9
:1045E000FC20401A99885880881A9880F8BD00BF2E
:1045F00018080020280800206C1C0020F817002054
:104600000C0000202C170020D60700201A080020DC
:10461000200800203408002094070020FA0700201A
:10462000610700209C07002010B5074B074C596814
:1046300020468847064A204621461278FEF736F87B
:10464000BDE81040FFF706BF281C00206C1C0020AE
:10465000160800202DE9F84F414B188800286ED02D
:104660000024254626463E490A88B2F57A7F08D1BD
:104670003C4B3D4900271420EF5000FB0610FEF78D
:1046800053FCDFF8F0A0374F3AF90400EA59DFF89D
:10469000D8901318EB51FCF739FA4FF0140B0BFBC1
:1046A000069B01464FF000085846FEF740FC24F8F0
:1046B0000A80DFF8ACA02D48BAF8001024F800807A
:1046C000012933D15846FEF774FC294A834692F8F3
:1046D000F400E0B1FCF71AFA01465846FCF726FC54
:1046E000A8B14FF47A714846AAF80010FEF71CFCF6
:1046F00009F11400FEF718FC09F12800FEF714FC7C
:10470000C7F80880C7F80480C7F800800EE0154B92
:104710004FF47A72E858154B00F5FA7191FBF2F0FC
:10472000E0520F210A20012206F026F80136043556
:104730000234032E97D10A480288531E03800D4B82
:104740000A4A18881188401A188051885888928817
:10475000401A99885880881A9880BDE8F88F00BF61
:104760008008002084080020440800202E0C00202F
:10477000F8170020541C002010B5074B074C59684F
:1047800020468847064A204621461278FDF78EFFCC
:10479000BDE81040FFF75EBF3C1C0020541C002009
:1047A000900800202DE9F341524D53485349B5F884
:1047B000EE20FCF70FFE044618B1514D01242C7079
:1047C00019E04E48B5F8EE10FCF7D8FE064618B1D1
:1047D0004B49012008700EE04848B5F8EE10FCF790
:1047E00017FD044620B1464B01221A70344602E000
:1047F000032000F049FF3F4A92F8ED30052B2DD8F9
:10480000DFE803F007071E2C2C03022003F014FA44
:1048100024E000204FF448718DF80400ADF8061034
:1048200001A83549FCF760FC28B1364A364B012512
:104830000420157018702F4991F8ED50012D0DD0FE
:1048400064B12C4A2D492C48B2F8EE20FCF7C2FD89
:104850002D4D2C4B0220012118702970294A254D1D
:10486000107840B995F8ED3013B185F8ED00C2E746
:10487000022003F0E1F995F8E2400CB120490C70F8
:104880001C4A92F8E30008B11F4B187092F8E440FC
:104890000CB11E490C70022003F0BCF910B1164A8D
:1048A00010688047154B1C68A047082003F0B2F938
:1048B000174CD0B1174EB6F92870642697FBF6F561
:1048C0002846FCF723F906FB1572804610B2FCF768
:1048D0001DF91149FCF76EF901464046FCF762F8F4
:1048E0000E49FCF767F9206001E000212160BDE876
:1048F000FC8100BFF8170020281C00203C1C002071
:1049000090080020240800201608002040080020FD
:10491000640C00202C1700208988883C000020416E
:104920002DE9F84F9C4C2068838A9BB213F001025A
:1049300039D0018821F400631A04110C018001218F
:1049400006F0F2FE954A964B117800201870D9B106
:10495000944803781BB9944A1178FF2914D1012394
:10496000037092480278022A06D18B490B68188896
:1049700082B242F4006119808D4B87481978006833
:10498000012206F0EBFE2FE18948834B01780022DB
:10499000186806F0E3FE844A1178FF2900F02481AC
:1049A000FF207F4BDEE003F00201C9B200293DD0B9
:1049B000BFF35F8F7D4D2E78012E354616D1774996
:1049C0000B789BB177490B7883B1114606F0ACFEAA
:1049D000BFF35F8F20683146038B06F099FE754A5E
:1049E000206816704FF480613246FBE0038BBFF302
:1049F0005F8F6E490A78022A09D1684B1A7832B162
:104A0000684B1A781AB1002106F08EFEE5E00978AD
:104A1000032907D1614B1A7822B162490B78002B28
:104A200040F0DD804FF480610122DBE003F00406FA
:104A3000F6B2002E71D0594BDFF878811A78012632
:104A400088F80060574B002A4DD01A78002A4AD0C7
:104A5000564D2F78524D022F574F29D906F064FE3C
:104A6000206895F80090D7F800A006F074FE4FFA81
:104A700089FB0AF80B0009EB060031462870206814
:104A800006F046FE206888F800603F6895F80080D0
:104A900006F061FE4FFA88F907F80900B044206873
:104AA0004FF48061324685F8008006F049FE2BE025
:104AB000314606F02DFE20682E78D7F8008006F0EB
:104AC0004AFE4FFA86F9731C08F80900D9B220682B
:104AD0004FFA81F83F68297006F03DFE033607F86B
:104AE00008002E7010E01B78012113B9334A1378A7
:104AF0002BB106F00DFE2A480278511C03E006F0A7
:104B0000FBFD284801210170234A11680B8803F43A
:104B1000807082B2002AF9D166E003F040010F46AE
:104B20001F4D09B3244B2F78D3F8008006F013FEF5
:104B30004FFA87F908F80900781CC1B229701B4D9B
:104B40004FB22A780337BA4205D120684FF480610A
:104B5000324606F0F5FD124B28781A7851B2884299
:104B600042D1501C18703FE01B063DD52B785EB239
:104B7000721C27D0124901330A682B70915D06F030
:104B8000E8FD0A4895F90020017891422CD120686F
:104B90004FF480613A4625E0A8080020A6080020CE
:104BA000A4080020A50800209508002096080020F1
:104BB000AD08002094080020980800209C080020E0
:104BC000A0080020154A2970117806F0C2FD14488B
:104BD000017811B9134B1A7832B9134800684FF4B1
:104BE0008061002206F0ACFD0E4A104B117893F95B
:104BF00000004A1C90420ED10D4B0E49187800223D
:104C00000A7028B1084908684FF4407106F098FD11
:104C1000094B00221A70BDE8F88F00BF95080020EC
:104C2000A608002096080020A8080020A40800205C
:104C300094080020A5080020AC080020FFF770BEF3
:104C4000FFF76EBEF0B5484C89B04FF440651C23A9
:104C500007460226204602A9ADF808508DF80A3012
:104C60008DF80B6000F0B2F94048142107608DF810
:104C70000E10204603A9ADF80C508DF80F6000F01F
:104C8000A5F925610825384CA268520503D40A20ED
:104C900000F07EFCF7E74FF480660A20666100F0C2
:104CA00077FC6F1E0A20266100F072FC17F0FF05EA
:104CB000E9D14FF4006767610A2000F069FC666182
:104CC0000A2000F065FC26610A2000F061FC022049
:104CD00027611C218DF80F002046244C4FF44063BF
:104CE0008DF80E1003A9ADF80C3000F06FF92068B4
:104CF00006F064FC04A806F0E5FC20682A464FF4A0
:104D0000407106F01DFD1A484FF480434BF6FF72C8
:104D1000049001212068ADF81C30ADF81620ADF8E4
:104D2000145006F0DDFC04A9206806F061FC4FF485
:104D3000A06005F05FFF2221012201A88DF8041078
:104D40008DF805508DF806508DF8072005F05CFFB2
:104D5000212301A82E468DF804308DF8055005F06A
:104D600053FF09B0F0BD00BF000C0140A8080020AF
:104D7000801A060010B54000244CC0B220702448B0
:104D8000244C017000212170234C01202070234C01
:104D90002360234C2360234B1A70234A107023484E
:104DA000017023490868838803F4007291B2A1B9A5
:104DB000038803F4807291B241B9038803F400724E
:104DC00091B20029F9D1012106F096FC18484FF460
:104DD00040710068012206F0B3FC47F23053124ADA
:104DE000117811B1013BFAD100E053B911490A8899
:104DF000501C83B20B800E490868FFF723FF002088
:104E000010BD0A4B187880F0010010BDAD080020DD
:104E1000950800209C080020A60800209808002083
:104E2000A008002096080020AC0800209D08002063
:104E3000A80800209208002010B54000244CC0B201
:104E400020702448244C017024490120087000215E
:104E50002170234C2360234C2360234B1A70234A78
:104E600010702348017023490868838803F4007296
:104E700091B2A1B9038803F4807291B241B9038859
:104E800003F4007291B20029F9D1012106F034FC3B
:104E900018484FF440710068012206F051FC47F2B7
:104EA0003053124A117811B1013BFAD100E053B9E5
:104EB00011490A88501C83B20B800E490868FFF71D
:104EC000C1FE002010BD0A4B187880F0010010BD13
:104ED000AD08002095080020A60800209C080020AE
:104EE000A00800209808002096080020AC080020A8
:104EF0009D080020A80800209208002007B502ABFA
:104F000003F8012D0122FFF797FF0EBD274B37B5A0
:104F10001868818A8AB20192019B13F4706F02D0E3
:104F2000234A01211170019B13F4E06F31D04FF43B
:104F300080610022038B06F003FC0198810528D4D0
:104F40001A4D2868018801F4007293B20BBB0488E3
:104F500004F480718CB29CB1028802F4807399B21F
:104F60000029F9D1012106F0D3FB1048006802881E
:104F700002F4007399B20029F9D1FFF763FE08E04B
:104F8000012106F0C5FB28684FF44071224606F067
:104F9000D7FB06480268938A23F470610804030C67
:104FA0000449938200220A703EBD00BFA808002079
:104FB0009D080020AC080020FFF7A8BFFFF7A6BFA0
:104FC000014B188880B27047920800202DE9F0410B
:104FD0000F88002347FA03F2D2072DD58A7803F011
:104FE0000705DC08AD0012F0100F18BF91F803C0E0
:104FF00002F00F0618BF46EA0C064FF00F0C0CFA31
:1050000005FC06FA05F550F82480282A28EA0C0C3D
:1050100045EA0C0540F8245006D1012202FA03F2B9
:10502000C46824EA020206E0482A05D1012202FAF5
:1050300003F2C4682243C2600133102BCAD1BDE819
:10504000F08108B503681A68904708BD38B5054671
:105050000C4614F8011B19B12846FFF7F2FFF8E7D8
:1050600038BD08B503685968884708BD08B50368A6
:105070009968884708BD08B50368DA68904708BD95
:1050800008B503681969884708BD08B503685A69F7
:10509000904708BD7047036B13B15A68006C01E07C
:1050A000026AC069101A18BF01207047436B13B120
:1050B00090F844007047826A406A111A4B4253EBE1
:1050C00001007047836A8169426BC918D160416AE7
:1050D000994203D9CB1A5360816204E00169CB1A6B
:1050E000536000228262002180F84410406B01214D
:1050F00006F0E1BB30B50446007985B000230D46CB
:105100000091C107ADF80430ADF80630ADF80830B5
:10511000ADF80C30ADF80A3002D50422ADF80A2003
:10512000820705D5BDF80A1041F00803ADF80A3032
:10513000A06C694606F0A0F8A56005B030BD026B12
:10514000034610B5406942B11A6CD9688C1A013A0D
:1051500018BF1146005D196410BD196ADA68405C19
:105160000131B1FBF2F402FB1411196210BD10B54C
:10517000426A8469A154416A02690131B1FBF2F4C7
:1051800002FB1411426B416232B11368DB070BD48E
:10519000BDE81040FFF796BF806C40F227710122F6
:1051A000BDE8104006F0CCB810BD0000214B13B58F
:1051B000986021480C4658612048214A21491863CB
:1051C00014381A6099614FF48072586301214FF4CA
:1051D0008040DA601A6106F0B9F94FF400710223D9
:1051E0001822ADF80010A1078DF803308DF80220C9
:1051F00003D515486946FFF7E9FE48234FF4806060
:10520000E207ADF800008DF8023003D50E4869467C
:10521000FFF7DCFE01220E2101A88DF804108DF8A5
:1052200005208DF806208DF8072005F0EDFC0148DB
:105230001CBD00BF700B00206E0A00205800024009
:10524000CCEB0008EE080020000801401F4B13B50E
:105250001F4A98600C4680204021D86019611D4883
:105260001D491A601D4A986199644FF4003001216C
:105270005A6106F077F90223042218208DF80330D2
:10528000A307ADF800208DF8020003D51448694645
:10529000FFF79CFE08214823E007ADF800108DF8C9
:1052A000023003D50E486946FFF790FE0120262202
:1052B0008DF8050002218DF8070001A88DF8042063
:1052C0008DF8061005F0A0FC00481CBDBC0B0020AA
:1052D000CCEB0008AE08002000440040EE0900209E
:1052E000000801402DE9F0411E46584B90B098420D
:1052F00005468846174604D110463146FFF756FF4B
:1053000007E053480024854204D110463146FFF798
:105310009DFF0446002106F004022671A760019754
:10532000A5642162E161A1626162C4F82C80ADF8DC
:10533000081002F0FF0732B14FF40053ADF80A3005
:105340004FF4806701E0ADF80A700020ADF80C70F2
:1053500016F00107ADF8100002D1ADF80E7002E0B2
:105360000421ADF80E1006F0020606F0FF082EB17B
:10537000BDF80E2042F00803ADF80E30284601A912
:1053800005F07AFF0121284605F0CEFF05A806F0BA
:1053900085FA0023281D4FF48051802205900E913C
:1053A0000F9309930B930A920C9317B3206BD0B110
:1053B0006269E168079320230D930692089106F035
:1053C000D5F9206B05A906F049FA206B012106F0FA
:1053D00072FA28464021012205F0CCFF206B06F02E
:1053E0007FFA206405E0284640F22551012205F0AD
:1053F000A7FFB8F1000F24D0606BE0B1266910213F
:105400000896002607910D9606F0B0F9606B05A985
:1054100006F024FA0122606B022106F057FA606B55
:10542000314606F05BFA606B802146600122284617
:1054300005F0A0FF05E0284640F22771012205F0A3
:105440007FFF204610B0BDE8F08100BF003801406A
:105450000044004010B50B4C4FF4005006F044FAE5
:105460000021606B06F027FA626AA36A9A4204D0B0
:105470002046BDE81040FFF725BE012084F8440017
:1054800010BD00BF700B00200D4B986C028802F01D
:1054900080018AB29AB19A6A596A8A420AD0996995
:1054A000895C013281801969B2FBF1F001FB1022A5
:1054B0009A62704740F22771002205F041BF7047A1
:1054C000700B00201C4B10B59A6C1488A4B204F029
:1054D000200188B290B1D96A19B1938898B28847EF
:1054E0000CE09288D9695869D2B24254D869DA6816
:1054F000411CB1FBF2F002FB1011D96104F08004F1
:10550000A4B2C4B10C4B9A6A586A82420BD0986913
:10551000996C805C013288801969B2FBF1F001FB63
:1055200010229A6210BD986C40F227710022BDE8EB
:10553000104005F005BF10BDBC0B002070470000F7
:10554000024B1A68501C1860704700BF080C0020FE
:1055500010B5094A094913688C6810688342F8D16C
:10556000074A106811684FF47A725043001BB0FB71
:10557000F1F102FB031010BD080C002010E000E068
:105580000C0C0020014B1868704700BF080C00206D
:1055900038B50446FFF7DCFF0546FFF7D9FF401B8F
:1055A000A042FAD338BD10B504462CB14FF47A703E
:1055B000FFF7EEFF013CF8E710BD000010B586B024
:1055C00005F054F90121254805F0CCFF012144F6EE
:1055D0001D2005F0BBFF0120014605F0ABFF0024B4
:1055E00005F0E4FF4FF6FF7369461D48ADF8003043
:1055F0008DF80240FFF7EAFC69461A48FFF7E6FC1F
:1056000069461948FFF7E2FC1848426842F0007109
:105610004160FFF793FF01A805F03EFF019B14488E
:10562000144AB3FBF0F11448116001684FF47A7327
:10563000B1FBF3F2114B501E114A5860F0210720C4
:1056400082F823109C6018600E48FFF7FBFAFCF705
:105650006FF86420FFF7A7FF06B010BD07004000F9
:1056600000080140000C0140001001400000014012
:1056700040420F000C0C00204C01002010E000E024
:1056800000ED00E00058004010B540F2DB1460432C
:10569000841E2046FFF787FF1920FFF784FFF8E7F5
:1056A00010B1034A034B1A6003480449C8607047AD
:1056B000EFBEADDEF04F00200400FA0500ED00E083
:1056C000024B5A780AB1002058707047E31C002042
:1056D0002DE9F84F384E04463768384606F00EF983
:1056E0000546384606F07EF976688046304606F074
:1056F00005F98346304606F075F9D4F8049006465D
:1057000029464846FBF756FAA7688246414638467E
:10571000FBF750FA01465046FBF742F921688246F2
:105720005846FBF747FA414604464846FBF742FA1B
:105730003146FBF73FFA01462046FBF733F9314685
:1057400004463846FBF736FA2946FBF733FA01469A
:105750002046FBF727F90146504606F0CFF91749D6
:10576000FBF728FAFAF762FE11A3D3E90023FAF750
:10577000DBFF134B044618680D46FAF757FE024646
:105780000B4620462946FAF7F3FC00220D4BFAF7A8
:10579000CBFFFBF7B1F806F0E5F881B20A0444BF8D
:1057A00000F5B47189B208B2BDE8F88FAFF300809C
:1057B000182D4454FB210940200C00200000E14436
:1057C000640C00200000244010B5194C2088FBF721
:1057D0009DF91849FBF7EEF906F0C4F8164B18804E
:1057E0002088FBF793F901461448FBF797FA144910
:1057F000FBF794FA134908601348B0F87000FBF700
:1058000085F901461148FBF789FAFAF70FFE06A35E
:10581000D3E90023FAF75EFEFBF76EF80C4A10603E
:1058200010BD00BFAFF300803B597E90A9E78140D7
:105830000C000020C903683F100C00200AE81C413E
:1058400000401C46681C00202C170020000061440A
:10585000841C0020AFF300802DE9F041044600686D
:105860000D460146FBF7A6F9D4F8048006464146EA
:105870004046FBF79FF901463046FBF793F8A768CF
:10588000064639463846FBF795F901463046FBF7A0
:1058900089F806F035F900210646FBF71FFB70B9C1
:1058A00020683146FBF73AFA314628606068FBF71A
:1058B00035FA31466860A068FBF730FAA860BDE8A9
:1058C000F0812DE9F04F0C68836889B0D0F800A012
:1058D000D0F804800646204603938B4606F00EF867
:1058E0000746204606F07EF8DBF804408146204655
:1058F00006F004F80546204606F074F8DBF80820A8
:1059000004461046019205F0F9FF8346019806F01F
:1059100069F8394602905846FBF74CF9394604902D
:105920000298FBF747F9594605904846FBF742F9BC
:10593000029906904846FBF73DF9294607905846DC
:10594000FBF738F901465046FBF734F92146834608
:105950000698FBF72FF901460598FBF723F8014657
:105960004046FBF727F901465846FBF71BF821464E
:1059700083460498FBF71EF901460798FBF710F8D9
:1059800001460398FBF716F901465846FBF70AF85B
:105990003060029905F10040FBF70CF901465046D2
:1059A000FBF708F9214683460798FBF703F9014600
:1059B0000498FAF7F5FF01464046FBF7FBF801466D
:1059C0005846FAF7EFFF214683460598FBF7F2F8B1
:1059D00001460698FAF7E6FF01460398FBF7EAF856
:1059E00001465846FAF7DEFF214670605046FBF745
:1059F000E1F82946044609F10040FBF7DBF80146CF
:105A00004046FBF7D7F801462046FAF7CBFF394668
:105A100004462846FBF7CEF801460398FBF7CAF880
:105A200001462046FAF7BEFFB06009B0BDE8F08F2E
:105A30001FB50B684A6889680193039101A9029216
:105A4000FFF73FFF05B000BD80EAE073A3EBE07312
:105A50008B4206DB002801DD401A704702D0401857
:105A600070470020704700002DE9F041524B86B08E
:105A70001A685B6802F1004203F1004301934F4B47
:105A80000646B3F900000092FBF740F800F1004031
:105A9000FAF7CCFC46A3D3E90023FAF71BFDFAF78B
:105AA0002BFF474C0290B4F90000FBF72FF803904E
:105AB000B4F90200FBF72AF80490B4F90400FBF7EC
:105AC00025F86946059003A8FFF7FBFE3D4B93F8C8
:105AD0004030012B16D13C48417869B93B4C4025F8
:105AE000226892FBF5F7D01BFBF710F80599FAF73F
:105AF00059FFFBF725FA2060344B4021186890FBD2
:105B0000F1F001E0324B1888FBF700F801460598E8
:105B1000FAF746FF05903046FAF7F4FF2D4907469D
:105B2000FAF740FF01463846FBF7F8F82A4D0746DA
:105B30002C6805982146FAF733FF01463846FBF7F3
:105B400039F801462046FAF72DFF244C28601D4DF8
:105B500007460398D4F8008005F004FF95F830104C
:105B6000FFF772FF08EB000204982260D4F804806B
:105B700005F0F8FE95F83010FFF766FF08EB00031C
:105B800038466360D4F8088005F0ECFE95F82F10D5
:105B9000FFF75AFF1249134B0A684044A060186887
:105BA000B6180E60411C196006B0BDE8F08100BF58
:105BB000399D52A246DF913F200C00204E1C002050
:105BC0007C1C00202C170020E31C0020340C00203B
:105BD0000C0000203661823C580C00205C1C002028
:105BE000380C0020540C00202DE9F04F87B0FEF750
:105BF000C3FD022002F00EF8002800F0A781FEF796
:105C000013FDFFF7A5FCAA4C05462768C71B3846BD
:105C1000FAF778FFA749C968FAF7CCFF8346A64888
:105C2000256090F82E8000252C462E46A34A105F52
:105C3000FAF76CFF5946FAF7BDFF03AB5851B8F1BC
:105C4000000F27D04046FAF761FF01464FF07E5023
:105C5000FBF764F8DFF8A492824651464FF07E507D
:105C6000FAF79EFE55F80910FAF7A4FF9449034687
:105C7000085F0193FAF74AFF5146FAF79BFF014686
:105C80000198FAF78FFE49F80500FBF759F98D4A9C
:105C9000105303E08A498B4A605AA052894B04355D
:105CA000E15E0234062C01FB0166BFD1864A642006
:105CB000138846435B43854803A996FBF3F6FFF739
:105CC000B7FE082001F0A6FF20B1814803A9FFF725
:105CD000AFFE07E07F4803A9FFF7AAFE7D48014613
:105CE000FFF7BAFD493EB1B23B2904D9082001F0C3
:105CF00091FF48BB50E0784CB4F8F000FAF702FF8F
:105D00004FF07E518046FAF74DFE01464FF07E502F
:105D1000FBF704F8002406466C4D404655F8141075
:105D2000FAF748FF81466748005FFAF7EFFE014641
:105D30004846FAF737FE3146FAF73CFF45F81400BB
:105D40000234062CE8D1D1E7634A0024B2F8F2000D
:105D5000FAF7D8FE4FF07E518046FAF723FE01464F
:105D60004FF07E50FAF7DAFF0646594D404655F897
:105D70001410FAF71FFF594B8146185FFAF7C6FE59
:105D800001464846FAF70EFE3146FAF713FF45F88A
:105D900014000234062CE8D151494C4DB1F90000F1
:105DA000FAF7B4FEAC68014620460126FBF7BEF8C0
:105DB00000B906464B4821464673686805F09EFECA
:105DC000494C2A682060686802F100460146FAF7EB
:105DD000F1FED5F80880054641464046FAF7EAFE4E
:105DE00001462846FAF7DEFD05F08AFE01463046F8
:105DF00005F084FE60602068FAF718FB2AA3D3E957
:105E00000023FAF767FBFAF777FD05F0ABFD374D96
:105E100028806068FAF70AFB23A3D3E90023FAF786
:105E200059FBFAF769FD05F09DFD6880082001F037
:105E3000F1FE2F4C08B1264800E02648FFF748FC49
:105E40001D4D20803846FFF70FFE95F87230002B6D
:105E500000F080801D4908688C684F680146FAF799
:105E6000A9FE394606463846FAF7A4FE01463046F2
:105E7000FAF798FD214606462046FAF79BFE0146B2
:105E80003046FAF78FFD05F03BFE01462046FAF753
:105E900045FF18490446FBF735F888B3164A002039
:105EA000108057E0AFF300803B597E90A9E7814016
:105EB000280C00203C1C00202C170020541C002023
:105EC0006C1C00207C1C00200C000020881C002082
:105ED000140C002010000020F8170020341C0020B3
:105EE000100C0020E31C0020200C00203C0C0020A3
:105EF0004E1C00208FC2753C5C0C0020440C00201E
:105F0000204605F0ABFD264B1968FAF753FE05F065
:105F100029FDB0F5617FA8BF4FF46170FAF774FAFC
:105F20001DA3D3E90023FAF7FFFBFAF7E5FC05F020
:105F300059FD044695F87200FAF7E8FD2146FAF794
:105F400039FE05F00FFD174B188003E0164B188043
:105F500058809880154B5979154B012907D0154861
:105F60001A8859889B8802804180838011E01249F9
:105F7000B3F90420B1F9000002EB4000032290FBCA
:105F8000F2F080B20B4A088019885B8890801180FB
:105F9000538007B0BDE8F08FA2EB0FE5DD16964009
:105FA000841C00205C0C00206C1C0020F8170020D2
:105FB000541C00205E0C0020500C0020AFF3008029
:105FC00010B5054C00202188FBF76EFE618801208A
:105FD000BDE81040FBF768BE1C0000200A4A02EB37
:105FE000C00393F87B10FF2904D019B1074830F89B
:105FF000110007E00728DABF02EBC000B0F8780014
:1060000040F2DC5000B270472C170020241D002005
:1060100010B500244FF48040FCF7D2FD064B10B1C0
:10602000B3F8DA0001E0B3F8D400044AA052023415
:10603000182CEFD110BD00BFF8170020AC1C0020B9
:10604000F8B53B4D3B4E6B793B4C06EBC3004178BA
:1060500020202160FCF7B4FD324608B101262660FD
:106060006B79162B1CD10024314E0021A619306902
:10607000FAF734FF28B14FF48040FCF7A1FD50BB84
:1060800023E02E4B06F110001D190FC885E80F0004
:106090002B4910340A78531CC02C0B70E4D1EAE76A
:1060A000274F12F8336002EBC3003E704768002FA1
:1060B000E1D00024B442DEDA204D21016D187A18B7
:1060C0000FCA013485E80F00F4E719481D4B4179E8
:1060D000082923D124E01A4E3678012EF5D91A4C1E
:1060E00000251034B542F0DA54F8100C4FF07C5112
:1060F000FAF760FD4FF07C5144F8100C54F8140C82
:10610000FAF758FD4FF07C5144F8140C54F80C0C7D
:10611000FAF750FD013544F80C0CE2E70E2901D1E5
:10612000012200E000221A74BDE8F840FFF770BFBA
:10613000F817002054ED0008700C0020740C0020AB
:106140006C0C0020E31C00207C0C0020F0B5002328
:10615000461C0E4A002198181033C02B0161F8D15B
:106160000B4F07EBC6035F6807B9F0BD0024084A70
:1061700012F83600844208DA064D21014D197B18C9
:106180000FCB013485E80F00F1E7F0BDF8170020D0
:1061900054ED000808180020284B10B51868002896
:1061A0004AD027494A79531E142B3DD8DFE803F023
:1061B0000B3C3C24403C3C1C3C3C3C3C3C2C3C3C94
:1061C0003C3C3C242C001F4890F8BB1031B11E4BC6
:1061D00000205989BDE81040FBF766BD1B4A507886
:1061E0000028F4D10146F5E7174C0020E188FBF7C1
:1061F0005BFD01202189EDE7134C00202189FBF78D
:1062000053FD01206189E5E70F4C0020E188FBF791
:106210004BFD01202189FBF747FD02206189FBF737
:1062200043FD0320A189D5E72020FCF7C9FC18B164
:10623000BDE81040FFF7C4BE10BD00BF700C0020C9
:10624000F81700202C1700201C000020E31C002061
:1062500010B50024064B1878A04208D905492046FD
:1062600031F814100134FBF711FDE4B2F2E710BD70
:106270006C0C0020941C0020064B1A780023D9B225
:10628000914204D2044921F813000133F7E7FFF7E4
:10629000DFBF00BF6C0C0020941C00202DE9F84FDC
:1062A000B24B187803280FD9B149B24CB1F9042088
:1062B0006FF06305002AB8BF5242A91AB4F904006E
:1062C0006432FCF729FEA080A84A1678012E1DD85A
:1062D000A94EAA4C75796A1E142A00F2F981DFE8EA
:1062E00012F0C200F701F7018400D500F701F701B1
:1062F0007101F701F701F701F701F701F100F7016B
:10630000F701F701F701F7015E00C7019B48994BC0
:1063100090F9BA90964FB3F90440C9F10001B7F86B
:1063200006A004FB01F95F88B3F80080944C0025B7
:106330001034B542CCD20FFA8AF0FAF7E7FB54F8E2
:10634000101CFAF737FC834638B2FAF7DFFB54F833
:10635000081CFAF72FFC01465846FAF723FB834640
:106360000FFA88F0FAF7D2FB54F80C1CFAF722FC6B
:1063700001465846FAF716FB83464846FAF7C6FB2D
:1063800054F8041CFAF716FC01465846FAF70AFBC3
:10639000FAF7D6FD7B4B23F815000135C8E794F8D2
:1063A0009A20744D12F0010F6B880CBF01264FF03C
:1063B000FF365E43744CB7B204202781FFF70EFE10
:1063C00029886E4D381895F8A230208113F0010FFE
:1063D0000CBF01224FF0FF324A43052096B266817E
:1063E000FFF7FCFD3718678172E194F89A50614815
:1063F00005F002084FFA88F6002E0CBF01214FF07D
:10640000FF3115F0010F45880CBF01224FF0FF321C
:106410006A438688042001FB06F497B2FFF7DEFD8D
:106420001FFA84F808EB00035448F91890F8A2709A
:10643000554C07F0020253B22181002B0CBF012101
:106440004FF0FF314E4317F0010F0CBF01204FF00A
:10645000FF3045430520FFF7C1FDB6B2ADB2371896
:10646000EA19628134E1434994F8A2408E8814F01D
:10647000010F0CBF01234FF0FF3305205E43FFF7F0
:10648000ADFDB5B2404F2818788121E10020FFF71B
:10649000A5FD3E4F94F97A30B7F902603A4D734347
:1064A000322693FBF6F1401828800120FFF796FD75
:1064B000B7F9002094F98240544394FBF6F3C718CF
:1064C0006F8005E1324C607820B9B6F8D4202E4BAD
:1064D000DA810AE02649B6F8D220B1F90600B6F80A
:1064E000D010FCF719FD284DE881274E254CF7897F
:1064F0002780214F97F8190130B3204D0220FFF774
:106500006DFDB5F98410B5F98620FCF705FD214B2A
:10651000B7F812111A880C1A16B220B2864203DAA2
:1065200097F81961B41803E003DD97F81971D41BCB
:106530001C8095F98A50B3F9003064226B43124FE6
:1065400093FBF2F00918B980114C0F4DA67A56B1A1
:10655000074B1A880324EA802A8198886881598821
:10656000A981094D18E0034BF3E700BF6C0C002034
:10657000C41B0020CC1B0020F81700202C17002083
:10658000740C0020941C00201C0000203C0C0020F7
:10659000E31C00206E0C0020AA4FB5F9062007EB83
:1065A000C40696F97A3064205A4392FBF0F7EF80E4
:1065B0002046FFF713FD01343918E9800235072C16
:1065C000EAD185E0A04B5A7822B9B6F8D4709F4939
:1065D000CF810AE09E48B6F8D010B6F8D220B0F9C4
:1065E0000600FCF799FC994EF081964E974B964A1F
:1065F00096F89270974DDC89907A17F0010F2C80F5
:106600000CBF01254FF0FF3508B1914900E09249D8
:10661000488807F00204454396F89A60098862B2F8
:10662000002A0CBF01274FF0FF3716F0010F0CBFF7
:1066300001244FF0FF3407FB0155604306F00202CE
:1066400057B2DD80002F0CBF01254FF0FF3505FB51
:10665000010018810320FFF7C1FC7C4EF388C118AC
:106660000420F180FFF7BAFC3489021932812FE04F
:10667000794F0324BF88734B03EBC40090F87A6012
:10668000C4F1060306F002014DB2002D0CBF012239
:106690004FF0FF327A437049580831F8105016F025
:1066A000010F0CBF01264FF0FF3606FB0522674D98
:1066B00096B225F814602046FFF790FC331825F8B1
:1066C00014300134072CD6D1614F6249F888088014
:1066D0002020FCF775FA002841D00020FFF77EFC4F
:1066E0005A4C054620800120FFF778FC5B4A608009
:1066F000137AA3B3534F5A4A97F8BC1001F002061D
:10670000F3B2CBB1B2F9003097F9821097F97A70F1
:10671000B2F9022059437B425343322691FBF6F1F2
:106720006FF0310789B293FBF7F28F187D1993FB55
:10673000F6F625808E1910E097F97A10B2F902600A
:1067400097F982704E43B2F900203221574396FBED
:10675000F1F3ED18258097FBF1F680196080414C2C
:10676000384D04F11006B4F90200B5F97410B5F90A
:106770007620FCF7D1FB24F8020F0835B442F2D1A1
:10678000304991F8BC3003F00402D7B22FB9314838
:10679000354B07881C7801221CE0344D68790E289F
:1067A0000AD0082808D0324C04EBC0014B78002BEB
:1067B00014BF0225002500E0042500242D4F621996
:1067C00007EB4401D0B209890134FBF76DFA042CC0
:1067D000F4D1DCE7A24209D21E483FB230F91210D0
:1067E0000132B942A8BF0F46BFB2F3E70024A0466A
:1067F0001D4A1178884567D21C4D3BB2B5F8D200CE
:10680000834204DD134DC21B615B501860534FF48B
:106810008040FCF7D5F90F4D70B3164B40F2DC51B8
:10682000B3F90620114B8A42285FC7BFB3F8D810CE
:10683000B3F8D220B3F8D410B3F8D620FCF76CFB31
:10684000285336E02C170020E31C00201C000020F9
:10685000C41B0020941C0020CC1B0020F41C002032
:106860003C0C00201A0000206C0C0020F8170020BF
:1068700054ED0008241D0020144E285FB6F8D010F7
:10688000B6F8D220FCF748FB114BB6F81411B3F957
:10689000062005EB04098A4228530ADA1020FCF787
:1068A0008FF910B9B6F8D00001E0B6F8D400A9F815
:1068B0000000084A507818B90749084B625AE2525A
:1068C00008F10108023493E7BDE8F88FF8170020BB
:1068D000241D0020E31C0020AC1C0020941C002080
:1068E000024B1868003018BF01207047700C002060
:1068F00044F25063984203DDA0F50C40A038704785
:1069000003498842BCBF00F50C40A030704700BF6F
:10691000B0B9FFFF10B5FAF7F9F800210446FAF70D
:1069200005FB08B1204601E004F100400549FAF7F3
:10693000F5F90549FAF73EF904F0E0FF034B18605A
:1069400010BD00BF8096184B35FA8E3C2C000020FD
:1069500010B5044C002320702361FEF713FE606124
:1069600010BD00BFC81C0020F8B51D4614460E46D9
:10697000FAF7CCF86968FAF71DF93146FAF71AF90F
:106980002168FAF70FF82060FAF7DAFAED6807469F
:1069900005F10040FAF7D4FA06462846FAF7D0FA8D
:1069A000314602463846FCF7B7FAFAF7AFF82060EE
:1069B000FAF7C6FAF8BD0000F8B5101A0C461F46E3
:1069C000FAF7A4F80546381BFAF7A0F8174B079E0C
:1069D0001968FAF7EFF8294604462846FAF7EAF864
:1069E000214607462046FAF7E5F801463846F9F70A
:1069F000D9FF05F085F80E49FAF7DCF8FAF7C6FA80
:106A000006990860214605F1004005F077F809492C
:106A1000FAF7D0F80849F9F7C5FFFAF791FA002814
:106A2000BCBF00F50C40A0303060F8BD2C00002049
:106A30002C7D8E3FA00CB34500A00C4610B504463B
:106A4000002003460D49CA5CA2B12E2A04D10133AD
:106A500094B1C91800220A55084A0A21D25C484359
:106A6000A2F13001092901D8303880180E2B02D844
:106A70000133E7E710BD002010BD00BF310F00203B
:106A8000F8B52D4B93F81C0110B1012850D10AE044
:106A90002A4B2B4A58782B4B02EB00114968586857
:106AA000FEF7E9FA41E0274D6868FEF7E9FA0028A9
:106AB0003ED0224C2178264601291ED1FEF762FDE8
:106AC00006466069321A632A35D92169042912D829
:106AD0001B4F686807EB01135968FEF7CCFA607822
:106AE00007EB0017B9686868FEF7B0FA22696661BB
:106AF000511C21611CE0022018E022693AB9647837
:106B00000F4B686803EB04114968FEF7B4FA336968
:106B10000A4C8B2B09D80C4A0A48D15C4068FEF716
:106B200090FA21694B1C236102E00320FFF710FF5C
:106B3000024A00205060F8BDF8170020C81C002051
:106B400074F20008681D00200CF1000810B50B4C11
:106B5000E37A8BB10A48017804290DD9094A0A4B16
:106B60001068516818605960FFF7D4FE0748084B59
:106B7000028801211A80217310BD00BFE31C002090
:106B80000E1C0020F01B0020D41B00204E1C0020F7
:106B9000AC0E0020002370B51C460F48002119528E
:106BA000142060430D4A0E4E0E4D99520022325071
:106BB000595335180C4E6960AA60325035180B4E87
:106BC00001346960AA6002333518022C32506960C2
:106BD000AA60E2D170BD00BFA81B0020F40700200E
:106BE000A80D0020AC1B0020600D0020EC0E002042
:106BF00070B5204C204D6079F9F784FF1F49FAF7F2
:106C00008DF82860E07BF9F77DFF1C49FAF786F8DC
:106C10001B4E6860EE60A079F9F774FF1949FAF726
:106C20007DF8194D2860207CF9F76CFF1349FAF7BD
:106C300075F86860A07EF9F765FF1449FAF76EF8F9
:106C4000EE60A860E079F9F75DFF0E49FAF766F8A3
:106C50000F4D2860607CF9F755FF0849FAF75EF898
:106C60006860E07EF9F74EFF0849FAF757F8EE60E2
:106C7000A86070BD2C170020980E00200000C842AC
:106C80000000FA4400002041CC0E002000007A44AD
:106C9000980D002070B5124C05460020FFF758FEF5
:106CA0006570FEF76FFC0F4BA06093F81C01002687
:106CB0006660B0420CBF01240324FFF799FF0A4924
:106CC000234601EB05156A6831460848FEF70AFBC2
:106CD000074A50600120BDE87040FFF739BE00BF91
:106CE000C81C0020F817002074F20008004400407F
:106CF000681D002038B5114B187803281BD1104CA3
:106D00006068FEF7AEF938B160682568FEF7AEF945
:106D100001462846FEF795F92068094DFEF7A1F9CE
:106D20000028ECD095E81100FEF7A0F901462046B6
:106D3000FEF787F9E3E74FF0FF3038BDC81C0020AD
:106D4000681D0020F7B50368164C174D23600968CD
:106D5000164E61600068FFF7DDFD94E80C001448F2
:106D60000196009095E80300FFF726FE6B68114A34
:106D700061683668C81A1660F9F7C8FE0E4A0F4FE8
:106D80001168F9F717FFFAF7DBF8296878602068CF
:106D90000B4A431A0B483B60B0F8C4100A4B16600C
:106DA0001980FEBDB40E0020F01B0020140F00203F
:106DB000200F0020B00E00202C000020600F0020CB
:106DC000280F00202C170020560F0020264BF0B56E
:106DD0001D68024600F1100116781446AB195B7865
:106DE000013203F00403DBB263B18A42F4D1002024
:106DF000F0BD13B10A225343DBB210F8011B303946
:106E00005B18DBB2211A0229F3DC0021844209D984
:106E100011B10A225143C9B210F8012B303A891836
:106E2000C9B2F3E72E2E11D10134042000220A2624
:106E300072432678AF197F7807F00407FFB217B1C5
:106E4000303A921901340138F1D100E00022074CA8
:106E50006420614300FB021106240548B1FBF4F2F3
:106E600000FB0320F0BD00BF6801002040420F007E
:106E700080969800000000002DE9F04F9A4B91B0E9
:106E80005868C0B9994C21784A1E032A00F202863C
:106E9000DFE812F0C605C605DF05C9056068FEF724
:106EA000E5F89349044691F81C31012B00F0DF808E
:106EB00008D3022B06D08C4C6068FEF7D2F800286D
:106EC000ECD1DFE7242C07D18A4B8B4A8B4C002175
:106ED000197011702170C5E02C2C02D02A2C40F0C2
:106EE0008280854D834A2978854B15780020585437
:106EF000844AB5B918781570472868D1597850294F
:106F000065D19878472840F0B385D978472940F073
:106F1000AF851B79412B40F0AB850120107000F04C
:106F2000A7BD117801293AD1022D05D11846FFF7E6
:106F30004DFF754908604AE0032D07D119785329A0
:106F400045D1714802685342036040E0042D05D1E9
:106F50001846FFF73BFF6C4B586038E0052D07D112
:106F60001B78572B33D168494A68504248602EE05D
:106F7000062D07D119786548302994BF00210121D9
:106F8000C17224E0072D04D1FFF758FD604A10704C
:106F90001DE0092D1BD1FFF751FD5E4B16E00229C4
:106FA00015D1072D0CD10120FFF748FD41F2184201
:106FB00050434FF47A71584BB0FBF1F0188006E063
:106FC000082D04D10120FFF739FD544B1880494B9F
:106FD0004949013500202A2C1D70087039D15048CC
:106FE000012404703EE00D2C4D4A01D00A2C26D11C
:106FF0001478FCB1424C21786478A1F13000C3B21E
:10700000092B84BFA1F13703DBB2A4F1300003F0F8
:107010000F02C3B21101092B84BFA4F13703DBB205
:10702000364C03F00F0289182078CBB2C21A5142B5
:1070300051EB02043A4B002018707CB912E02E4943
:107040000B780E2B03D82E48C45401330B701278E2
:1070500042B92A4B1A7854401C7003E0294A107830
:10706000012800D00020C00700F1338123E72D4B19
:107070000022197808293FF61EAFDFE801F00A0563
:107080001119275F7C96A000622801D1022105E03A
:107090001A70B52C7FF40FAF1C78611C19700AE7C9
:1070A0002149224A03261E7008701070204B0BE005
:1070B0001E4E0421197032781D4BA1181878CAB2DF
:1070C000101818701B4B32701C70F4E605211970F3
:1070D000164B174E1A783078A118CAB210183070B3
:1070E000154E1A703480E6E6681D0020C81C00208A
:1070F000F8170020540F0020240F0020C40E002099
:10710000310F0020E80E0020F01B0020E31C0020BF
:107110000E1C0020A61B0020B01B0020140800201D
:10712000AA0E0020AB0E0020E90E0020A80E0020C1
:10713000A90E00205C0D0020960D00206C4906264B
:107140001E700A786B4BA6181878F2B210181870D7
:10715000694B0A70198801EB0424A6B2B6F5007FCA
:1071600001D81E8003E000221A80644B1A700024AC
:10717000634B00F052BC5E495E4E0A783078A3182B
:10718000DAB2101830705E4E0A7033885A4AC72B34
:1071900098BF5C49108898BFCC545C1CA1B288424F
:1071A00031807FF488AE072107E0514A08261E701F
:1071B000137883423FF47FAE0021504B6EE74D4E73
:1071C0001A70337883427FF476AE4F4C20780628CD
:1071D0003BD005D8022813D003287FF46CAE23E0FF
:1071E000122847D030287FF466AE464A474C1679BD
:1071F000444A102E88BF102626702178002347E0CD
:10720000404C434E6368A06821697360414B4FF462
:107210007A723060404C91FBF2F618783F49268034
:10722000C87201223E4923E036494A7912F0010032
:1072300004D00E79F41E634253EB04003549087004
:10724000002839D1354AD07236E02E4EF47A14F047
:10725000010104D0B07AC21E534253EB02012D4EFD
:10726000317009B92D4CE17226482E4990F82F2033
:107270000A7021E023482C498669426942F2107461
:107280002A4B96FBF4F00A80188001222849EFE788
:107290000C328B4210DA12F8046C264812F8034CB8
:1072A0001E54254E25489C5512F8014C16781C5446
:1072B000234C1E550133EBE719490A78002A3FF4A5
:1072C000FAAD1B4B1E78002E3FF4F5AD00240C7078
:1072D0001C701C4CA068E060FEF754F9A0602020F0
:1072E00000F0A2FC18490A78012A2FD100232EE0D1
:1072F000A80E0020A90E0020960D0020AB0E002045
:107300006A0F0020D00D00205C0D00200F1C002013
:10731000F01B0020480F0020A61B0020E31C0020CB
:107320005C0F00200E1C0020B01B00201408002061
:10733000300F0020941B0020DE1B0020F81B0020D3
:10734000181C0020C81C00208407002001237E4C4C
:107350000B70E07A00283FF4AEAD7C490A78042A2D
:107360007FF6A9AD677807B92773257B15B90FB1EB
:10737000FFF7ECFB764E05213378764F5C1C94FBCF
:10738000F1F001FB10423270734E97F800C0734D5C
:1073900006EB82020023724C72491F59DFF810E29B
:1073A0007148724E5F5097FBFEF1195006FB017059
:1073B000DFF8009203EB040A42F2107490FBF4F73A
:1073C0001668BCB253F809701060C6EB0708404459
:1073D000052643F8090090FBF6F00EFB0101644816
:1073E000BCF1010F25F8024F195005D1023CB4F54C
:1073F000797F98BFCAF8001004331432082BCAD121
:10740000FEF7C0F85B4D5C4C2A68801AF9F77AFBEE
:107410005A49F9F783FC2060FEF7B4F82860256824
:107420004FF07E512846F9F763FD08B94FF07E55BD
:1074300025600CA90DAC4A48514B0194009103C83A
:107440000CCBFFF7B9FA0C9A64234E49B2FBF3F068
:1074500008800D9A3C4892FBF3F34B4C027B23804F
:107460000AB90A80228049490C78002C36D0424F54
:107470004FF07E503968F9F751FC454D384E2B6876
:1074800004463068C01AF9F741FB2146F9F792FB30
:10749000F9F756FD726869683E4D0746501AF9F7CC
:1074A00035FB2968F9F786FB2146F9F783FBF9F7E5
:1074B00047FD04B238480225B0F902303FB2E21865
:1074C00092FBF5F1B0F900208BB2B918334C91FB67
:1074D000F5F291B263802180438001802B4B012023
:1074E0001F4C1870184B6168294A20681C7A51603B
:1074F00010601CB9DA79002A3FF4DDAC284E294D22
:10750000294C01960095164F94E80C00FFF754FAA9
:1075100061687868254E081AF9F7F8FA1D4B196862
:10752000F9F748FBF9F70CFD70600A48226890F9FA
:1075300000303C68012BC4EB020131603CD0022BCF
:107540007FF4B9ACF2E000BFE31C00200E1C002069
:10755000680F00209D070020340D0020C40E00207D
:10756000F01B0020400F0020E00E0020806967FF24
:107570004C0F0020900D0020DC0E002000007A440B
:10758000D41B0020D21B0020DC1B0020880D002013
:10759000BC0E00202C0000202C0F0020580F0020D3
:1075A000140F0020200F0020B40E0020600F0020D8
:1075B00080969800180F0020002634463546DFF8E4
:1075C00074B28B4F5BF82580DFF864924046F9F780
:1075D0009DFA3968F9F7EEFAF9F7B2FC34F80910B8
:1075E000844B421A90B2E05207B2CDF80890DFF80F
:1075F000489238460397F9F789FAD9F80010F9F755
:10760000D9FAF9F79DFC81B27B48142202FB0507E9
:10761000DFF800A2039B089103EB0800DAF80010E2
:107620004B463A46FFF7A0F90899DFF810820A188E
:107630005BF82500DAF800B024F8082008905846D6
:10764000F8F7F4FED7F808A0CDE904015046F8F7A2
:10765000EDFE6A4BCDE9060193F8C000F9F752FA46
:10766000F8F7E4FE60A3D3E90023F8F733FF0246FE
:107670000B4600206249F9F757F8DDE90423F8F7D3
:1076800077FD0B460246DDE90401F9F74DF8089A4B
:10769000CDE9040179680135501AF9F737FA5946EE
:1076A000F9F73CFB5146F9F77BF9F8F7BFFE0246C4
:1076B0000B46DDE90401F8F70DFF0B460246DDE954
:1076C0000601F8F755FDF9F717F90899386179605F
:1076D000B860D9F80810F9F76DFAF9F731FC4949A3
:1076E0004FF4FA62FBF718FCDDF808C034F8081014
:1076F00034F80C20313293B2622B98BF002040182E
:1077000082B224F8082010B23F4940F6B832FBF7A5
:1077100003FC394B28F8040099593C480234315095
:107720001436022D7FF44BAFFFF7C5BB2F68334DE6
:10773000374CB5F9C6807E08B04528BFB0462588CD
:107740001FFA88F80FFA88F229B28A420BDD314815
:1077500031490068F9F72EFAF9F7F2FB43191FFADD
:1077600083F8A4F800802D4E2D4D34682A68A61A9F
:107770003046FFF7BDF80028D8BF404241F29311D0
:107780008842CCBF00200120002859D03046F9F7AC
:10779000BDF92449F9F70EFA04F024F905463846F4
:1077A000F9F7B0F901462846F9F704FAF9F7C8FBEA
:1077B0001D4B1549188040F6B83200B2FBF7ACFB00
:1077C000201848F6A044A04203DDA0F50C40A038E4
:1077D00004E00028BCBF00F50C40A030134A106044
:1077E00030E000BFAFF30080182D4454FB21194056
:1077F000980E00208A0D0020600D00202C1700201C
:107800000000F03F30F8FFFF48F4FFFFEC0E0020CF
:10781000560F0020DC0E00200000C842140F00208C
:10782000280F0020D3023739940D0020B00E00201D
:10783000580F0020600F0020CC0E0020AC1B002051
:10784000994F3C60984E002531682C46C1F50C508C
:107850002830F9F75BF99549F9F7ACF9074604F0D8
:107860004DF80F90384604F0BDF82F460E900FFAF1
:1078700088F0F9F74BF90EAB53F82710F9F79AF99E
:1078800006468B48DFF86CA2005FF9F73FF9014626
:107890003046F9F785F8F9F753FB864924F80A00D2
:1078A0004FF47A7200B2FBF737FB82B211B2DFF805
:1078B000489224F80A2008460391F9F727F9D9F8E5
:1078C0000010F9F777F9F9F73BFB83B27A481426F1
:1078D00006FB0706DFF824B2039ADBF800100693D4
:1078E00010464B463246FFF73FF8DBF800C034F94C
:1078F0000A1009906046D6F808A00891CDF808C093
:10790000F8F794FDCDE904015046F8F78FFDDFF854
:10791000F0B1CDE90A019BF8C000F9F7F3F8F8F7E8
:1079200085FD5FA3D3E90023F8F7D4FD02460B469B
:1079300000206249F8F7F8FEDDE90423F8F718FCA7
:1079400002460B46DDE90401F8F7EEFE089BCDE99F
:10795000040170680137181AF9F7D8F8DDF808C083
:107960006146F9F7DBF95146F9F71AF8F8F75EFDC9
:1079700002460B46DDE90401F8F7ACFD02460B4672
:10798000DDE90A01F8F7F4FBF8F7B6FF089A099B5E
:1079900072603061B060069ED9F80810F618F9F7E9
:1079A00009F9F9F7CDFA3018454E81B2A15308B262
:1079B00040F6B8324349FBF7AFFA3F4A3053424BE7
:1079C000A8580234E8501435022F58467FF44FAFC0
:1079D00090F8C21031B1344A642413683B4A93FBD7
:1079E000F4F111803A4BB0F8BE001C6884420ED905
:1079F000384939480A68036842F21074D01AFEF711
:107A000077FF0028B8BF4042A0427FF754AA33480E
:107A1000334A012104882D4B11701C80FFF74BBAAB
:107A2000FFF72EF836E062686078531C411CCAB23A
:107A300063600523B2FBF3F003FB10216170FDF7D7
:107A4000A1FD284AA06028480023C37213700120BA
:107A50000BE0FDF797FDA36840F6C411C01A8842F9
:107A600018D9202000F0E8F80420FEF771FF11E09B
:107A70001E498A78522A7FF4AAAACB784D2B7FF42C
:107A8000A6AA087943287FF4A2AA194A02211170F4
:107A9000FFF79DBA11B0BDE8F08F00BFAFF30080D3
:107AA000182D4454FB211940B00E0020D302373961
:107AB000580F002018FCFFFFEC0E00200000F03FE4
:107AC000AC1B002048F4FFFF600D00204C1C002080
:107AD000200F0020140F0020280F0020AC0E0020E3
:107AE0009D0700200E1C0020E31C0020310F002009
:107AF000E80E00208A0D0020980D0020DC0E0020EA
:107B00002C170020AFF300803B4B2DE9F047B3F971
:107B10000000F8F7FBFF3949F9F74CF8044603F089
:107B200061FF0646204603F0E9FEDFF8E4900546D3
:107B300099F8C180324FB8F1000F29D0314CB7F914
:107B40000200B4F802A00FFA8AF1401AFEF7D0FE44
:107B5000C8F100014246FBF7DFF9B4F80080B7F93D
:107B600000700FFA88F300EB0A02F81A6280FEF741
:107B7000BFFE99F8C1205142FBF7CEF9404487B2CD
:107B80002780B4F90200F8F7C1FF804638B206E05A
:107B9000B7F90200F8F7BAFF8046B7F90000F8F726
:107BA000B5FF294607464046F9F704F831468146B5
:107BB0003846F8F7FFFF01464846F8F7F1FE12494C
:107BC000F9F7ACF8F9F7BCF9104C31462080404683
:107BD000F8F7F0FF294606463846F8F7EBFF01466E
:107BE0003046F8F7DFFE0849F9F798F8F9F7A8F9F1
:107BF0006080BDE8F08700BF4E1C002035FA8E3C47
:107C0000AC1B0020A81B002000002041F40700202E
:107C10002C170020034B196808420CBF00200120DC
:107C2000704700BF6C0F0020024B1A6810431860A9
:107C3000704700BF6C0F0020024B1A6822EA000058
:107C4000186070476C0F0020014B1868704700BF28
:107C50006C0F0020037A0A46032B0FD8DFE803F0ED
:107C60000202060A0649074B00F0ECBA0449054B2C
:107C700000F040B90249034B00F00ABA704700BF58
:107C80000A1D0020B40F002038B504460D4600231D
:107C900061890B4A99520233242BF9D10820FAF753
:107CA0008FFF28B120462946BDE83840FFF7D2BFF4
:107CB0000448054A2946BDE8384000F0D9B800BF5D
:107CC000241D00200A1D0020B40F00202DE9F843D8
:107CD000074608208846FAF773FF70B10024224A4D
:107CE000414613683846E2B29847204921F814000B
:107CF0000134082CF3D1BDE8F8831D4A1D4D1378DB
:107D0000591CCCB204F00306147005EB4609044676
:107D1000064615484146036832463846984729F8D2
:107D200024002A886988AB885018EA88C118881806
:107D300003B2991C042291FBF2F00C4A0E4BA15E97
:107D4000E052CB1E984201DA811CA152135FD91C6C
:107D5000884201DD023810530136F6B2023408358C
:107D6000082ED6D1BDE8F883B40F0020241D0020D2
:107D7000700F0020720F0020B80F002010B544785B
:107D80000078002303FB03F11939614301F6C411A4
:107D90005943414340F6C41291FBF2F1034A22F8E1
:107DA00013100133072BEDD110BD00BF481D00207B
:107DB0002DE9F04F85784FF00A0C0CFB05FCC778D5
:107DC000C5F164086E425FFA88F8C7F16409B6B27B
:107DD000002330B2002804DCB8BF2C4602DB0124AB
:107DE00000E0444600FB00FB64430BFB07FB9BFBEE
:107DF000F4F44C4444434FF00A0B94FBFBF00CEBBF
:107E0000000420B2C1EB020A00FB0AF44FF47A70BE
:107E100094FBF0F404480C191C5202335E44182BF6
:107E2000B6B2D6D1BDE8F08F0C1D0020F8B50546DE
:107E30000F46441E14F8011F49B1054E304605F0A7
:107E4000B9FE0028F6D0861B631BBB55F2E7F8BDD0
:107E5000C4F2000810B50446805CF9F733FFA0F2C5
:107E6000EE2291B240F2DC53994288BF608910BD86
:107E7000024B082113600170704700BF557E000857
:107E8000825C044B53F82200410801F5777290B2EE
:107E9000704700BFCC0F002038B50446FDF758FBF3
:107EA000104B40F6C4111A68821A8A421A460E4BC9
:107EB00001D9002119701B7810600BB90F2C10D15B
:107EC0000A4800210170084A4BB1094D182B1D4486
:107ED00005F8014C03D101230370117038BD013343
:107EE000137038BDEC0F0020F00F0020C80F0020E9
:107EF000F10F002038B540891C460E4B0D461A6024
:107F0000A0F577710C4A4B00136053609360D36007
:107F1000136153619361D36108490948094A0523F4
:107F2000FDF7E0F90849C8600CB108482060082353
:107F30002B7038BD90110020CC0F0020997E0008D6
:107F400000440040A0860100681D0020817E0008DA
:107F500070B5294D287800284CD0284CA67DC6F352
:107F6000C006002E44D1264B186801680A68904765
:107F700061782278234B01F0070042EA00221A6060
:107F8000A2782E7002F03F00400140EAD101596012
:107F9000E078810041EA9211227902F0010041EA81
:107FA00080219960617901F00F00C00140EA52021E
:107FB000DA60A27902F07F00000140EA1111196134
:107FC000E079410041EAD212217A01F0030042EA4D
:107FD00040225A61627A02F01F00800140EA91015A
:107FE0009961A07AC10041EA5212DA61012070BDA4
:107FF0000020287070BD00BFC80F0020F10F0020C6
:1080000090110020CC0F0020825C034B53F822001B
:10801000C0F3CF00704700BF2810002010B5044601
:10802000FDF796FA154B1A68811AB1F57A6F1A4660
:10803000134B01D9002119701060187820B9A82CB1
:108040001AD1104B187006E0022802D10E4A1470A3
:1080500001E0142801D80D490C540B490130C3B27A
:108060000878074A4100481D8342137004D1002359
:108070000449137001220A7010BD00BF20100020B7
:10808000481000201F100020241000200A1000209B
:1080900038B51C46084B0D461A60084908484FF48D
:1080A000E1320123FDF71EF90649C8600CB106480C
:1080B000206008222A7038BD901100201D80000821
:1080C00000440040681D002009800008154B10B5D1
:1080D0001A780AB9002010BD1349002018704B7897
:1080E000012BF7D1114A106801680B6898471048B6
:1080F0000278082A01D90821017001780D4A00236D
:10810000D8B2023288420AD212F8010C12F8024C9C
:1081100040EA0424084840F823400133F0E70120F6
:1081200010BD00BF1F1000200A1000209011002079
:10813000241000200D100020281000201F4B2DE9D6
:10814000F0431B7823B31E4C1E4D277891F800C0D6
:1081500095F8008002231C4C03F10109E65C46FA05
:1081600007F606F00F05EEB266450BD20B2E09D8C6
:10817000E65C14F8094006EA080604EB0626134CF0
:1081800044F825600233102BE5D10C4B00241C7001
:108190000978914202D90E4B197811B94089BDE88E
:1081A000F0830C4B825C1978084B53F8220001B124
:1081B000400800F5777188B2BDE8F0834A100020CE
:1081C0004910002052100020561D00205C10002095
:1081D0005010002051100020134B012210B51A70CE
:1081E0000446FDF7B5F9114A0146106811600B1AF3
:1081F0000F4841F288318B4203600E4B01D90022B7
:108200001A7018780C49E4B20F280C5408D10B4BA3
:108210000B491A680120087010680168884710BD72
:10822000044A431C137010BD501000204C10002055
:108230005410002058100020561D002090110020DE
:108240004A10002010B51C46134B1A60027A5AB12E
:10825000012A13D1114B03201870114B07201870FD
:10826000104802700C2208E00C4B022018700C4BD6
:10827000032018700B48027007220A700A490B4845
:108280004FF4E1320123FDF72DF80949C8600CB124
:10829000084B236010BD00BF901100204910002042
:1082A0005210002051100020D981000800440040E5
:1082B000681D00203D810008014B1878704700BF01
:1082C0004A10002008B54FF40060FAF779FC08B9AD
:1082D000002008BD4020FAF773FC094B20B993F841
:1082E0002D21501E0128F3D993F82C01012805D126
:1082F000034991F82D31002BEAD008BD012008BDBB
:10830000F8170020084B93F82D215AB993F82E0145
:1083100010B9064A537801E005490B7D181C18BFB7
:108320000120704701207047F8170020E31C00204F
:10833000F41C002010B5084B93F82C211C460AB9F8
:1083400000F0ACF894F82C01012803D1BDE81040EE
:1083500000F062BA10BD00BFF817002038B50E4B10
:108360001878C0B1FFF7CEFF0C4904460A78824264
:1083700011D060B10A4D95F82C310BB900F098F886
:1083800095F82C01012804D100F03EFA01E0FFF736
:10839000D1FF02490C7038BD8D1000208C100020D8
:1083A000F817002038B504464020FAF709FC0B4DB9
:1083B00008B985F82D01FFF785FF094B187095F86E
:1083C0002D01012801D1074803E002280CBF06480F
:1083D0002068A060BDE83840FFF7C0BFF817002054
:1083E0008D10002094110020DC1300200B4B10B5E1
:1083F000187888B1FFF786FF70B1094991F82C21F0
:108400000C460AB900F06CF894F82C31012B03D11A
:10841000BDE8104000F008BA10BD00BF8D1000206C
:10842000F817002038B5064C05465E21A068FCF719
:1084300008FEA0682946BDE83840FCF702BE00BF30
:10844000681D0020024B5E219868FCF7FABD00BF52
:10845000681D002010B50A4C5E280146A06805D1B1
:108460005D21FCF7EEFDA0683E2105E05D2903D10A
:10847000FCF7E7FDA0683D21BDE81040FCF7E1BD39
:10848000681D002010B50446C0B2FFF7E3FFC4F337
:108490000720BDE81040FFF7DDBF0000034B93F855
:1084A0002D0108B900F092BA704700BFF8170020FC
:1084B000044B93F82D0118B94FF4165000F078BA18
:1084C000704700BFF817002008B5044B9868FCF708
:1084D000C8FDD0F1010038BF002008BD681D002094
:1084E0002DE9F041FFF7F0FF002800F04081FDF793
:1084F00049F8A04B1A68811A7C2940F2388118602B
:108500009D480478651C0570002404F12406F0B22F
:10851000FFF788FF994B33F91400F8F7F7FA984AF8
:1085200005461088F8F7F2FA01462846F8F7F6FBF8
:108530009449F8F73FFBF8F703FD013400B2FFF769
:10854000A1FF032CE1D13020FFF76CFF8E49B1F978
:108550000000FFF797FFFFF775FF8748067816F0D2
:10856000030629D1894D1020FFF75CFF2B68642496
:1085700093FBF4F210B2FFF785FF2120FFF752FFC3
:10858000296891FBF4F004FB101484EAE473A3EB74
:10859000E47318B2FFF776FF1420FFF743FF7C4A1D
:1085A000B2F90000FFF76EFF1C20FFF73BFF3046DB
:1085B000FFF768FFFFF746FF6F490878430740F071
:1085C000B080744D0220FFF72DFFB5F900300A2569
:1085D00093FBF5F0FFF756FF0220FAF7F1FA0028B7
:1085E00047D06D4F6D4E3878347840F63401B4FB87
:1085F000F0F26B4C4A4321882A2391FBF0F800FBF0
:108600001810B2FBF3F24FEA001399B241EA022CC0
:108610001FFA8CFEC2F303224EEA02080620FFF77F
:1086200001FF0FFA88F0FFF72DFF20883F78431CE9
:108630009AB292FBF7F107FB1120367820806E2466
:108640007443152394FBF3F43A206427FFF7EAFE02
:10865000B4FBF7F63046FFF715FF3B20FFF7E2FECD
:1086600007FB164291B24C1D94FBF5F000B2FFF7E8
:1086700009FF2020FFF7CEFA002850D0494C1320E4
:10868000FFF7D0FE2568484F002DB8BF6D4295FB1F
:10869000F7F630B2FFF7F6FE1B20FFF7C3FE2368A4
:1086A0000A26002BB8BF5B4293FBF6F142F210752D
:1086B00091FBF5F205FB121000B2FFF7E3FE232059
:1086C000FFF7B0FE2368002BACBF4E205320FFF70E
:1086D000D9FE1220FFF7A6FE61680029B8BF494203
:1086E00091FBF7F210B2FFF7CDFE1A20FFF79AFECA
:1086F00060680028B8BF404290FBF6F696FBF5F3A1
:1087000005FB136108B2FFF7BDFE2220FFF78AFECA
:108710006268002AACBF45205720FFF7B3FEFFF781
:1087200091FE15480378282B21D100240470FCF712
:1087300029FF4FF47A753C24B0FBF5F61720FFF7BC
:1087400071FEB6FBF4F5B5FBF4F104FB1152100217
:1087500000B2FFF797FE1820FFF764FE04FB1563D5
:1087600018B2FFF78FFEBDE8F041FFF76BBEBDE822
:10877000F08100BF941000208E1000207C1C00208F
:108780000C00002000007A44680C0020400C0020FF
:108790004E1C0020A41B00200400002024170020F1
:1087A00090100020F01B0020A0860100154B2DE941
:1087B000F04180460F4698680221FCF766FC0024D1
:1087C0002646781E84420F4D0DDA18F80410A8686A
:1087D0008E190134FCF735FC4FF47A70B6B2FCF711
:1087E000D7FEE4B2EDE7F1B2A868FCF72AFC4FF43B
:1087F0007A70FCF7CDFEA8680121BDE8F041FCF7D6
:1088000044BC00BF681D0020024B01219868FCF7A2
:108810003CBC00BF681D0020024B03219868FCF798
:1088200034BC00BF681D0020F8B5544CA068FCF7AC
:1088300018FC002800F0A080A068FCF717FC054693
:108840000520FCF7B0FE8A2D21D08E2DEDD14C4CA9
:1088500000212E22204605F0F1F84A4A7C2323709D
:108860001378E0207D21E07084F82C1014204FF460
:10887000FA71A37723754822782320766076618386
:108880006570628484F8243020462E2171E0202017
:10889000FFF7C0F90028C8D03B4C00212C2220460D
:1088A00005F0CCF8A021E170384B39497C207D22BD
:1088B000207084F82B201878CA7A6570A076002A78
:1088C00052D0344934480F686625FE0F97FBF0FC00
:1088D0006672324E5FFA8CFC06FB0C7284F82950EB
:1088E00006256A4342F21073B2FBF3FE03FB1E2718
:1088F0004968277391FBF0F03F0AC0B26773CF0F4E
:1089000006FB00116943B1FBF3F5642203FB151369
:10891000E9B202FB0010010AE073214821740188CA
:108920005FFA8EFE63741B0A02FB0CECA374B1FBAE
:10893000F2F224235A4390B21A4A010A1388E071D2
:108940002172180A1849207518480A8801884FEAC8
:108950001C2EE374130A84F80AC084F80BE0A77392
:108960006275A375217702E0202384F82930064838
:108970002C21FFF71BFF58E7F8BD00BF681D002042
:10898000C410002024170020981000200E1C002086
:10899000E31C0020F01B0020A08601006079FEFF90
:1089A000B01B0020D21B0020A61B0020DC1B0020D7
:1089B00008B50246032303480021FCF793FC024B51
:1089C000186008BD00380140681D0020024B18687F
:1089D0000068FFF7EDBF00BFF410002008B5044B9E
:1089E0001860FFF7F3FFBDE8084001F0EFB800BFE3
:1089F000F4100020034B187808B100F0F1BE01F02C
:108A00005FB900BFF8100020232801D100F0E8BEB4
:108A1000044B19688A7A824202D10120FCF740BED9
:108A2000704700BFF410002070B50646B6FBF2F4A4
:108A30000846154614B12046FFF7F6FF05FB1464FF
:108A4000024B195D00F8011B70BD00BF48F400081F
:108A50002DE9F041027803460130202AFAD0092A94
:108A6000F8D02D2A02D10346414D04E02B2A08BF3D
:108A700003464FF07E551E460024334616F8010B80
:108A8000A0F13007F9B209290DD83A492046F8F784
:108A900091F804463846F8F739F801462046F7F7CA
:108AA00081FF0446E9E72E2817D1324F334616F8E6
:108AB000010B3038C2B2092A0FD8F8F727F8394627
:108AC000F8F72CF901462046F7F76CFF29490446D0
:108AD0003846F8F76FF80746E8E71878652801D0B8
:108AE000452839D15E782D2E02D19F1C012605E044
:108AF0002B2E01D05F1C00E09F1C00267B1E002750
:108B000013F8012F303AD1B2092903D80A2000FB0B
:108B10000727F5E7B7F59A7F28BF4FF49A77B8464D
:108B20004FF07E51B8F1070F07D908461249F8F700
:108B300041F8A8F108080146F4E707F0070737B144
:108B400008460C49F8F736F8013F0146F7E72EB121
:108B50002046F8F7E3F804E04FF07E512046F8F79E
:108B600029F801462846F8F725F8BDE8F08100BF4E
:108B7000000080BF0000204120BCBE4C10B5441E48
:108B800014F8011F21B1034B1868FCF75AFAF7E7F4
:108B900010BD00BF681D00200148FFF7EFBF00BFF8
:108BA0006DF4000810B50748FFF7E8FF0024064BF6
:108BB00006481A19E15852680C34FAF7DBFAC02C4F
:108BC000F5D110BD9BF400086CF30008B1F4000867
:108BD00070B5FCF7D7FC244C244B4FF47A71B0FBF2
:108BE000F1F11A7822482378FAF7C4FAFFF72CF843
:108BF00005462048204902682048B2FBF1F1FAF707
:108C0000B9FA00241E4B53F8241051B1012000FA88
:108C100004F0284202D01B48FAF7ACFA0134E4B25F
:108C2000F0E70220FEF7F6FF68B1174A174B1178FC
:108C3000174853F82110FAF79DFA1648017A11B136
:108C40001548FAF797FA154C1548FFF797FF24884F
:108C5000FCF7B6F90246134821464FF46673BDE8A7
:108C60007040FAF787BA00BF0400002024170020E4
:108C7000B9F400084C01002040420F00F7F400084E
:108C80008C02010815F50008240800202CF40008C7
:108C900019F50008281C002023F50008F80700201B
:108CA000D6F7000827F5000838B50C6805462046B9
:108CB00005F05CF8024628682146BDE8384005F01A
:108CC00085B8000008B50548FFF758FF0A20FCF7F3
:108CD0006AFC0020BDE80840FCF7E2BC59F500083A
:108CE00008B50748FFF74AFF064B93F89403F9F7D6
:108CF00009FFF9F717FFBDE80840FFF7E3BF00BF22
:108D000068F50008F81700207FB5044605F02EF836
:108D1000082825D100231F49E25C086885186E7871
:108D200006F00301022908BF203AE2540133082B60
:108D3000F1D10025665D1848314604F03BFF28B1AB
:108D400001356019314604F035FF18B11348FFF7BB
:108D500015FF1DE0082DEDD120461149FFF766F8FB
:108D60001048FFF70BFF00230F4A04A9981890F84A
:108D700008218818084A995C0133082B00F80C1C5C
:108D8000F2D100208DF80C0001A90848FAF7F2F999
:108D90007FBD00BF68010020C4F2000872F5000822
:108DA0000019002092F50008F8170020B4F400081C
:108DB00008B5FDF79FFF01300CBF03480348BDE82D
:108DC0000840FFF7DBBE00BFA7F50008CDF500089F
:108DD0002DE9F041054604F0C9FF0446FAF796F87C
:108DE000064694B92A48FFF7C9FE2A4951F82410CB
:108DF00049B1012202FA04F2324202D02648FAF7BF
:108E0000B9F90134F1E7254821E0284624492246F2
:108E100004F0DCFF58B92348FFF7B0FE224C54F8A9
:108E2000041F0029EFD01C48FAF7A4F9F7E72B78C4
:108E30002D2B04D10135013C4FF0010801E04FF02A
:108E400000080026134850F8267027B91748BDE8D7
:108E5000F041FFF793BE28463946224604F0B6FF9C
:108E6000A0B9012000FA06F0B8F1000F03D0FAF71C
:108E700045F80F4802E0F9F7ADFE0E48FFF77EFE19
:108E80000D483946BDE8F041FAF774B90136D9E723
:108E9000EBF50008D0F2000815F50008D6F7000839
:108EA00096000108FEF50008CCF2000813F6000851
:108EB0002DF6000837F60008B4F4000810B5044693
:108EC0000848FFF75BFE084A084809490023036089
:108ED00013700B70FDF79CF82046BDE81040FFF7BB
:108EE000FFBE00BF40F60008F91000202C11002042
:108EF000F810002008B50448FFF740FEF9F772FEAD
:108F0000BDE80840FFF7DEBE58F60008F8B5074692
:108F100004F02CFF044638B91A491B4B4A791B4808
:108F2000511E53F8211028E038461949224604F012
:108F30004DFF60B91748FFF721FE174C54F8041F86
:108F400019B11648FAF716F9F8E7154805E00025B3
:108F50000D4B53F8256026B91248BDE8F840FFF7DD
:108F60000DBE38463146224604F030FF0135002858
:108F7000EED10448314645710B48BDE8F840FAF798
:108F8000F9B800BFF817002010F3000871F60008C8
:108F90009600010885F600080CF3000815F5000896
:108FA000D6F7000898F60008B0F6000810B5044699
:108FB000204604F0DBFE10F0FF0F07D10B490C48F0
:108FC00091F89413BDE81040FAF7D4B8204604F0A5
:108FD000EBFB022808D8054B064C83F89403F9F7FD
:108FE000A1FDF9F75BFDE3E710BD00BFF817002016
:108FF000C2F60008E6F9000870B5044604F0B6FEB3
:1090000008B9204830E020461F4905F027FB00241E
:109010002646254678B12CB1012C06D104F0C4FBBC
:10902000064602E004F0C0FB054600201649013464
:1090300005F014FBEEE70B2D05D914480C21BDE813
:109040007040FAF797B8012C08DC114A114832F940
:1090500015202946BDE87040FAF78CB8A6F57A735A
:10906000B3F57A7F04D90C48BDE87040FAF782B8AE
:109070000A4829463246FAF77DF8054820F8156077
:1090800070BD00BFD8F60008B0F9000812F700085C
:10909000AC1C002038F7000850F7000872F70008F1
:1090A00038B5054604F062FEC0B268B904461249FC
:1090B000124801EB4402B2F8422021460134FAF78B
:1090C00059F8152CF3D138BD284604F06DFB14284F
:1090D00004460BDC2021284604F06CFD04F064FB00
:1090E000054B03EB4404A4F8420038BD04481521A5
:1090F000BDE83840FAF73EB82C1700208BF700087F
:1091000097F70008931E222B88BF0A22031E10B572
:109110000C4603DA2D2001F8010B5842FFF784FCBE
:1091200000210170204610BD30B587B005460C46C1
:1091300003A800210C2204F081FC28460021F7F747
:10914000F5FE20B128462949F7F72CFC03E0284614
:109150002649F7F725FC2649F7F72CFDF7F7F0FE2F
:10916000054685EAE570A0EBE5700A226946FFF73F
:10917000C9FF002D01DB202300E02D2368468DF878
:109180000C3004F0F3FD012807D130228DF80D20BA
:109190008DF80E208DF80F200CE0022805D130212B
:1091A0008DF80D108DF80E1004E0032802D1302048
:1091B0008DF80D00694603A804F0D6FC03A804F05E
:1091C000D5FDC51EEDB22A4603A9204604F06CFE6B
:1091D000002363552046074904F0C6FC03A9204636
:1091E000491904F0C1FC204607B030BD6F12033AA4
:1091F00000007A4466F5000837B5037904460D4649
:10920000052B34D8DFE803F003060A0D111481683A
:1092100009782DE0806890F9001029E083681988AA
:1092200026E08268B2F9001022E0816809681FE038
:10923000806869460068FFF777FF01461148F9F733
:1092400099FFF5B1E068F7F761FC6946FFF76CFF3D
:1092500001460D48F9F78EFF2069F7F757FC69467C
:10926000FFF762FF01460848F9F784FF09E0002193
:109270000648F9F77FFF25B10548E1682269F9F74B
:1092800079FF3EBD20F500081FF50008C1F7000872
:10929000BDF700082DE9F047064604F067FD0546D6
:1092A00020B1012819D133782A2B16D14748FFF76E
:1092B00065FC002414266643454F4648F159F9F7EA
:1092C00059FFB8192946FFF797FF01344248FFF7C5
:1092D00055FC6F2CEED1BDE8F08730463D2104F0FF
:1092E00069FC002857D0441C204604F05DFA8246F1
:1092F0002046FFF7ADFB0027054614247C43DFF82A
:10930000D09054F80980404604F030FD41460246B2
:10931000304604F05BFD002835D14C44E068F7F797
:10932000F5FB01462846F7F7F7FD002829D020690C
:10933000F7F7ECFB01462846F7F7E4FD002820D0BC
:1093400020792279052818BF5546052A0FD8DFE86D
:1093500002F003030606090CA1680D7007E0A2687D
:10936000158004E0A068056001E0A1680D60414639
:109370001A48F9F7FFFE20460021BDE8F047FFF745
:109380003BBF174803E001376F2FB6D11548BDE842
:10939000F047FFF7F3BB0446142565430C4F3146F5
:1093A00055F80780404604F0E3FF50B109484146B4
:1093B000F9F7E0FE78190021FFF71EFF0648F9F7DC
:1093C000D9FE01346F2CE7D1BDE8F087C4F700085F
:1093D000AC020108A3F80008D6F70008D9F7000886
:1093E000E4F7000809F800082DE9F043584885B073
:1093F000584CF9F7BFFE5848FFF752FE6279574BB9
:10940000511E574853F82110F9F7B4FE2069002186
:10941000F7F764FD002858D1002526690021304661
:10942000F7F75CFD00284CD101354E482946D4F8A9
:109430001490D4F81880E769F9F79CFE30460021B3
:10944000F7F756FD10B14848F9F794FE69463046E3
:10945000FFF76AFE01464548F9F78CFE48460021B1
:10946000F7F746FD10B14048F9F784FE69464846D3
:10947000FFF75AFE01463D48F9F77CFE40460021C1
:10948000F7F736FD10B13848F9F774FE69464046E3
:10949000FFF74AFE01463548F9F76CFE38460021D1
:1094A000F7F726FD10B13048F9F764FE69463846F3
:1094B000FFF73AFE01462E48F9F75CFE10340C2DFA
:1094C000ABD12C48691CF9F755FEF9F71FFD2A4C62
:1094D000064654F8041F19B12848F9F74BFEF8E77F
:1094E0000D46274850F8251049B1012202FA05F22D
:1094F000324202D02348F9F73DFE0135F1E7154B22
:10950000214ACE1896F808418B5C04A80131051950
:10951000082905F8103CF2D100241C4869468DF852
:109520000840F9F727FE14256543194E1948A95933
:10953000F9F720FE00217019FFF75EFE013416488E
:10954000FFF71CFB6F2CEED105B0BDE8F08300BF28
:1095500026F80008F8170020E6F9000810F30008C4
:1095600056F8000861F80008B0F9000820F5000876
:10957000B4F4000869F80008CCF200087BF8000891
:10958000D0F2000889F80008C4F2000896F8000834
:10959000AC0201089FF80008D6F700082DE9F04357
:1095A00089B0044604F0E2FBC6B2002E6AD17948C5
:1095B000FFF7E4FA784C20690021F7F78FFC38BBFD
:1095C000013676483146F9F7D5FD206904A9FFF741
:1095D000ABFD01467248F9F7CDFD606904A9FFF7BC
:1095E000A3FD01466E48F9F7C5FDA06904A9FFF780
:1095F0009BFD01466A48F9F7BDFDE06904A9FFF744
:1096000093FD01466748F9F7B5FD10340C2ED2D111
:109610000025654C2F46A8464FF000091034B1458F
:1096200014DA404654F8101CF7F7BCF954F80C1C37
:1096300080462846F7F7B6F954F8081C0546384620
:10964000F7F7B0F909F101090746E7E75748CDF800
:10965000048002950397FFF791FA002401A823588C
:10966000534923F00040F7F761FC5249524A043451
:10967000002814BF10460846FFF780FA0C2CEDD1E5
:109680004E4870E020464E49052204F09FFB38B951
:10969000414B0022C1181030C0280A61F8D176E091
:1096A00020464849042204F091FB0546204605BBAC
:1096B000202104F07FFA002869D0461C304604F0CF
:1096C00055FB2C460746404850F824500DB93F48FA
:1096D00049E030462946FAB204F078FB38B9204612
:1096E000FCF734FD3A482946F9F744FD47E00134D8
:1096F000E9E704F059F8461E0B2E074643DC2046E6
:10970000202104F057FA054640B1451C2846FFF7D2
:109710009FF9214B3F01D851012400E0044628461F
:10972000202104F047FA054640B1451C2846FFF7C2
:109730008FF91949013401EB0612506128462021A6
:1097400004F038FA054640B1451C2846FFF780F979
:10975000114B013403EB061188612846202104F0E7
:1097600029FA18B91B48FFF709FA10E00130FFF792
:109770006FF9094A032C02EB0616F061F2D1164884
:10978000FFF70CFF03E015480C21F9F7F3FC09B0D3
:10979000BDE8F083B1F80008F8170020DCF80008F5
:1097A000E2F80008B4F400080C180020E6F80008FD
:1097B0000AD7233CADF80008A9F80008D6F700083E
:1097C000F5F80008FBF8000810F3000898F6000808
:1097D00000F9000813F90008E6F900084DF900083F
:1097E000F0B5694B87B01A783AB90120187067480C
:1097F000FFF7C4F96648FFF7C1F9664C2068FBF72C
:1098000030FC002800F0BD802068FBF72FFC092801
:109810000146614A01D03F2851D1002517685F4CAD
:109820002E462FB15E4821683A4604F0CFFA10B9AF
:10983000254606B926465B490C348C42F1D3C6B1A5
:109840003468D5F800E03B46E05C1EF80310814226
:109850000DD1534A41B92D2B06D820244E48D4545B
:1098600001330360D15404E0D0540133ECE74A499A
:109870000B60494A14681CB1AE4201D13C4612E06B
:109880004948FFF77BF9AE4209D856F80C0BFFF7B1
:1098900075F9404B09211868FBF7D3FBF3E73C4807
:1098A000FFF76CF900243C4B18688442A5D2394973
:1098B0003B4A0868115DFBF7C4FB0134F3E713680A
:1098C0002BB9042838D13648FFF7F8FA59E00C28AC
:1098D00001D136488CE70A2901D00D2948D12E4DF7
:1098E0003348FFF74BF92E4C2A6832490023A35422
:1098F0000493009103A8294910220C23039403F038
:1099000057FF054638B1006804F030FA0130AA6804
:109910002018904702E02848FFF730F90021302254
:109920001F4804F08BF818481B4B0278002119607F
:10993000002A7FF45FAF24E00C28CAD07F2903D12E
:109940005BE72F2B3FF659AF1F297FF656AF7E29D5
:109950003FF653AF13B920293FF44FAF104C0E48D8
:109960000C4AE154013303601068FBF76AFB44E7DB
:109970007F29E6D10A485C1E0021015514600F487A
:1099800039E707B0F0BD00BFF810002075F90008F6
:10999000ADF90008681D00202C1100206CF30008B0
:1099A000F91000202CF40008B2F90008B7F90008FB
:1099B000D6F70008A98C0008C2F90008E3F90008EE
:1099C000F8B5174E174C184D0746C1B230682170D4
:1099D000FBF737FB22782B78C7F3072182EA0300D5
:1099E000287030682170FBF72CFB21782A783068CA
:1099F00081EA0203C7F307412B702170FBF721FBBB
:109A00002078297880EA0102390E306821702A70A6
:109A1000FBF717FB2B78207880EA03012970F8BD4B
:109A2000681D00203411002030110020F8B50D4EC3
:109A30000D4D0E4CC1B2074630682970FBF701FB93
:109A40002A782378391282EA03002070297030685E
:109A5000C9B2FBF7F6FA23782A7882EA030020706D
:109A6000F8BD00BF681D0020331100203011002018
:109A7000054B10B5044621461868FBF7E2FA034887
:109A800002785440047010BD681D00203011002081
:109A9000034B04491A78885C01321A70704700BF82
:109AA000311100204E11002010B5FFF7F1FF0446E0
:109AB000FFF7EEFF04EB002080B210BD10B5FFF7FA
:109AC000F3FF0446FFF7F0FF04EB004010BD000079
:109AD00038B5044624200D46FFF7CAFF4D20FFF796
:109AE000C7FF002C0CBF3E202120FFF7C1FF064B13
:109AF000002228461A70FFF7BBFF04480078BDE833
:109B00003840FFF7B5BF00BF3011002038110020EA
:109B100001460020FFF7DCBF01460120FFF7D8BF58
:109B2000014B1878FFF7A4BF3011002070B505462F
:109B300008460E46FFF7ECFF2C467219D0B2E3B28E
:109B4000984204D014F8010BFFF792FFF5E770BDBF
:109B500010B5441E14F8010F10B1FFF789FFF9E7A3
:109B600010BD00002DE9F843002701240025144B07
:109B7000187885421CDA1349134B15F801800C2222
:109B800002FB0830406804F0F1F881460CB13F1840
:109B90000CE026464E4509DA0B4A0C2101FB08234E
:109BA0005868805DFFF764FF0136F3E70135DEE7B3
:109BB00024B1F8B2FFF7ACFF0024D7E7BDE8F88383
:109BC00037110020391100203000002070B5394DC8
:109BD000FF211522284603F031FF002302202B70BD
:109BE000FEF718F8012418B102206C70A870032445
:109BF0000420FEF70FF868B12E4E03214FF40050F9
:109C00003155651CF8F7DCFF18B104227255023497
:109C100000E02C460220FDF7FDFF48B1254B052052
:109C20001E190621072518557170B570033404E01C
:109C30000820FDF7EFFF0028F0D12020F8F7C0FF43
:109C400018B11C4B08221A5501344FF48070F8F7F4
:109C5000B7FF30B117480A2601190B2506554D707C
:109C60000234154A134B5079082801D00E2802D12E
:109C70000C261E5501340D2104201955651CF8F7DA
:109C80009FFF18B10B4811224255A51C0A49132306
:109C900091F82E21074E6C1C101C18BF0120735523
:109CA000F8F78EFF10B114203055AC1C034B1C701C
:109CB00070BD00BF39110020F817002037110020B7
:109CC000F8B5B54C2068FBF7CCF9002800F04785C3
:109CD0002068FBF7CBF9B14A0346117871B9B0F1AE
:109CE0002404634253EB040111700029E9D1AC4A0A
:109CF0005478002CE5D1FEF787FEE2E7012904D174
:109D00004D280CBF0223002321E0022904D13C2866
:109D10000CBF032300231AE003290FD140284FF082
:109D2000000101D91170CCE79E489F4C03709F48F9
:109D3000217001709E490B70042308E0042908D1AA
:109D40009B499C480C78037063400B70052313708B
:109D5000B7E70529B5D19448924C017822788A4218
:109D6000934A07D914785C401470934A53544B1C9F
:109D70000370A6E71078984240F0EC848D4B197878
:109D80007B2900F0318300F2C5806E2900F07B83CF
:109D900060D8682900F0448325D8652900F0108236
:109DA00019D8642940F0D1840720844CFFF7B0FE15
:109DB000E620FFF75DFE6079FFF75AFE0020FFF70F
:109DC00057FE94F819017E4B7E4A00280CBF1046BE
:109DD000184600F06BBC662900F07082672940F0DD
:109DE000B48479481DE36B2900F02B8323D86929BB
:109DF00000F01B836A2940F0A8841020FFF788FE3A
:109E00006748724CC07AFFF733FE71490878FFF754
:109E10002FFE2068FFF7D4FD6068FFF7D1FD6D4A83
:109E2000B2F90000FFF702FE6B4BB3F90000FFF739
:109E3000FDFD6A4A24E36C2900F015836D2940F08A
:109E400084840620FFF764FE65490868FFF7B8FDC3
:109E5000644A15E3732900F083833CD8702900F02D
:109E60004183C0F02183712900F04F83722940F0B3
:109E70006C84524C1620FFF74BFE0020FFF7D6FDF6
:109E8000B4F9D000FFF7D2FD574DB4F9D200FFF777
:109E9000CDFDB4F9D400FFF7C9FDB5F9B600FFF761
:109EA000C5FD0020FFF7C2FD0020FFF789FDB5F9D1
:109EB00028000A2390FBF3F0FFF7B8FD94F80401A3
:109EC000FFF7D6FD94F80601FFF7D2FD94F80501DF
:109ED000FFF7CEFD73E3762900F04D830DD874298A
:109EE00000F02B83752940F030842F20FFF710FEFF
:109EF0003E48FFF72DFE00F02BBC772900F02083B1
:109F0000782940F02284384C3820FFF701FE04F114
:109F1000400537E2D02900F0878300F2CA80CA29C1
:109F200000F00F816CD8A42900F0EE8310D8A0298E
:109F300040F00B840C20FFF7EBFD2D492D4C0868F9
:109F4000FFF73EFD2C4A1068FFF73AFD2068ADE3AD
:109F5000C82900F0ED80C92940F0F783FFF798FD8C
:109F60000F4B1A4CD872FFF793FD19490870FFF791
:109F7000A5FD2060FFF7A2FD6060FFF795FD154A83
:109F80001080FFF791FD144B18801C48017841F0B8
:109F900002040470E4E000BF681D002032110020BC
:109FA000E31C002035110020361100203111002063
:109FB00030110020381100204E110020F817002029
:109FC0001C000080140000801C000020F01B0020FA
:109FD0000E1C0020A61B0020B01B0020140800202F
:109FE000741C0020680C00202C170020580B01085E
:109FF000E8F7FF1FF0F7FF1FECF7FF1F84070020B3
:10A00000CD2900F01B8322D8CB2900F0AB80CC29CE
:10A0100040F09B83FFF73CFDC74CE077FFF738FD2E
:10A0200084F82000FFF734FD84F82300FFF730FDAB
:10A0300084F82400FFF72CFD84F82500FFF728FDA5
:10A0400084F82100FFF724FD84F8220088E0CE295F
:10A0500000F0FE82CF2940F07883FFF725FDFFF75F
:10A0600023FDB64CB44DA4F8D000FFF71DFDA4F8B5
:10A07000D200FFF719FDA4F8D400FFF715FDA5F8ED
:10A08000B600FFF711FDFFF719FDFFF70DFD0A23DD
:10A0900058432885FFF7FCFC84F80401FFF7F8FC1F
:10A0A00084F80601FFF7F4FC84F80501FFF7F0FCE3
:10A0B00056E0D52900F0A6810FD8D2296BD0C0F088
:10A0C0008282D32977D0D42940F03F839A4C002054
:10A0D000FFF71EFD04F1400568E1F02900F0D98288
:10A0E0000CD8D6294ED0EF2940F02F83FFF7DCFCA7
:10A0F000914CA085FFF7D8FC608531E0FA2900F08B
:10A10000AF82FE2940F021830820FFF701FD8C4C2F
:10A110008C488D4B01682068B1FBF3F2B0FBF3F380
:10A120004FF47A7101FB0234884AD4800024A8E2FB
:10A130000024FFF7B9FC864A10530234102CF8D1E2
:10A140000EE0844C04F10A05FFF7A2FC01346070B4
:10A15000FFF79EFCE072FFF79BFCAC426075F3D109
:10A1600000208BE200247C4801788C42F8D27B4DA1
:10A17000655DFFF799FC704A013402EB4505A5F8CF
:10A180004200F0E70024FFF78FFC754A10530234B9
:10A19000102CF8D1E4E7734C6478002CE0D1FFF781
:10A1A00077FC6649022881F8940388BF81F89443BC
:10A1B000F8F7B8FC3FE2FFF777FC6B490880CFE780
:10A1C0006A4D0B20FFF7A4FCB5F90000FFF72EFC49
:10A1D000FAF7F6FE00B2FFF729FC0220FDF71AFDA0
:10A1E00005460420FDF716FD04460820FDF712FD84
:10A1F000820042EA4401294320208CB2FDF70AFD87
:10A2000044EAC00084B21020FDF704FD44EA0013C4
:10A2100018B2FFF70BFC534A1079D17884005378B9
:10A22000907944EA4101194341EAC0045179537AD3
:10A2300044EA411040EA83144D48C17944EAC1130D
:10A24000047A417A43EA042343EA4124D379117A18
:10A2500044EA8324927A44EAC123417B43EA0234EC
:10A26000827B44EA4133017C43EA8234027944EA46
:10A270000143417C43EA0214827C44EA4143C17CAD
:10A2800043EA8244007D44EAC142334B42EA00542F
:10A290000020197803468B420AD2304D01225D5DC1
:10A2A00002FA05F525421CBF9A4010430133F2E73C
:10A2B000224CFFF785FB94F8940381E11220FFF70D
:10A2C00027FC2C490C88B4F5806F2B4CB4F90000A6
:10A2D00008D8FFF7ABFBB4F90200FFF7A7FBB4F90E
:10A2E00004000EE0082590FBF5F0FFF79FFBB4F9A2
:10A2F000020090FBF5F0FFF799FBB4F9043093FBF3
:10A30000F5F01E4CFFF792FBB4F90000FFF78EFB4F
:10A31000B4F90200FFF78AFBB4F90400184CFFF708
:10A3200085FBB4F90000FFF781FBB4F90200FFF7E9
:10A330007DFBB4F90400B6E12C170020F8170020CB
:10A340004C0100204801002040420F00BC1B0020AF
:10A35000241D00202B170020371100203911002068
:10A36000AC1C0020E31C00204C1C0020F80700203F
:10A37000F41C00200C0000207C1C00205E0C00203F
:10A38000341C0020B4F97400FFF750FBB4F97600D8
:10A39000FFF74CFBB4F97800FFF748FB94F87A001C
:10A3A0000834FFF765FBAC42ECD1D1E1FFF77CFB51
:10A3B000A4F87400FFF778FBA4F87600FFF774FBAD
:10A3C000A0F57A72072893B298BF84F87B00B3F5A2
:10A3D0007A7F98BFA4F87800FFF75AFB84F87A00D8
:10A3E0000834AC42E2D1B3E10820FFF791FB00242E
:10A3F000B04AA31893F87B000834FFF739FB402CD0
:10A40000F6D1A5E10020FFF783FB0024FFF740FB16
:10A41000A84AA3180834402C83F87B00F6D197E1B2
:10A42000A5481021FFF782FB92E11020FFF770FB97
:10A430000024A248005F0234FFF7F8FA102CF8D18C
:10A4400086E10520FFF764FB9D4BB3F90000FFF7A1
:10A45000EDFA9C48B0F90000FFF7E8FA9A490A784B
:10A4600002F00100ACE0994C0620FFF751FBB4F973
:10A470000000FFF7DBFAB4F90200FFF7D7FA944ABD
:10A48000B2F900000FE10720FFF742FB9148007886
:10A49000FFF7EEFA0020FFF7C9FA8F4BB3F900007F
:10A4A000FFF7C4FA0020FEE0824C0720FFF730FBE4
:10A4B000E07FFFF7DDFA94F82000FFF7D9FA94F86F
:10A4C0002300FFF7D5FA94F82400FFF7D1FA94F8A7
:10A4D0002500FFF7CDFA94F82100FFF7C9FA94F8A8
:10A4E00022006DE01E20FFF713FB7C4C04F10A05EF
:10A4F00001346078FFF7BCFAE07AFFF7B9FA607DC3
:10A50000FFF7B6FAAC42F3D122E175490A7854005C
:10A5100004F0FE00FFF7FCFA0024714803789C4227
:10A5200080F016816F496348625C013400EB42039E
:10A53000B3F94200FFF77AFAEFE7FFF713FB07E101
:10A54000674900240878FFF7E3FA654A10788442E7
:10A5500080F0FE80634B185DFFF78AFA0134F4E760
:10A560000820FFF7D5FA0124E0B20134FFF780FAA2
:10A57000092CF9D1ECE0FFF78BFA06461220FFF721
:10A58000C7FA0EB9584902E0102E03D157490D6899
:10A590004C6801E0002425463046FFF769FA28465A
:10A5A000FFF70EFA2046FFF70BFA514A1068FFF743
:10A5B00007FA0020FFF73AFA0020FFF737FA0020E9
:10A5C000FFF756FAC4E0FFF763FA0546FFF776FA9D
:10A5D0000746FFF773FA0646FFF770FA0446FFF7DF
:10A5E00063FAFFF761FAFFF753FA65B93E4841494C
:10A5F000012207604660CD710A73002C3FF4B0ADB4
:10A600003B4B1C60ACE5102D7FF4AAAD37480760CA
:10A6100046600CB1364A1460374B34480221197039
:10A62000011DFCF78FFB9BE53248417800297FF440
:10A6300097ADF8F7D7FAF8F731FA91E52D4C637832
:10A64000002B7FF48DAD2D494FF4C870088087E54D
:10A650002848417800297FF483AD012282737FE589
:10A66000244B5C78002C70D1254991F89403F8F7BD
:10A6700049FAF8F757FAF8F711FA2046FFF748FABF
:10A6800066E02048005F0234FFF7D0F9082CF8D1CB
:10A690005EE0084C0420FFF73BFAB4F92C00FFF70A
:10A6A000C5F9B4F92A00FFF7C1F951E0FFF788F9BD
:10A6B0004EE000BF2C170020941C0020241D002019
:10A6C000D21B0020DC1B0020840700203C0C002053
:10A6D0004E1C0020241700200C1C00202B170020EB
:10A6E0003711002039110020D41B0020B41B00209A
:10A6F000781C0020E31C00209D0700201808002083
:10A70000F8170020BC1B0020154C23789800411C32
:10A71000C8B2FFF7FDF92078FFF7AAF90024104A24
:10A7200013789C4214D20F48005DFFF7A1F90E493F
:10A73000085DFFF79DF90D4A105DFFF799F90C4B85
:10A74000185DFFF795F90134E9E70020FFF7E4F918
:10A75000FFF7E6F9074900200870FFF7B2BAF8BD25
:10A760000F1C0020941B0020DE1B0020F81B002083
:10A77000181C0020321100202DE9F04107468846C0
:10A7800016460024B4420ED00025BD4205D04046F6
:10A790000135FAF708FFEDB2F7E73C200134FAF78C
:10A7A00002FFE4B2EEE7BDE8F08100000F4B1A684B
:10A7B00042F00100186059680D4A0A405A60186852
:10A7C00020F0847121F480321A60186820F480210E
:10A7D00019605A684FF41F0122F4FE005860996016
:10A7E000044B4FF000629A60704700BF00100240B7
:10A7F0000000FFF800ED00E0164A174B516801F029
:10A800000C00042803D0082805D0144801E014499E
:10A810000868186011E051685068C1F38341023143
:10A82000C00301D40F4A06E052680D4812F4003FFD
:10A83000026818BF520851431960064B0A485A680B
:10A84000054BC2F30311415C1A6822FA01F21A6047
:10A85000704700BF001002404C01002000127A0037
:10A860004801002000093D00380100201FB50023E9
:10A87000574C4FF4E0110093019302930391226827
:10A8800042F480332360A16941F01002A261504C70
:10A89000236803F400310191009A531C009301993D
:10A8A00019B9009AB2F5A06FF1D12168484B11F4A3
:10A8B000003401D0022416E01A6842F00101196048
:10A8C0000094434B1C6804F00202019200994C1C56
:10A8D0000094019A1AB90099B1F5A06FF1D11B68E3
:10A8E00099073BD501243B4902940A6842F01003C2
:10A8F0000B600C6824F003020A600B6843F002044A
:10A900000C60A1F58053596859605A685A605C68B8
:10A91000314A44F480615960146824F07041116038
:10A920002E4C2F490C605C6824F47C145C60146825
:10A9300044F000441460946824F400449460043AA1
:10A940009268120449BF274A4FF4E0120A604FF49C
:10A95000801203920299012901D119E0FEE7022930
:10A960001AD168B10398B0F5801F02D14FF4A0123C
:10A9700005E0039BB3F5E01F02D14FF400120392F0
:10A98000134B5968039841EA000242F4803002E018
:10A99000596841F4601058600D4B1A68184642F02F
:10A9A0008071196002680A4B9201FBD5596821F049
:10A9B000030058605A6842F002015960044B58681D
:10A9C00000F00C02082AF9D1FFF716FF1FBD00BFE7
:10A9D00000100240002002400410014000127A00E2
:10A9E00048010020001BB70008B5154B98420BD159
:10A9F00001214FF4805000F0C1FD4FF48050002140
:10AA0000BDE8084000F0BABD0E49884207D14FF4B6
:10AA10008040012100F0BEFD4FF4804009E00A4A69
:10AA200090420BD14FF40040012100F0B3FD4FF4F0
:10AA300000400021BDE8084000F0ACBD08BD00BFEB
:10AA40000030014000380040003C00400B8810B549
:10AA50004C88028823438C8802F441522343CC88DB
:10AA600023430C8923434C8923438C892343CC897A
:10AA7000098A23431A4393B20380828B22F4006332
:10AA80001A04130C8383018210BD038819B199B293
:10AA900041F0400303E023F040010A04130C03805B
:10AAA000704781817047808980B27047038919425D
:10AAB0000CBF002001207047426810B522F47023BB
:10AAC0000A6823F4807444EA02030C7943EA0422FE
:10AAD0004260CB688A6884681A43084B234013435A
:10AAE0004A7943EA42038360097CC26A4B1E22F41E
:10AAF0007002D9B242EA0152C26210BDFDF7F1FF05
:10AB0000836811B143F0010101E023F0010181608C
:10AB10007047836811B143F4807101E023F48071C0
:10AB200081607047836843F00801816070478068E6
:10AB3000C0F3C0007047836843F004018160704730
:10AB40008068C0F380007047836811B143F4A001AE
:10AB500001E023F4A00181607047092970B54FF02E
:10AB600003040CD94C4307251E3C05FA04F503FAEF
:10AB700004F3C66826EA05052B43C3600BE04C438B
:10AB8000072505FA04F503FA04F3066926EA050524
:10AB900045EA03040461062A4FF005030DD8013A83
:10ABA00053431F2202FA03F201FA03F1446B24EA31
:10ABB000020242EA0103436370BD0C2A0DD85343DD
:10ABC0001F22233B02FA03F201FA03F1046B24EA89
:10ABD000020242EA0103036370BD53431F22413B5B
:10ABE00002FA03F201FA03F1C46A24EA02021143F1
:10ABF000C16270BD40F0BF60024B40F40031D960CB
:10AC0000704700BF00ED00E0C37810B503B3164CE9
:10AC1000E168CB43C3F302244178C4F1040201FA92
:10AC200002F10F2222FA04F28478037822400A43C8
:10AC3000110103F16043CAB203F5614181F80023B9
:10AC40000078012200F01F03410902FA03F007E037
:10AC50000078012200F01F03410902FA03F02031BD
:10AC6000024B43F8210010BD00ED00E000E100E0E0
:10AC700030B5048C24F001052C04250C0584048BCC
:10AC8000A5B225F0F3052A4342EA0313114A048CC6
:10AC90009042A4B29DB215D002F50063984211D043
:10ACA000B0F1804F0ED0A3F5983290420AD002F551
:10ACB0008063984206D003F58062904218BF24F06A
:10ACC0000A0401D124F0020444F001042143058365
:10ACD000018430BD002C014030B5048C24F01005F7
:10ACE0002C04250C0584048B058C24F44074240565
:10ACF000240D44EA022242EA0333144AADB29042E0
:10AD00009BB212D002F5006290420ED0B0F1804F9B
:10AD10000BD0A2F59832904207D002F580629042A3
:10AD200003D002F58062904207D125F0200242F064
:10AD3000100545EA011189B204E025F0A00545F0AF
:10AD4000100529430383018430BD00BF002C01405E
:10AD5000224A038890429BB212D002F500629042D0
:10AD60000ED0B0F1804F0BD0A2F59832904207D0B0
:10AD700002F58062904203D002F58062904203D1D6
:10AD80004A8823F070031343154A904208D002F515
:10AD90008062904204D023F44073CA889BB213436C
:10ADA00003808B880A8883850C4B028598420FD0DC
:10ADB00003F5006290420BD002F54063984207D041
:10ADC00003F58062904203D002F58063984201D17E
:10ADD000097A018601228282704700BF002C01405F
:10ADE00000100040038C70B523F001021404250C00
:10ADF0000584068C8388028B9CB222F073052B0499
:10AE00000D881A0C26F0020633042A434E880D8959
:10AE10001B0C3543ADB22B43134DA8420FD005F5A3
:10AE20000065A8420BD005F54065A84207D005F59E
:10AE30008065A84203D005F58065A8420ED123F0B5
:10AE400008064B898D881E4326F004032B43CE89C8
:10AE50008D8924F440743543ADB22C43C988848075
:10AE600002838186038470BD002C0140038C30B5C1
:10AE700023F010021404250C0584038C8288048BB3
:10AE800023F0200324F4E6452C040D88240C44EA26
:10AE900005241D042B0C0D8992B243EA05134D883D
:10AEA000A4B243EA0513124D9BB2A84203D005F5A4
:10AEB0000065A84215D14D8923F080039BB243EA77
:10AEC00005134FF6BF751D408B8822F4406245EA9A
:10AED0000315ABB28D8942EA8502CD8942EA85022B
:10AEE00092B2C988828004830187038430BD00BF89
:10AEF000002C0140038C30B523F480721404250C1F
:10AF00000584038C8288848B23F4007324F07305FA
:10AF10002C040D88240C2C431D042B0C0D8992B29B
:10AF200043EA05234D8843EA0523124D9BB2A8420C
:10AF300003D005F50065A84215D14D8923F40063BF
:10AF40009BB243EA05234FF6FF351D408B8822F460
:10AF5000405245EA0325ABB28D8942EA0512CD89FC
:10AF600042EA051292B2C988828084838187038471
:10AF700030BD00BF002C0140038C30B523F480525B
:10AF80001404250C0584038C8288858B94B225F4E7
:10AF9000E64215042A0C0D8823F4005342EA0522E8
:10AFA0001D042B0C0D8992B243EA05334D8843EA08
:10AFB00005330A4D9BB2A84203D005F50065A842AF
:10AFC00005D18D8924F4804444EA8514A4B2C9884B
:10AFD00084808283A0F84010038430BD002C01409F
:10AFE00000214FF6FF7383800180C1804180017290
:10AFF00070470023038043808380C38003814381A3
:10B000008381C381704700230122038043808280B3
:10B01000C38003817047038819B199B241F00103DD
:10B0200003E023F001010A04130C03807047B0F819
:10B03000443029B16FEA43436FEA53418AB201E0D9
:10B0400059044A0CA0F84420704783899BB20AB186
:10B05000194301E023EA010181817047038B23F04A
:10B06000080213041A0C114301837047038B23F465
:10B07000006213041A0C42EA01218BB20383704769
:10B08000838B23F0080213041A0C11438183704749
:10B09000838B23F4006213041A0C42EA01218BB261
:10B0A0008383704781847047038B23F00C02130461
:10B0B0001A0C0283038B9AB2114301837047038BEE
:10B0C00023F4406213041A0C0283038B9AB242EAFF
:10B0D00001218BB203837047838B23F00C0213048E
:10B0E0001A0C8283838B9AB2114381837047838BBE
:10B0F00023F4406213041A0C8283838B9AB242EACF
:10B1000001218BB283837047F8B50B880D46044646
:10B110004988AA8843B92B89FFF7AAFDE988204608
:10B12000BDE8F840FFF7C0BF042B08D12B89FFF71B
:10B13000D3FDE9882046BDE8F840FFF7C0BF082BE3
:10B140000E462F89008C3BD120F480731804030C29
:10B150002384A08B83B223F0F30343EA0717374B12
:10B16000208CBFB29C4280B247EA020212D003F5A3
:10B1700000639C420ED0B4F1804F0BD0A3F59833FE
:10B180009C4207D003F580639C4203D003F58063A3
:10B190009C4207D120F4007040EA06218BB243F4B0
:10B1A000807305E020F4206041F4807140EA0103DF
:10B1B000E9882046A2832384BDE8F840FFF78CBFCE
:10B1C00020F480531804030C2384A38B208C23F4D5
:10B1D00040731B051B0D43EA022242EA0733174A5C
:10B1E00080B294429BB212D002F5006294420ED01B
:10B1F000B4F1804F0BD0A2F59832944207D002F5FB
:10B200008062944203D002F58062944207D120F418
:10B21000005040EA063291B241F4805205E047F610
:10B22000FF52024041F480510A43E9882046A3833B
:10B230002284BDE8F840FFF75ABF00BF002C014050
:10B24000808E80B27047008F80B27047808F80B24E
:10B250007047B0F8400080B27047038A828911EAD3
:10B26000030092B203D011420CBF002001207047AE
:10B27000C9438AB202827047038A30B50D4604463C
:10B28000EA8898B220F4405111432182A389288989
:10B29000A98823F4B05340EA0102688923F00C0125
:10B2A00002430804030C1A4391B2A181A08AAA891F
:10B2B00083B223F4407187B01143A18201A800F04A
:10B2C000EBF81848A38984420CBF0498039819B27C
:10B2D00000294FF019032A6803FB00F001DA51003E
:10B2E00000E09100B0FBF1F16423B1FBF3F2120135
:10B2F000100903FB1011A08900B2002806DAC9006A
:10B300003231B1FBF3F303F0070005E009013231FC
:10B31000B1FBF3F303F00F00024390B2208107B0BA
:10B3200030BD00BF00380140838919B199B241F4A2
:10B33000005303E023F400510A04130C8381704787
:10B34000C1F3421310B5012401F01F01A34204FA16
:10B3500001F101D10C3004E0022B01D1103000E0EA
:10B360001430036812B143EA010201E023EA01024A
:10B37000026010BD838A9BB20AB1194301E023EA3F
:10B380000101818270470000034A044B02F18830BA
:10B390005A605860704700BF230167450020024093
:10B3A000024B1A6942F08000186170470020024089
:10B3B000014BD860704700BF00200240084BDA689C
:10B3C000D20709D4D868400708D4D96811F0100F03
:10B3D0000CBF0420032070470120704702207047F3
:10B3E0000020024010B50446FFF7E8FF012806D10F
:10B3F0001CB1FFF7E3FF013CF8E7052010BD002C6E
:10B4000008BF052010BD000073B5002306464FF4A9
:10B4100000500D460193FFF7E5FF04281AD10E4CAA
:10B42000AAB2206940F0010121614FF4005032803E
:10B43000FFF7D8FF042808D102360196019B2D0C96
:10B440001D804FF40050FFF7CDFF216941F6FE72D9
:10B450000A4022617CBD00BF0020024038B505468D
:10B460004FF43020FFF7BEFF042812D1094C2369A6
:10B4700043F002002061656121694FF4302041F002
:10B4800040022261FFF7AEFF216941F6FD730B40D8
:10B49000236138BD00200240204B10B55A6802F0ED
:10B4A0000C01042903D0082905D01D4B01E01D4CD7
:10B4B0002368036011E05C685968C4F38342941CFC
:10B4C000C90301D4184A06E016495B680A6813F4F8
:10B4D000003F18BF520854430460104B5968C1F331
:10B4E000031212498C5C026822FA04F242605C6822
:10B4F000C4F302240C5D22FA04F484605C68C4F393
:10B50000C224095D22FA01F2C2605B680849C3F3F4
:10B510008133CB5CB2FBF3F2026110BD001002403C
:10B5200000127A004801002000093D00540100206B
:10B5300050010020044B5A6909B1104301E022EA8E
:10B5400000005861704700BF00100240044B9A6928
:10B5500009B1104301E022EA00009861704700BF82
:10B5600000100240044BDA6909B1104301E022EAFD
:10B570000000D861704700BF00100240044BDA6839
:10B5800009B1104301E022EA0000D860704700BF13
:10B5900000100240044B1A6909B1104301E022EA8D
:10B5A00000001861704700BF00100240024B5A6A49
:10B5B00042F08070586270470010024008B50B4B93
:10B5C000984207D14FF400100121FFF7E3FF4FF439
:10B5D000001006E04FF480000121FFF7DBFF4FF47D
:10B5E00080000021BDE80840FFF7D4BF00540040B0
:10B5F000F0B58688044687B026F03F000D4601046A
:10B6000001A80E0CFFF748FF2C4A0399B1FBF2F09A
:10B6100087B23E43A680238823F0010213041A0C4C
:10B6200022802B68264A93420AD85B00B1FBF3F0D4
:10B63000013783B2BFB22784032B98BF042320E0D5
:10B64000EE884BF6FF72964204D103225343B1FBBE
:10B65000F3F305E019225343B1FBF3F141F48043C6
:10B6600099B20A054FF4967208BF41F001015043A8
:10B6700041F400434FF47A7190FBF1F0421C91B217
:10B680002184A383228891B241F001032380208882
:10B6900020F4816222F002010B04AA886989180C47
:10B6A00041EA02032989AA89184380B241EA0203C8
:10B6B000208098B2208107B0F0BD00BF40420F004B
:10B6C000A086010041F28833002103604BF6FF722F
:10B6D0004FF480438180C280018141818381704722
:10B6E000038819B199B241F0010303E023F001018D
:10B6F0000A04130C03807047038819B199B241F40E
:10B70000807303E023F480710A04130C03807047F4
:10B71000038819B199B241F4007303E023F4007176
:10B720000A04130C03807047038819B199B241F4DD
:10B73000806303E023F480610A04130C03807047E4
:10B7400083889BB20AB1194301E023EA0101818099
:10B75000704701827047008AC0B2704712B141F051
:10B76000010101E001F0FE010182704702684FF61D
:10B77000FE73134003602D4B00219842016041602D
:10B780008160C16022D02A49884229D0294B984241
:10B7900030D02949884237D0284B98423ED0284B98
:10B7A000984206D153F8681C41F4700043F8680CC5
:10B7B00070472449884206D151F87C0C40F07062F1
:10B7C00041F87C2C7047204B984206D153F8042C4A
:10B7D00042F00F0143F8041C70471C49884206D10F
:10B7E00051F8183C43F0F00041F8180C7047184B22
:10B7F000984206D153F82C2C42F4706143F82C1C6B
:10B8000070471449884206D151F8403C43F47040D7
:10B8100041F8400C7047104B984205D153F8542C16
:10B8200042F4702143F8541C704700BF08000240E6
:10B830001C00024030000240440002405800024018
:10B840006C00024080000240080402401C040240D8
:10B8500030040240440402405804024070B50668B7
:10B860008C680D6A26F4FF4222F070060A6945EAE8
:10B8700004034C6913438A692343CC6913431C4373
:10B880004B6A44EA03028B6A1A4332430260CB6874
:10B890000A68496843608260C16070BD002303602C
:10B8A00043608360C360036143618361C36103627A
:10B8B00043628362704719B1016841F0010303E0FC
:10B8C00002684FF6FE7313400360704703680AB1C5
:10B8D000194301E023EA01010160704741607047AC
:10B8E000406880B270470000C3004CBF014B024B60
:10B8F00058607047000402400000024000B540F666
:10B90000D87320F00042C3F649739A4283B00146CF
:10B9100015DDB2F1FF4F03DBF5F742F803B000BDD0
:10B92000694600F095FB00F00302012A0098019996
:10B930000ED0022A07D082B900F0A0FDEEE7002168
:10B9400000F09CFDEAE700F099FD00F10040E5E71A
:10B9500001F040FC00F10040E0E7012201F03AFC78
:10B96000DCE700BF30B5C0F3C754A4F17F031E2B42
:10B9700083B0014621DC581C1DDBCD0F162B0CDDDE
:10B9800021F07F4323F4000040F40000963C00FACD
:10B9900004F005B1404203B030BD114850F82540D5
:10B9A0002046F4F7FFFF019021460198F4F7F8FFD5
:10B9B00020F0004121B90020EDE7F5F7C1FAEAE7F0
:10B9C00020F07F4222F40003C0F3C75043F400018B
:10B9D000C0F1960221FA02F0002DDCD0DAE700BFB8
:10B9E000380C010800B540F6D87320F00042C3F6C9
:10B9F00049739A4283B0014616DDB2F1FF4F03DB73
:10BA0000F4F7CEFF03B000BD694600F021FB00F063
:10BA10000300012815D002280BD0B8B9009801996D
:10BA2000012201F0D7FBEDE70021002201F0D2FB5B
:10BA3000E8E700980199012201F0CCFB00F10040F9
:10BA4000E0E70098019900F019FDDBE70098019903
:10BA500000F014FD00F10040D4E700BF70B58AB0DB
:10BA6000064600F09BF8224C054694F9003001335D
:10BA700003D0304601F0B0FD10B928460AB070BDC1
:10BA8000304601F05BFD4FF07E51F5F74FFA00288C
:10BA9000F3D0184A01210025304601920091089503
:10BAA000F4F7C4FC02460B461348CDE90423CDE964
:10BAB000022301F011FC94F90030CDE90601022BBC
:10BAC0000BD0684601F006FC38B1089850B9DDE9A2
:10BAD0000601F4F711FF0546CFE701F089FE2121A9
:10BAE0000160F2E701F084FE089A0260EFE700BF10
:10BAF00064010020400C0108480C010800F002BA63
:10BB000070B58AB0054600F04FFC224C064694F909
:10BB10000030013308D0284601F05EFD20B12846F0
:10BB20000021F5F7E5F910B930460AB070BD1A4AA0
:10BB3000012128460026009101920896F4F776FC30
:10BB40002478CDE90401CDE902017CB9002200236B
:10BB5000CDE90623684601F0BDFB88B10898A0B97D
:10BB6000DDE90601F4F7C8FE0646DDE70020002106
:10BB700002460B46F4F7D8FD022CCDE90601E9D1C7
:10BB800001F036FE21230360E8E701F031FE089959
:10BB90000160E5E7640100204C0C0108F8B520F0D5
:10BBA0000043B3F17E5F044613D00BDCB3F17C5F3E
:10BBB00014DAB3F10C5F00F3A48040F6DB70C3F637
:10BBC000C970F8BD0146F4F7EBFE0146F5F7A6F89B
:10BBD000F8BD002840F30E810020F8BD0028C0F217
:10BBE0000E8101464FF07E50F4F7DAFE4FF07C51A3
:10BBF000F4F7E0FF044600F0D7FB4EF60871064666
:10BC000020F47F65C3F611012046F4F7D3FF47F611
:10BC10000471C3F64F21F4F7C5FE2146F4F7CAFFBD
:10BC200041F24611C3F62451F4F7BAFE2146F4F767
:10BC3000C1FF40F6A821C3F64E61F4F7B3FE2146DA
:10BC4000F4F7B8FF4BF29001C3F6A661F4F7A8FE33
:10BC50002146F4F7AFFF4AF6AB21C3F62A61F4F7A9
:10BC6000A1FE2146F4F7A6FF4CF22E610746C3F66B
:10BC70009D512046F4F79EFF43F26131C3F63071C7
:10BC8000F4F78EFE2146F4F795FF45F22D71C4F2CC
:10BC90000101F4F787FE2146F4F78CFF4DF23911CC
:10BCA000C4F21901F4F77CFE2146F4F783FF4FF04C
:10BCB0007E51F4F777FE01463846F5F72FF8314606
:10BCC000F4F778FF25F00F05074629462846F4F7D4
:10BCD00071FF01462046F4F763FE294604463046CC
:10BCE000F4F760FE01462046F5F718F8014638469D
:10BCF000F4F758FE2946F4F755FE0146F4F752FED4
:10BD0000F8BD0146F4F756FF4EF60871C3F611016F
:10BD10000546F4F74FFF47F60471C3F64F21F4F7D9
:10BD200041FE2946F4F746FF41F24611C3F624517D
:10BD3000F4F736FE2946F4F73DFF40F6A821C3F696
:10BD40004E61F4F72FFE2946F4F734FF4BF29001D1
:10BD5000C3F6A661F4F724FE2946F4F72BFF4AF652
:10BD6000AB21C3F62A61F4F71DFE2946F4F722FF42
:10BD70004CF22E610646C3F69D512846F4F71AFF91
:10BD800043F26131C3F63071F4F70AFE2946F4F745
:10BD900011FF45F22D71C4F20101F4F703FE2946AB
:10BDA000F4F708FF4DF23911C4F21901F4F7F8FD68
:10BDB0002946F4F7FFFE4FF07E51F4F7F3FD0146FC
:10BDC0003046F4F7ABFF01462046F4F7F3FE014698
:10BDD00042F26810C3F2A230F4F7E2FD01462046B9
:10BDE000F4F7DEFD014640F6DA70C3F6C970F4F7E9
:10BDF000D7FDF8BD40F6DB70C4F24900F8BD4FF046
:10BE00007E51F4F7CFFD4FF07C51F4F7D3FE4EF6A0
:10BE10000871C3F611010446F4F7CCFE47F604712D
:10BE2000C3F64F21F4F7BEFD2146F4F7C3FE41F2FD
:10BE30004611C3F62451F4F7B3FD2146F4F7BAFED8
:10BE400040F6A821C3F64E61F4F7ACFD2146F4F7A5
:10BE5000B1FE4BF29001C3F6A661F4F7A1FD2146B5
:10BE6000F4F7A8FE4AF6AB21C3F62A61F4F79AFD6F
:10BE70002146F4F79FFE0646204600F095FA4CF264
:10BE80002E610546C3F69D512046F4F793FE43F21A
:10BE90006131C3F63071F4F783FD2146F4F78AFE71
:10BEA00045F22D71C4F20101F4F77CFD2146F4F74F
:10BEB00081FE4DF23911C4F21901F4F771FD2146EA
:10BEC000F4F778FE4FF07E51F4F76CFD01463046F2
:10BED000F4F724FF2946F4F76DFE42F26811C3F22D
:10BEE000A231F4F75DFD01462846F4F75BFD0146FB
:10BEF000F4F758FD014640F6DA70C4F24900F4F751
:10BF00004FFDF8BDF8B521F00044B4F1FF4F0346F2
:10BF100017DC20F00045B5F1FF4F064611DCB1F10A
:10BF20007E5F42D08F1707F0020040EAD37775B9E1
:10BF3000022F35D0032F08D140F6DB73CCF2490332
:10BF400003E01846F4F72EFD03461846F8BDD4B1B9
:10BF5000B4F1FF4F2DD0B5F1FF4F14D02C1BE415D9
:10BF60003C2C18DC002952DB1846F4F7D7FE01F010
:10BF7000E5FA01F0B7F9012F46D0022F35D0002F96
:10BF800025D10346E1E7002E40F6DB731CDBC3F648
:10BF9000C9731846F8BD40F6DB70C3F6C970EAE70E
:10BFA00040F6DB73C4F24903CFE7BDE8F84001F087
:10BFB00099B9B5F1FF4F2FD0022FF1D0032FBBD08D
:10BFC000012F34D00023C0E7CBF6C973BDE74BF691
:10BFD0002E51C3F2BB31F4F7E5FC40F6DB71C4F23D
:10BFE0004901F4F7DDFC0346AFE74BF62E51C3F2EF
:10BFF000BB31F4F7D7FC014640F6DB70C4F24900D0
:10C00000F4F7CEFC0346A0E700F100439DE714F1EE
:10C010003C0FA9DA0020AEE7022F13D0032F0CD07B
:10C02000012F40F6DB7305D0C3F649738DE74FF05F
:10C0300000438AE7CBF6497387E74CF6E433CCF24A
:10C04000160382E74CF6E433C4F216037DE700BF23
:10C050002DE9F04F40F6D87320F00044C3F6497341
:10C060009C4289B006460D4640F38B804CF6E33186
:10C07000C4F216018C4226DC4FF478610028C3F626
:10C08000C97140F32B81F4F78BFC4FF47D6224F0EF
:10C090000F04C3F6C9729442064600F0818044F250
:10C0A0004341C3F23571F4F77BFC0146286030460A
:10C0B000F4F776FC44F24341C3F23571F4F770FCB7
:10C0C0000127686061E04FF47867C4F24937BC42E9
:10C0D00040F38180B4F1FF4F5BDA4FEAE459A9F1F4
:10C0E0008609A4EBC9542046F4F72AFFF4F70EFDA5
:10C0F0000246014620460592F4F752FC4FF0874174
:10C10000F4F758FD0746F4F71BFFF4F7FFFC014670
:10C11000044638460694F4F743FC4FF08741F4F7A1
:10C1200049FD00210790F4F7D9FE002800F0F680C1
:10C130000327204600210DF11808013FF4F7CEFE39
:10C1400040B158F8044D00212046013FF4F7C6FEE7
:10C150000028F6D1924B02200090019305A83B469F
:10C1600029464A4600F066FA002E07460DDA95E8A1
:10C170000C0002F1004103F1004229606A6047426D
:10C1800003E00023286000274B60384609B0BDE873
:10C19000F08F0146F4F704FC002768602860F4E79C
:10C1A0004FF48841C3F23571F4F7FAFB4AF20831D3
:10C1B000C2F685610446F4F7F3FB01462860204689
:10C1C000F4F7EEFB4AF20831C2F68561F4F7E8FBBA
:10C1D00001276860D9E701F0B1F94FF68411C3F681
:10C1E00022718046F4F7E6FC4FF07C51F4F7DAFB5D
:10C1F000F4F7A6FE0746F4F789FC4FF47861C3F61E
:10C20000C9718346F4F7D6FC01464046F4F7C8FBF3
:10C2100044F243418146C3F235715846F4F7CAFCF3
:10C220001F2F8246514648461FDC5E4B7A1E53F84C
:10C23000223024F0FF029A4217D0F4F7B1FB804677
:10C24000C5F8008041464846F4F7AAFB5146F4F78A
:10C25000A7FB002E686098DA08F1004800F1004161
:10C26000C5F8008069607F428FE7F4F799FBE3151A
:10C270008046C0F3C750191A0829E1DD4FF4884100
:10C28000C3F2357158460393F4F794FC8246514645
:10C290004846F4F785FB044621464846F4F780FB00
:10C2A0005146F4F77DFB4AF208318146C2F68561BA
:10C2B0005846F4F77FFC4946F4F772FB8246514634
:10C2C0002046F4F76DFB039BC0F3C7528046981AD3
:10C2D000192841DCC5F80080A146B3E7F4F762FBFA
:10C2E0004FF47D6724F00F04C3F6C977BC420646BD
:10C2F00016D044F24341C3F23571F4F753FB0146C3
:10C3000028603046F4F74CFB44F24341C3F23571E8
:10C31000F4F748FB4FF0FF37686036E7032719E76B
:10C320004FF48841C3F23571F4F73CFB4AF208310F
:10C33000C2F685610446F4F735FB014628602046C5
:10C34000F4F72EFB4AF20831C2F68561F4F72AFBB6
:10C350004FF0FF37686018E74FF42341C2F685615C
:10C360005846F4F727FC804641462046F4F718FB70
:10C37000814649462046F4F713FB4146F4F710FB8B
:10C3800043F232110446C2F28D415846F4F712FCD2
:10C390002146F4F705FB8246514648464DE700BF6B
:10C3A000D40C0108540C010820F00042B2F1FF4FF8
:10C3B000F8B50446034646D2002A42D0002852DB94
:10C3C000C415B2F5000F09D210F4000553D15B007B
:10C3D00001351902FBD5C5F10100241823F07F4176
:10C3E0007F3C21F40006E20746F4000048BF40000D
:10C3F00043004FF08072002760109A423C462CDDCB
:10C400005B004FF400021825A61851089E4205F162
:10C41000FF3502DCB4189B1BBF185B0062189A4200
:10C4200002DC9B1A54187F185B004A08013DEBD1CF
:10C4300013B107F001017F187C1004F17C5303EB6A
:10C44000C0542046F8BD0146F4F7B4FB014620462F
:10C45000F4F7A8FA04462046F8BD4FF0007403F143
:10C460007F431746CCE70146F4F79AFA0146F4F702
:10C4700055FC0446E5E70120AFE700BF2DE9F8438E
:10C4800020F00046B6F1485F05460F465BDAF4F748
:10C4900057FD002800F0CA8029462846F4F78AFB99
:10C4A0004DF24E71CAF647510446F4F783FB47F24A
:10C4B000F641C3F20F11F4F775FA2146F4F77AFB4F
:10C4C0004FF27C21C3F29341F4F76AFA2146F4F764
:10C4D00071FB40F60151C3F2D071F4F763FA2146C3
:10C4E000F4F768FB40F66131C3F6B621F4F758FA69
:10C4F0002146F4F75FFB4AF6AB21C3F62A51F4F765
:10C5000051FA2146F4F756FB804620464FF07C5105
:10C51000F4F750FB414606462046F4F74BFB3946FC
:10C5200004462846F4F746FB01462046F4F738FA5D
:10C5300001463046F4F734FA01464FF07E50F4F7E6
:10C540002FFABDE8F8830146F4F734FB4DF24E7143
:10C55000CAF647510446F4F72DFB47F2F641C3F201
:10C560000F11F4F71FFA2146F4F724FB4FF27C2158
:10C57000C3F29341F4F714FA2146F4F71BFB40F69B
:10C580000151C3F2D071F4F70DFA2146F4F712FB12
:10C5900040F66131C3F6B621F4F702FA2146F4F70A
:10C5A00009FB4AF6AB21C3F62A51F4F7FBF9214601
:10C5B000F4F700FB49F69913C3F699639E4280464F
:10C5C000A3DD0020C3F64870864227DC06F17F46D3
:10C5D0004FF07E503146F4F7E3F9814620464FF0A4
:10C5E0007C51F4F7E7FA3146F4F7DAF941460646AA
:10C5F0002046F4F7DFFA394604462846F4F7DAFA1B
:10C6000001462046F4F7CCF901463046F4F7C8F964
:10C6100001464846F4F7C4F9BDE8F8834FF0000935
:10C620000026C3F63879C3F69066D7E74FF07E5000
:10C63000BDE8F8832DE9F04FDFB00C930C9D224B41
:10C64000689C0A91691ED61E48BF161D834653F882
:10C650002400F71027EAE7730890049104980D93DB
:10C66000089DDC43DDF834C002EBC4024119079297
:10C67000C0EB0C0750D47E18699BC7EB0609013646
:10C68000002F03EB870522AC09F0010AC0F2FE82FD
:10C690002868F4F73BFA0137B74220604FF00408EE
:10C6A0003AD0BAF1000F26D0002FC0F2F18255F82F
:10C6B0000800F4F72BFA0137B74244F8080008F1F4
:10C6C000040818D128E000BFEC0F010855F8080055
:10C6D000F4F71CFA013708F1040944F8080013D4F0
:10C6E00055F80900F4F712FA0137B74244F8090087
:10C6F00009F1040810D0002FE8DA0020013708F112
:10C70000040944F80800EBD501370020B74244F88B
:10C71000090009F10408EED1089A002AC0F2458503
:10C7200008990C9E8D004AAB5C19039549AF0294A1
:10C730004FEA860A049A002AC0F296820DF1880810
:10C7400008EB860555F8041CAAF10403DBF8000089
:10C75000C3F38009F4F72EFA01460020F4F722F91A
:10C760000424043D544580462BD0B9F1000F0DD070
:10C7700055F8041DDBF80400F4F71CFA01464046A6
:10C78000F4F710F90824544580461AD055F8041CD3
:10C790005BF80400F4F70EFA01464046F4F702F99C
:10C7A0000434804655F8081C5BF80400F4F702FADC
:10C7B00001464046F4F7F6F80434083D54458046F7
:10C7C000E4D1029847F8048F01368742B2D1039F23
:10C7D0000EA9CE190996089EB2005EAB9D18002ED8
:10C7E000029255F8509C7DDD0DF5947C4FF06E5112
:10C7F00048460DACA7180CEB0205F4F7DBF9F4F78B
:10C800009FFBF4F783F94FF087410190F4F7D2F9D9
:10C8100001464846F4F7C4F8F4F792FB0EAC2060EA
:10C820000198014655F8040DF4F7BCF8BC42814666
:10C83000C7F3800156D0E9B14FF06E51F4F7BAF961
:10C84000F4F77EFBF4F762F94FF087410190F4F7BB
:10C85000B1F901464846F4F7A3F8F4F771FB019AE1
:10C860000FAC2060114655F8040DF4F79BF8BC425C
:10C87000814637D04FF06E514846F4F79BF9F4F7F4
:10C880005FFBF4F743F94FF087418046F4F792F9E4
:10C8900001464846F4F784F8F4F752FB41466060DD
:10C8A00055F8040DF4F77EF84FF06E518146F4F719
:10C8B00081F9F4F745FBF4F729F94FF087418046F9
:10C8C000F4F778F901464846F4F76AF8F4F738FBCC
:10C8D0004146A06055F8040DF4F764F80834BC42F2
:10C8E0008146C7D10799484600F0A2FE4FF0785123
:10C8F0000546F4F75FF900F025FE4FF08241F4F7AA
:10C9000059F901462846F4F74BF80746F4F718FBA7
:10C910008146F4F7FBF801463846F4F741F80799E9
:10C920000746002940F33981721E0EAC079D54F86A
:10C930002230C5F1080043FA00F101FA00F0C5F118
:10C9400007041B1A43FA04F40DF1380C89444CF81F
:10C950002230002C55DD002E09F1010940F39481AD
:10C96000029D0EABDDF808C053F8042B281F0DF113
:10C97000380E00250EEB0C01C0F3800022B1C2F589
:10C98000807243F8042C01258B4226D060B10F9AA7
:10C990000433002D40F0F38022B1C2F5807543F8D6
:10C9A000045C01258B4218D053F8042B002D40F075
:10C9B000EC80C2F5807012B143F8040C012553F8E5
:10C9C000042B002D40F0DB80C2F58070002AE9D0F6
:10C9D00001258B4243F8040CE6D1079900290DDDAF
:10C9E000012900F0E280022908D1701E0DF1380EF5
:10C9F0005EF8202002F03F034EF82030022C00F0B9
:10CA0000E08038460021F4F769FA002800F0F3804E
:10CA10000898751EA84225DC029B0DF1380E0EEB1E
:10CA200003010B46DDF824C053F8042DCCEB0100C4
:10CA3000011F6345C1F3800011D030B153F8041DCC
:10CA4000DDF824E00A43734509D0099F53F8040D2B
:10CA500053F8041D0243BB4242EA0102F6D1002A08
:10CA600040F01A81089F0EAD781E55F82020002A4C
:10CA700040F0108105EB8004012354F8041D0133BC
:10CA80000029FAD0F018771C87420B9075DCDDF88E
:10CA900010E00D9D0B9B0C9C0EEB0702DDF808C00F
:10CAA000699F991B06EB05094AA8A61922AB07EB5B
:10CAB000890900EB0C05571C8A0003EB86010295DF
:10CAC00006920591002659F8040FF4F71FF8059C0B
:10CAD000A051049800285EDB22AD05EB8702AAF185
:10CAE0000403C3F3800452F8041CDBF80000039431
:10CAF000141FF4F75FF801460020F3F753FF4FF0DF
:10CB00000408D04505462DD0039971B154F8041D91
:10CB1000DBF80400F4F74EF801462846F3F742FF2D
:10CB20004FF00808D04505461CD054F8041C5BF8AB
:10CB30000800F4F73FF801462846F3F733FF08F101
:10CB40000408054654F8081C5BF80800F4F732F8AE
:10CB500001462846F3F726FF08F10408083CD045B3
:10CB60000546E2D1DDF808E0069804364EF8045F89
:10CB700001378642CDF808E0A5D10B9E2CE6C2F124
:10CB8000FF0243F8042C01250CE7C2F1FF0543F82E
:10CB9000045C012513E70025E4E75ED1701E0DF16A
:10CBA000380E5EF820301C12D3E6711E0DF1380CE1
:10CBB0005CF82100022C00F07F024CF821207FF469
:10CBC00020AF39464FF07E50F3F7EAFE0746002DBE
:10CBD0003FF417AF07994FF07E5000F029FD014652
:10CBE0003846F3F7DDFE074638460021F4F776F9BC
:10CBF00000287FF40DAF0294079C38466142CDF8BF
:10CC0000109000F015FD4FF087410546F4F784F9C8
:10CC1000002800F0D2824FF06E512846F3F7CAFF89
:10CC2000F4F78EF9F3F772FF4FF087410746F3F7F9
:10CC3000C1FF01462846F3F7B3FEF4F781F90EA9C8
:10CC400041F826003846F4F77BF9079A0136083296
:10CC50000EAC079244F8260034E04FF07C51F4F714
:10CC60005BF958B90024CCE64FF00008029847F869
:10CC7000048F013687427FF45DADA8E50224002EC3
:10CC800009F101093FF76CAE0025A6E6002002E598
:10CC9000002010E50123F5E6079A0EAE56F8253080
:10CCA000083ACDF8109002940792002B40F08E8243
:10CCB00006EB85042E4654F8045D013E083A002D2B
:10CCC000F9D007924FF07E50079900F0B1FC002E8A
:10CCD0000446C0F2AC804FEA860AC6EB867B0EAFF4
:10CCE0004FEA8B095744C9F100034AA9386801EBA0
:10CCF0000A08C3F3800BF3F709FF2146F3F75AFF45
:10CD00004FF06E51C8F800002046F3F753FFA9F129
:10CD100004096FF0030ACA45054631D0BBF1000F84
:10CD20000BD057F8040CF3F7F1FE2946F3F742FF56
:10CD30006FF0070A48F8040C1AE057F80A00F3F7F6
:10CD4000E5FE2946F3F736FF4FF06E5148F80A002A
:10CD50002846F3F72FFFAAF1040405463859F3F7E4
:10CD6000D5FE2946F3F726FFAAF1080A48F8040081
:10CD700028464FF06E51F3F71DFFCA450546DCD13A
:10CD8000701CDFF84C94DDF820A003900027059676
:10CD9000BAF1000FC0F20582002FC0F20282002615
:10CDA00000241AF0010F354620D0D8F80010D9F829
:10CDB0000000F3F7FFFE01462046F3F7F3FD0125DF
:10CDC000AA45044626DB0426BD420FDD22E0BB4512
:10CDD00020DC58F8021059F80200F3F7EBFE014688
:10CDE0002046F3F7DFFDBD42044613DC58F8061079
:10CDF00059F80600F3F7DEFE01462046F3F7D2FDB0
:10CE000005F1010B06F104020235DA45044602F190
:10CE10000406DCDA5EABDDF80CC003EB87010137FA
:10CE2000674541F8A04CA8F10408B1D1059E689C63
:10CE3000032C16D8DFE814F085011F011F011B0029
:10CE400000230299002900F00B81379C369804F1E9
:10CE500000420A9C00F1004503F100432560626036
:10CE6000A360049D05F007005FB0BDE8F08F002EC1
:10CE7000E6DD06F1FF3836AF07EB88094D4655F879
:10CE800004290DF1D40AD5F808B01046594601928C
:10CE9000F3F788FD804641460198F3F781FD01468E
:10CEA0005846F3F77FFD5545C9F38003A860C5F8E0
:10CEB000048044D0BBB155F80429D5F808B0104619
:10CEC00059460192F3F76EFD0199804608464146A6
:10CED000F3F766FD01465846F3F764FD5545C5F87E
:10CEE0000480A8602BD02C4654F80439D4F808B03C
:10CEF000184659460193F3F755FD8046414601987F
:10CF0000F3F74EFD01465846F3F74CFDC4F8048094
:10CF1000A06055F804BC251FD5F808805846414646
:10CF2000F3F740FD044621465846F3F739FD014624
:10CF30004046F3F737FD55456C60A860D3D1012E0C
:10CF40007FF77EAF4D4655F804B9C7EB090ED5F80B
:10CF500008A058465146AEF10409F3F723FD804678
:10CF600041465846F3F71CFD01465046F3F71AFDBB
:10CF7000BD42C9F38009C5F80480A86043D0B9F167
:10CF8000000F15D055F804A9D5F808905046494629
:10CF9000F3F708FD804641465046F3F701FD014690
:10CFA0004846F3F7FFFCBD42C5F80480A8602AD0CC
:10CFB0002C4654F804A9D4F8089050464946F3F793
:10CFC000F1FC804641465046F3F7EAFC01464846EC
:10CFD000F3F7E8FCC4F80480A06055F8049C251F12
:10CFE000D5F8088048464146F3F7DCFC0446214664
:10CFF0004846F3F7D5FC01464046F3F7D3FCBD4263
:10D000006C60A860D4D1013607EB860708353E4630
:10D010007A1B131F56F8041D0020C3F38007F3F793
:10D02000C1FCAE4203463FF40CAF3FB156F8041DBD
:10D03000F3F7B8FCAE4203463FF403AF184656F888
:10D04000041C341FF3F7AEFC083E54F8041CF3F73D
:10D05000A9FCAE42F3D10299034600297FF4F5AE54
:10D06000DDF828C036993798CCF80010CCF80400C9
:10D07000CCF80830F5E60023002E29DB36AF751C0E
:10D0800007EB85042546E21B55F8041DA2F1040EAA
:10D090000020CEF38008F3F785FCBD42034617D08D
:10D0A000B8F1000F06D055F8041DF3F77BFCBD4224
:10D0B00003460DD0184655F8041C2C1FF3F772FCDC
:10D0C000083D54F8041CF3F76DFCBD42F3D1034650
:10D0D0000299002967D003F10040DDF828C0194605
:10D0E000CCF800003698F3F75BFC002E034621DDF8
:10D0F00036AF07EB8606F51B2A1F3799C2F3800768
:10D10000F3F750FC37ACB442034613D037B1616833
:10D11000F3F748FC38ACB44203460BD0184654F839
:10D12000041FF3F73FFC54F8041FF3F73BFCB44231
:10D13000F5D10346029909B103F100430A9C6360EB
:10D140008FE6002E40DB36AF013607EB8600054642
:10D15000C21B55F8041D0020141FF3F723FCBD4229
:10D16000C4F38006034615D036B155F8041DF3F715
:10D1700019FCBD4203460DD0184655F8041C2C1F5F
:10D18000F3F710FC083D54F8041CF3F70BFCBD4208
:10D19000F3D10346029909B103F100430A9C2360CD
:10D1A0005FE6002436E6184697E7DDF830E09000A9
:10D1B00003904FEA8E0AFFF70ABB2846F3F7C0FE3A
:10D1C0000EAB43F826007DE50023E3E72E4679E524
:10D1D000F80F01082DE9F84320F00043B3F1485F50
:10D1E00004460F46904603DAF3F7AAFE002859D00A
:10D1F00021462046F3F7DEFC21460546F3F7DAFC2C
:10D200004CF6D311C2F62E7106462846F3F7D2FC2F
:10D2100042F63471C3F2D721F3F7C2FB2946F3F784
:10D22000C9FC4EF61B71C3F23861F3F7BBFB29460C
:10D23000F3F7C0FC40F60151C3F65011F3F7B0FB11
:10D240002946F3F7B7FC48F68901C3F60841F3F71E
:10D25000A9FB8146B8F1000F27D04FF07C5138462A
:10D26000F3F7A8FC494680463046F3F7A3FC014695
:10D270004046F3F795FB2946F3F79CFC3946F3F754
:10D280008FFB4AF6AB210546C3F62A613046F3F719
:10D2900091FC01462846F3F785FB01462046F3F74B
:10D2A0007FFB04462046BDE8F88301462846F3F795
:10D2B00081FC4AF6AB21C3F62A61F3F771FB3146D4
:10D2C000F3F778FC01462046F3F76CFB0446204652
:10D2D000BDE8F8830020704700210020C7F6F871F0
:10D2E000704700BF2DE9F04120F00045B5F1A14F96
:10D2F000044606460DDBB5F1FF4F00F39C80002885
:10D3000040F6DB7440F3D480C3F6C9742046BDE810
:10D31000F0814FF6FF73C3F6DF639D4200F3A280F6
:10D32000B5F1445FC0F28E804FF0FF3721462046B2
:10D33000F3F740FC01468046F3F73CFC46F6D71174
:10D34000C3F685410546F3F735FC4DF65921C3F682
:10D350004B51F3F727FB2946F3F72CFC46F6353102
:10D36000C3F68851F3F71EFB2946F3F723FC42F678
:10D370006E61C3F6BA51F3F715FB2946F3F71AFCB1
:10D3800044F62511C3F61261F3F70CFB2946F3F7B7
:10D3900011FC4AF6AB21C3F6AA61F3F703FB414641
:10D3A000F3F708FC4AF221218046CBF615512846B6
:10D3B000F3F700FC4FF26B11C3F66E51F3F7F0FA7E
:10D3C0002946F3F7F7FB48F29571C3F69D51F3F741
:10D3D000E7FA2946F3F7EEFB48F63861C3F6E35166
:10D3E000F3F7DEFA2946F3F7E5FB4CF6CD41C3F639
:10D3F0004C61F3F7D5FA2946F3F7DCFB7B1C0146B9
:10D40000404658D0F3F7CEFA2146F3F7D3FB494B09
:10D4100053F82710F3F7C4FA2146F3F7C1FA01468F
:10D42000454850F82700F3F7BBFA002E3DDB0446D1
:10D430002046BDE8F0810146F3F7B4FA04462046E1
:10D44000BDE8F0814FF2CA21C7F24911F3F7AAFAF9
:10D450004FF07E51F3F76AFD00283FF465AF204698
:10D46000BDE8F08100F06AF84FF6FF71C3F69771DE
:10D470008D4204464FF6FF7228DCC3F62F729542A8
:10D4800046DC0146F3F78EFA4FF07E51F3F788FA47
:10D490004FF0804105462046F3F784FA01462846BE
:10D4A000F3F73CFC0027044640E700F100442DE779
:10D4B000CBF6C9742AE7F3F775FA2146F3F77AFB3E
:10D4C00001462046F3F76CFA04461FE7C4F21B023C
:10D4D000954214DC4FF07F51F3F762FA4FF07F5121
:10D4E00005462046F3F766FB4FF07E51F3F75AFAF4
:10D4F00001462846F3F712FC0227044616E70020EF
:10D500002146CBF68070F3F709FC032704460DE7AC
:10D510004FF07E51F3F744FA4FF07E510746204614
:10D52000F3F740FA01463846F3F7F8FB01270446C3
:10D53000FCE600BF241001083410010820F0004070
:10D54000704700BFF8B520F00046F50D7F3D162D61
:10D55000014604461BDC002D074620DB4FF6FF7317
:10D56000C0F27F0343FA05F606420ED04FF2CA21FD
:10D57000C7F24911F3F716FA0021F3F7D7FC18B1F7
:10D58000002C1BDB27EA060421460846F8BDB6F14D
:10D59000FF4FFAD3F3F706FA01460846F8BD4FF2FB
:10D5A000CA21C7F24911F3F7FDF90021F3F7BEFCD8
:10D5B0000028E9D0002C07DB0024E5E74FF4000049
:10D5C00040FA05F56719DDE70021CBF68071002EE2
:10D5D00018BF0C46D8E700BF08B902207047B0F169
:10D5E000004FFAD0A0F500026FF001439A4201D833
:10D5F0000420704700F1FF419942F9D94FF6FE73BC
:10D60000421EC0F27F039A4201D80320704700F106
:10D6100000414A1E9A42F8D9B0F1FF4F05D010F5EB
:10D62000000F14BF0020012070470120704700BF89
:10D6300038B530F00044034602460D460FD0B4F131
:10D64000FF4F0ED2B4F5000F11D3E40D6419FE2C78
:10D6500033DC002C1BDD22F0FF4141EAC4531846A5
:10D6600038BD0146F3F79EF90346184638BD4FF022
:10D670009841F3F79FFA43F6B041CFF6FF718D4220
:10D68000034612DBC0F3C7540246193CDEE714F12F
:10D69000160F21DA4CF25032954219460EDC44F254
:10D6A0006020C0F6A25000F023F844F26021C0F6DA
:10D6B000A251F3F77FFA0346D1E719464FF2CA2089
:10D6C000C7F2491000F014F84FF2CA21C7F249110D
:10D6D000F3F770FA0346C2E722F0FF4304F11900A2
:10D6E00043EAC0504FF04C51F3F764FA0346B6E7F3
:10D6F00001F0004120F00040084370472DE9F0415F
:10D70000274C84B025680746D5F84841002C41D005
:10D7100066681F2E1CDD234810B94FF0FF301FE054
:10D720004FF4C870039102920193AFF30080039904
:10D730000446029A019B0028EFD0D5F848610020EA
:10D7400060602660C5F84841C4F88801C4F88C01BF
:10D75000656847B9A81C013544F8201065600020B1
:10D7600004B0BDE8F081012000FA05F0D4F888612A
:10D7700004EB85080643022FC8F88820C4F88861A6
:10D78000C8F80831E6D1D4F88C3143EA0002C4F875
:10D790008C21DFE705F5A674C5F84841B8E700BF5E
:10D7A0004C1101080000000000210A2201F028B8F5
:10D7B0002DE9F84FDDF828B081468A4698469AB19F
:10D7C00093B11646002503E00FD0651CAE420BD97D
:10D7D0007419640808FB04A748463946D84700284E
:10D7E000F2DA2646AE42F3D800273846BDE8F88F75
:10D7F00040F29853C2F2000318687047114B124A66
:10D8000070B5981A831018D0591E02EB83040D4688
:10D8100054F8042D01F00106904775B126B154F873
:10D82000040D8047013D08D054F8043D9847013D60
:10D8300054F8041D8847013DF6D1BDE8704003F05F
:10D840008DBC00BF7411010870110108F8B5204F9C
:10D85000204C381B871017D07A1E2368012502F050
:10D8600001069847AF420FD02EB154F8041F02258D
:10D870008847AF4208D0606880470235A268261DFD
:10D8800090470834AF42F6D1134F144C03F060FCBC
:10D890003B1B9F1018D07D1E216805F00106012555
:10D8A0008847AF4211D02EB154F8040F02258047AB
:10D8B000AF420BD0626890470235A368261D984797
:10D8C0000834AF42F6D1F8BDF8BDF8BDF8BD00BFD1
:10D8D0006811010868110108701101086811010838
:10D8E0000F2A2DE9F00340F2A18041EA00039B07D3
:10D8F00040F09E800C68A2F1100504604B68AC46B5
:10D9000043608C68BCF10F0F8460CC68C5F30015D0
:10D91000C46000F1100301F110042BD975B1256822
:10D92000ACF1100C1D6065685D60A5689D60E568E0
:10D930001034DD601033BCF10F0F1BD9276804F1E0
:10D9400010061F60676803F110055F60A768ACF1FF
:10D95000200C9F60E768DF6024691C61776806F12E
:10D9600010046F60B7682033AF60F668BCF10F0F2A
:10D97000EE60E3D8A2F1100828F00F0302F00F04C4
:10D9800003F1100C032C00EB0C0301EB0C0851D934
:10D99000211F4FEA9109444608EB890C54F8046BA7
:10D9A000C8EB0C010CF1040C1D46644545F8046BF2
:10D9B000C1F3800112D029B154F8041B644545F825
:10D9C000041B0BD0274657F8041B2E4646F8041BB1
:10D9D00064686C603C1D351D6445F3D109F1010C90
:10D9E0004FEA8C0902F0030208EB09014B44D2B163
:10D9F0000D789A18DC4303F8015B1419934204F084
:10DA0000010410D02CB111F8014F03F8014B9342DF
:10DA100009D04D781C4604F8015B8D7802315D70A9
:10DA2000631C9342F5D1BDE8F00370470346DEE77F
:10DA30000346DDE741462246D9E700BFF0B484073C
:10DA4000034600F08D80541E002A00F08780E50711
:10DA5000CEB211D41A4602F8016B1346154692074E
:10DA600010D0621E002C79D003F8016B14469A077F
:10DA70001D4607D0013CEDE7034603F8016B9A070A
:10DA80001D46F7D1032C52D9CEB246EA06270F2CF9
:10DA900047EA07432DD9A4F1100217460F2FC2F30E
:10DAA00000162B606B60AB60EB6005F1100216D9BD
:10DAB0003EB1103F136053609360D36010320F2F5C
:10DAC0000DD9203F02F11006136053609360D360BC
:10DAD000136153619361D36120320F2FF1D8A4F108
:10DAE000100222F00F0204F00F041032032C154430
:10DAF0001DD9271F3E462A46032E42F8043BC7F392
:10DB000080070DD927B1043E032E42F8043B07D904
:10DB1000174647F8043B083E53603A1D032EF7D8DA
:10DB2000231F23F00302131D04F00304ED18ACB10E
:10DB3000C9B2EA432C1905F8011BA318A54203F04A
:10DB400001020BD01AB105F8011BA54206D02B46E5
:10DB500003F8011B69705D1CA542F8D1F0BC704749
:10DB6000054614468EE700BF830770B5064614D1FC
:10DB70000368A3F1013222EA030010F0803F0CD1C8
:10DB8000331D1A4653F8044BA4F1013525EA040469
:10DB900014F0803FF5D0104600E0304603782BB1FA
:10DBA000421C147810460132002CFAD100F080F8A3
:10DBB000304670BDC9B2F0B400294BD082070FD0F7
:10DBC0000278002A71D0914242D0431C05E013F83C
:10DBD000012B002A3BD091423AD09A071846F6D141
:10DBE000036841EA0127A3F1013222EA030212F09D
:10DBF000803F47EA07471CD17B40A3F1013222EA6C
:10DC0000030313F0803F14D1021D02E014F0803FA3
:10DC10000FD1104652F8043BA3F1013687EA030402
:10DC200026EA0303A4F1013513F0803F25EA04043A
:10DC3000ECD00278002A38D0914209D0431C01E090
:10DC4000914205D0184613F8012B002AF8D110464E
:10DC5000F0BC704783070BD00278002AF8D0431C31
:10DC600003E0017801330029F2D099071846F8D172
:10DC70000168A1F1013323EA010212F0803F0AD1C9
:10DC8000031D184653F8041BA1F1013424EA0102D4
:10DC900012F0803FF5D00378002BD9D0421C1178C8
:10DCA000104601320029FAD1D2E71046D0E700BF72
:10DCB00080EA0102844612F0030F4FD111F0030FE6
:10DCC00032D14DF8044D11F0040F51F8043B0BD044
:10DCD000A3F101329A4312F0803F04BF4CF8043B99
:10DCE00051F8043B16D100BF51F8044BA3F10132A7
:10DCF0009A4312F0803FA4F101320BD14CF8043B5F
:10DD0000A24312F0803F04BF51F8043B4CF8044B8F
:10DD1000EAD023460CF8013B13F0FF0F4FEA332300
:10DD2000F8D15DF8044B704711F0010F06D011F8DF
:10DD3000012B0CF8012B002A08BF704711F0020FCD
:10DD4000BFD031F8022B12F0FF0F16BF2CF8022BB8
:10DD50008CF8002012F47F4FB3D1704711F8012BDB
:10DD60000CF8012B002AF9D1704700BF20F0030105
:10DD700010F00300C0F1000051F8043B00F1040C66
:10DD80004FEACC0C6FF000021CBF22FA0CF21343D6
:10DD90004FF0010C4CEA0C2C4CEA0C4CA3EB0C029F
:10DDA00022EA030212EACC1204BF51F8043B043009
:10DDB000F4D013F0FF0F1FBF013013F47F4F013079
:10DDC00013F47F0F18BF0130704700BFF0B4002A72
:10DDD00063D0344B04461B6814F8010B571E1D1802
:10DDE0006E7807F0010706F00305012D58D011F8F1
:10DDF000015B5E19767806F00306012E08BF203518
:10DE0000401B4BD1002D49D0013A47D02FB314F815
:10DE1000010B1D186E7806F00305012D11F8015B4A
:10DE200008BF20305E19767806F00306012E08BF81
:10DE30002035401B32D18DB3013A0ED12EE011F8BE
:10DE4000012B9E18767806F00306012E08BF2032BB
:10DE5000801A23D112B36A1E20D014F8010B1D18AA
:10DE60006E7806F00305012D11F8015B08BF203024
:10DE70005E19767806F00306012E08BF2035401B98
:10DE80000CD15DB114F8010B551E1A18567806F026
:10DE90000302012AD3D12030D1E71046F0BC7047ED
:10DEA0002030A4E76801002041EA00039B07F0B49A
:10DEB00074D1032A72D90C4654F8045B161FA5F1DD
:10DEC000013727EA050717F0803F0346C6F3800CA9
:10DED00031D10346032E324643F8045B2AD9BCF104
:10DEE000000F0AD0214654F8045BA5F1013626EA5A
:10DEF000050616F0803F18D01DE0264656F8045B54
:10DF00002146A5F1013727EA050717F0803F12D116
:10DF100043F8045B65683146A5F1013626EA05063B
:10DF2000043A0C1D16F0803F05D1043A032A43F849
:10DF3000045BE2D821467AB30D78013A03F8015B1D
:10DF40009DB112F0010F1C462AD1234622B311F8CD
:10DF5000015F013A03F8015B3DB111F8015F013A3D
:10DF600065705C1C2346002DEFD1AAB100219C18DE
:10DF7000DA4303F8011BA218A34202F001020BD0FE
:10DF80001AB103F8011BA34206D01A4602F8011B7E
:10DF90005970531CA342F8D1F0BC70470346CAE73E
:10DFA00011F8015F1C4604F8015B013A2346002D7D
:10DFB000CBD1DAE72DE9F00701273C4600254FF0E9
:10DFC000FF3663198B4200EB060C0DD21CF804A03F
:10DFD00010F80380D0452ED201241D469F1B6319E3
:10DFE0008B4200EB060CF1D34FF0010A1760544648
:10DFF00000254FF0FF3C6319994200EB0C080ED945
:10E0000018F8048010F80390C1451AD901241D4660
:10E01000CCEB030A6319994200EB0C08F0D80CF121
:10E0200001000136B0423CBFBA463046C2F800A0FB
:10E03000BDE8F00770470BD001272E463C46ED198E
:10E04000BFE709D04FF0010AAC4654465544D2E729
:10E05000BC4205D00134B4E7544505D00134CAE7C9
:10E0600027461D460124ACE7A2461D460124C2E70F
:10E070002DE9F04FADF2244D15460646894610466F
:10E08000194607AA1C46FFF795FF07AB82460DF21B
:10E090001C411A1D5C6008338B425460F9D114B3E3
:10E0A00001232F78611E08A8A34240F8271001EA37
:10E0B000030218D032B16A7802234F1EA34240F8FF
:10E0C000227010D0B046A4465C1C15F803E0CE1AAE
:10E0D0002A5D02330F1B634540F82E6040F8227022
:10E0E000F2D146466446079928466918524600F020
:10E0F00045FC002840F0B6800AF1FF3E05EB0E0C0F
:10E10000CDF808E0CAF1010E834604F1FF38CDF8DE
:10E110000CC0CDF814E00746CDF810A04A46009593
:10E12000019408E027B1079FBB4201D20199CB1BA4
:10E130009B4400272246019CB0185C440021A21A8F
:10E1400000F07CFB002840F08780002C00F08480E9
:10E15000301910F8013C08A951F82330002BE1D107
:10E16000049B9F4228BF3B46434527D2DDF80090E1
:10E1700006EB0B0119F80350CA5C09EB030095424A
:10E1800066D1DD43454415F0010F024613D001333B
:10E19000434513D24078CD5C013285420BD057E025
:10E1A00012F8010FCD5C854252D1013312F8010FF4
:10E1B000CD5C85424CD101334345F1D3DDF810905D
:10E1C000029B4F4528BF4B4639D2DDF808C0DDF829
:10E1D000009006EB0B0519F80C1015F80C008142A5
:10E1E00040F0C080DDF80CE009EB070ACAEB0E0135
:10E1F000C80772461ED5DDF8089009F1FF31DDF839
:10E200000C90685C19F801CC09F1FF32844516D1F5
:10E210000B460FE012F8019C15F800E04A1EF1458C
:10E220000DD10346013815F800C011F8011C6145F5
:10E2300005D10346581E524502F1FF31EAD101379C
:10E240009F4200F29180079F019ABB44D71B71E760
:10E25000DDF814E0F3446BE7002009B00DF5806DA4
:10E26000BDE8F08FCAEB0400504538BF5046CAF1F4
:10E270000102431C0AF1FF3C05EB0A0704F1FF3BD6
:10E28000019200944A460793B1464FF00008644655
:10E290003E46009909EB020008EB0107BA1A00217B
:10E2A00000F0CCFA0028D7D1002FD5D009EB070019
:10E2B00010F8013C08AA52F8230000284AD1DA4598
:10E2C00009EB08002AD210F80A303178994218BFB9
:10E2D000534642D16FEA0A0303EB0B01C9073246EA
:10E2E000534618D50AF101035B4517D2324612F89E
:10E2F000011F10F803E08E450DD02EE012F8011F2B
:10E3000010F803C08C4528D1013312F8011F10F812
:10E3100003E08E4521D101335B45EFD3621C2346D8
:10E320009BD0295D025D914213D1E10709D5631E9F
:10E33000E95CC25C914204D00BE0E95CC25C9142B2
:10E3400007D15A1E002B88D0A95C825C023B914207
:10E35000F3D0079880443A469BE7DDF804C0E044D8
:10E360009844F8E7049B6AE706EB0B0075E700BFEB
:10E370002DE9F04F037889B080460D46002B00F060
:10E3800065810A789AB184460131012602E011F8CC
:10E39000012B5AB1934214BF002606F001061CF867
:10E3A000013F0C46002BF2D1207820B936B140460F
:10E3B00009B0BDE8F08F4FF00008F8E708F1010060
:10E3C0002978FFF7F7FB641B06460028F3D0012CE1
:10E3D00000F0B580A044404594BFC0EB080701277A
:10E3E0001F2C06D939462A462346FFF741FE8046B0
:10E3F000DDE7214607AA2846FFF7DCFD07990390D1
:10E4000069182846039A00F0B9FA002840F099806C
:10E41000DDF80CC0DDF80C900CF1FF3E05EB0E01B1
:10E42000C9F1010C8346CDF808E080460491CDF88F
:10E4300014C03A46B146019508EB040609EB020008
:10E440000021B21A00F0FAF90028B4D1002EB2D09F
:10E45000039B9B4528BF5B469C4227D9019D09EB46
:10E46000030010F80820E95CE81891425FD1DD4311
:10E470002D1915F0010F024609EB080113D00133E5
:10E480009C4213D94078CD5C013285420BD04EE0DE
:10E4900012F8010FCD5C854249D1013312F8010F0A
:10E4A000CD5C854243D101339C42F1D8DDF80CE0CC
:10E4B000029ADE4540F2CD80019B09EB0805995C8C
:10E4C000A85C814240F0C580DDF804A0049BDA44DA
:10E4D000CAEB0301C8071AD5029FDDF810C0791EE8
:10E4E000685C1CF8017C0CF1FF33874214D10A46AA
:10E4F0000DE013F801EC2F5C4B1EBE450CD102461B
:10E5000001382F5C11F8011CB94205D10246501E9A
:10E51000534503F1FF31ECD10BF1010B934500F2B0
:10E520009A80079A9044C2EB040B324684E7059D1B
:10E5300005EB080B0BEB03084FF0000BF5E78046EB
:10E5400035E7DDF80CA00399CAEB0403534538BF47
:10E550005346CAF1010B581C06EB0A0205EB0A08E8
:10E56000CDF808B03B4607904FF00009019201F149
:10E57000FF3B37468A4609EB0406F8180021F21AD9
:10E5800000F05CF900287FF416AF002E3FF413AFC3
:10E59000544598BF07EB09002CD9DDF804E098F842
:10E5A00000001EF8093098424AD16FEA0A02111998
:10E5B000C9074246534607EB090018D50AF1010383
:10E5C0009C4217D9424612F8011F10F803C08C452F
:10E5D0000DD036E012F8011F10F803E08E4530D15F
:10E5E000013312F8011F10F803C08C4529D1013303
:10E5F0009C42EFD8BBF1FF3F5B463FF4F8AE15F805
:10E600000B1010F80B20914216D11BF0010F0AD00D
:10E610000BF1FF33E95CC25C914204D00CE0E95C91
:10E62000C25C914208D15A1E002B3FF4E0AEA95CB7
:10E63000825C023B9142F2D00798814433469AE7CC
:10E640005346DDF808E0F1449944F7E70C4601260B
:10E65000AAE6039A60E74E46C844A8E640F29853FB
:10E66000C2F200031A6801235C3200F001B800BF57
:10E67000F0B4002825D0074638463E780D460137CD
:10E6800015F8014B3CB1A642FAD1002BF4D117602A
:10E6900007F8013C11E0C6B13D4600E01BB915F892
:10E6A000016B0C46284614F8013B9E42F6D136B168
:10E6B000002105F8011C1060781EF0BC7047304640
:10E6C000F9E710680028D6D1F7E716603046F4E77E
:10E6D0002DE9F00F494C82B0D4F800C001900F46EC
:10E6E0003C4614F8015B0CEB05004678274606F023
:10E6F0000800C6B2002EF3D12D2D61D02B2D04BF02
:10E70000244614F8015BB346002B41D1302D43D091
:10E710000A239A46BBF1000F0CBF6FF000474FF081
:10E720000047B7FBFAF90AFB1970009000208046F9
:10E730000CE0303DAB421BDD461C05D0C84539D846
:10E7400035D00AFB0858012014F8015B0CEB0506D4
:10E75000767806F00407FFB2002FEAD116F0030620
:10E7600006D0012E14BF57263726AD1BAB42E3DC83
:10E77000431C2AD0BBF1000F01D0C8F10008002AC9
:10E7800031D0D0B94046116002B0BDE8F00F7047FB
:10E79000102BBED1302DBCD12578782D25D0582D09
:10E7A00023D043BB4FF0080A30255346B2E7009808
:10E7B0008542C6DD4FF0FF30C6E74046611EE2E706
:10E7C00014F8015B4FF0010B9EE7BBF1000F0199BC
:10E7D0000CBF6FF000404FF0004022230B60002A76
:10E7E000D2D0611ECFE74046CEE74FF0100A6578E1
:10E7F000534602348EE79A4630258BE768010020A5
:10E8000070B440F29854C2F2000406460D462068E7
:10E81000134631462A4670BCFFF75ABF024B13B16C
:10E82000024800F005B8704700000000FDD700085E
:10E830000146002002460346FEF760BF8307F0B49E
:10E84000C9B200F09680531E002A00F0948002782E
:10E850008A420BD0421CD8071AD512F0030F10467B
:10E860001CD01478013B01328C4211D1F0BC7047AE
:10E87000002B7CD01278013B8A42F7D014F0030FB2
:10E88000204604F1010209D02478013B8C42EDD0EE
:10E8900012F0030F104602F10104E9D1032B3FD916
:10E8A000046841EA012545EA054585EA0407A7F120
:10E8B000013222EA07021E1F041D12F0803FC6F338
:10E8C00080072DD1032E334629D967B1266820460B
:10E8D00085EA0602A2F1013626EA0202043412F0A9
:10E8E000803F19D01CE020462468061D85EA0402FA
:10E8F000A2F1013424EA020212F0803F10D1346800
:10E90000043B85EA0402A2F1013424EA0202341D28
:10E9100012F0803F304603D1043B032BE3D820465E
:10E920005D1E23B303788B42A0D0431C0022E8076E
:10E9300014D51C781846012201338C4296D095429A
:10E94000184603F1010402F102020ED01B788B423B
:10E950008CD020462478431C8C4287D095421846A0
:10E9600003F1010402F10202F0D100207EE7184613
:10E970007CE7134692E7104678E700BF032AF0B41D
:10E9800031D941EA00039C072ED106680F68151F94
:10E99000031D0C1DBE42C5F3800C24D1032D2A4655
:10E9A0001FD9BCF1000F08D01E6825682146184603
:10E9B00004340433AE4211D015E0214618461C68D9
:10E9C0000B68051D0E1D9C420DD1314628462E6850
:10E9D0000D68043A031D0C1DAE4204D1043A032A0B
:10E9E000EBD8214618461AB303780C78A3420AD113
:10E9F000551E0022EB0714D510F8013F11F8014F06
:10EA00000122A3420DD0181B10E010F8013F11F8AD
:10EA1000014FA342F7D110F8013F11F8014FA34273
:10EA2000F1D1AA4202F10202EFD10020F0BC7047FE
:10EA30001046FBE71E1E6464646464641048494A1F
:10EA40004B4C4D44454647FF2021222324252627B1
:10EA500048498A8B8C8DFF0068EA00083CEA000870
:10EA600048EA000877EA00082021222324252627E7
:10EA700048494A4B4C4DFF1048498A8B8C8D848500
:10EA80008687FF00371D0008E51C0008091D0008E7
:10EA9000D11C0008D71C0008D31C0008000000404F
:10EAA0000008014001000000001C000000000040C0
:10EAB0000008014002000000041C000000000040AB
:10EAC0000008014004000000081C00000000004095
:10EAD00000080140080000000C1C00000004004079
:10EAE0000008014040000000001D0000000400403C
:10EAF0000008014080000000041D000000040040E8
:10EB0000000C014001000000081D0000000400404E
:10EB1000000C0140020000000C1D0000002C014010
:10EB20000008014000010000001B0100002C014012
:10EB300000080140000800000C1B01000008004014
:10EB4000000C014040000000001E000000080040D2
:10EB5000000C014080000000041E0000000800407E
:10EB6000000C014000010000081E000000080040E9
:10EB7000000C0140000200000C1E0000002C0140AF
:10EB80000000004000040040000800400004080CA1
:10EB9000D007320032003200320032003200320040
:10EBA000C800640000004145545231323334000043
:10EBB000CD3200085133000811330008ED3200084F
:10EBC00029330008AD330008D93200086F5100081E
:10EBD000975000083F510008F5500008AD5000085C
:10EBE000955000080000803F00000000A8AAAA3F3E
:10EBF0000000803F0000803F000080BFB0AA2ABF15
:10EC0000000080BF0000803F0000803FB0AA2ABF04
:10EC1000000080BF0000803F00000000A8AAAA3FBB
:10EC2000000080BF0000803F000080BFB0AA2ABF64
:10EC30000000803F0000803F0000803FB0AA2ABF54
:10EC40000000803F0000803F00000000A8AAAA3F0B
:10EC5000000000000000803F000080BFB0AA2ABF73
:10EC6000000000000000803F0000803FB0AA2ABFE3
:10EC7000000000000000803F000080BF0000803FD7
:10EC8000000080BF0000803F000080BF000080BF08
:10EC90000000803F0000803F0000803F0000803F78
:10ECA0000000803F0000803F0000803F000080BFE8
:10ECB000000080BF0000803F000000000000000056
:10ECC000000000000000803F000000000000000085
:10ECD000000000000000803F000000000000803FB6
:10ECE0000000803F0000803F000080BF000080BF28
:10ECF000000000000000803F000000000000803F96
:10ED0000000080BF0000803F0000803F000080BF07
:10ED1000000000800000803F000000000000803FF5
:10ED2000000080BF0000803F000080BF00000000A6
:10ED30000000803F0000803F0000803F0000000096
:10ED40000000803F0000803F00000000000080BF06
:10ED5000000080BF00000000000000000301000070
:10ED600044EC00080400000014ED0008040000005A
:10ED70004CEF000802010000ECEE0008000100006A
:10ED80000000000006000000E4EB000806000000A0
:10ED90008CEE0008010100000000000004000000EB
:10EDA0000CEF0008060000000CF00008080000004E
:10EDB0006CF00008080000000CEE000808000000DD
:10EDC0008CEF0008010100000000000000010000BD
:10EDD000000000000001000000000000040000002E
:10EDE000D4EC00080600000074EC000800010000EC
:10EDF0000000000002010000ECF00008010100002A
:10EE00000000000000000000000000000000803F43
:10EE1000F704353FF70435BF0000803F0000803F16
:10EE2000F70435BFF70435BF0000803F0000803F86
:10EE3000F70435BFF704353F0000803F0000803FF6
:10EE4000F704353FF704353F0000803F0000803F66
:10EE500000000000000080BF000080BF0000803F75
:10EE6000000080BF00000000000080BF0000803F65
:10EE7000000000000000803F000080BF0000803FD5
:10EE80000000803F00000000000080BF0000803FC5
:10EE9000D0B35DBF0000003F0000803F0000803F16
:10EEA000D0B35DBF000000BF000080BF0000803F06
:10EEB000D0B35D3F0000003F0000803F0000803F76
:10EEC000D0B35D3F000000BF000080BF0000803F66
:10EED00000000000000080BF0000803F0000803F75
:10EEE000000000000000803F000080BF0000803F65
:10EEF0000000803F00000000000000000000803F94
:10EF0000000080BF00000000000000000000803F03
:10EF1000000000000000803F000080BF0000803F34
:10EF2000000080BF000080BF000000000000803FA4
:10EF3000000000000000803F0000803F0000803F94
:10EF40000000803F000080BF000000000000803F04
:10EF5000000080BF0000803F000080BF0000803FB5
:10EF6000000080BF000080BF0000803F0000803FA5
:10EF70000000803F0000803F0000803F0000803F95
:10EF80000000803F000080BF000080BF0000803F85
:10EF90000000803F000000BF0000803F0000803F75
:10EFA000000000BF000080BF0000803F0000803FE5
:10EFB000000080BF0000003F0000803F0000803F55
:10EFC0000000003F0000803F0000803F0000803FC5
:10EFD0000000003F000080BF000080BF0000803FB5
:10EFE000000080BF000000BF000080BF0000803F25
:10EFF000000000BF0000803F000080BF0000803F95
:10F000000000803F0000003F000080BF0000803F04
:10F01000000000BFD0B35D3F0000803F0000803F94
:10F02000000000BFD0B35DBF0000803F0000803F04
:10F030000000003FD0B35D3F000080BF0000803F74
:10F040000000003FD0B35DBF000080BF0000803FE4
:10F05000000080BF00000000000080BF0000803F73
:10F060000000803F000000000000803F0000803F63
:10F07000000080BF0000803F000080BF0000803F94
:10F08000000080BF000080BF0000803F0000803F84
:10F090000000803F0000803F0000803F0000803F74
:10F0A0000000803F000080BF000080BF0000803F64
:10F0B000000080BF0000803F0000803F0000803FD4
:10F0C000000080BF000080BF000080BF0000803FC4
:10F0D0000000803F0000803F000080BF0000803FB4
:10F0E0000000803F000080BF0000803F0000803FA4
:10F0F0000000000000000000000080BF0000803F12
:10F1000000000000000000000000803FB562060122
:10F110000300F00500FF19B56206010300F00300CB
:10F12000FD15B56206010300F00100FB11B5620692
:10F13000010300F00000FA0FB56206010300F002BF
:10F1400000FC13B56206010300F00400FE17B5626F
:10F15000060103000102010E47B56206010300012A
:10F1600003010F49B56206010300010601124FB504
:10F1700062060103000112011E67B562061608004F
:10F1800003070300510800008A41B5620608060023
:10F19000C80001000100DE6A24505542582C343169
:10F1A0002C312C303030332C303030312C31313563
:10F1B0003230302C302A31450D0A0024504D544B4A
:10F1C0003235312C3131353230302A31460D0A009A
:10F1D00024505542582C34312C312C303030332CC3
:10F1E000303030312C35373630302C302A32440D27
:10F1F0000A0024504D544B3235312C3537363030DF
:10F200002A32430D0A0024505542582C34312C31F7
:10F210002C303030332C303030312C3338343030E7
:10F220002C302A32360D0A0024504D544B323531E1
:10F230002C33383430302A32370D0A0024505542EE
:10F24000582C34312C312C303030332C303030319C
:10F250002C31393230302C302A32330D0A00245010
:10F260004D544B3235312C31393230302A32320D57
:10F270000A0000000000000000C2010098F1000830
:10F28000BBF100080100000000E10000D0F100081F
:10F29000F2F10008020000000096000006F20008EB
:10F2A00028F2000803000000004B00003CF20008B8
:10F2B0005EF200080400000080250000E6F9000866
:10F2C000E6F9000841455254313233340000000061
:10F2D000170201081B02010820020108310201087F
:10F2E0003A02010845020108500201085B020108C8
:10F2F0003901010864020108330101086D020108A7
:10F30000770201088202010888020108000000005B
:10F31000690101086D010108730101087901010803
:10F320007C01010883010108860101088B010108A5
:10F33000970101089A010108A0010108A70101082D
:10F34000B1010108BB010108C4010108D201010893
:10F35000DE010108E5010108EB010108F8010108DF
:10F360000302010810020108000000007BFF0008F2
:10F370007FFF0008A1900008A6FF0008ABFF00086F
:10F380009D950008BFFF0008C8FF0008F58E000823
:10F39000E5FF0008EAFF0008E993000819000108EA
:10F3A000E6F90008BD8E00081E00010826000108CD
:10F3B000D18D00083A00010849000108B18D00080C
:10F3C00063000108E6F90008A58B00086800010841
:10F3D0006C000108098D0008B9FF000888000108C9
:10F3E0000D8F00089B000108A1000108F98F00089B
:10F3F000BC000108C4000108AD8F0008D30001085B
:10F40000D8000108E18C0008F7F80008E8000108BE
:10F4100095920008160101080A010108D18B000825
:10F420001D010108E6F90008998B0008E6F90008BB
:10F43000450101084D010108550101085D01010860
:10F4400064010108000000003031323334353637B2
:10F4500038394142434445464748494A4B4C4D4E52
:10F460004F505152535455565758595A004166728D
:10F470006F333220434C492076657273696F6E207A
:10F48000322E32204170722032312032303134201D
:10F490002F2032303A33373A313800417661696C87
:10F4A00061626C6520636F6D6D616E64733A0D0A05
:10F4B0000025730925730D0A0053797374656D2057
:10F4C000557074696D653A202564207365636F6EAD
:10F4D00064732C20566F6C746167653A2025642034
:10F4E0002A20302E315620282564532062617474FE
:10F4F000657279290D0A004350552025644D487ADC
:10F500002C2064657465637465642073656E736F25
:10F5100072733A20002573200041434348573A2034
:10F520002573002E2563004379636C652054696D53
:10F53000653A2025642C20493243204572726F724F
:10F54000733A2025642C20636F6E666967207369A7
:10F550007A653A2025640D0A000D0A5265626F6FC4
:10F5600074696E672E2E2E00536176696E672E2E9B
:10F570002E004D75737420626520616E79206F7264
:10F58000646572206F662041455452313233340D28
:10F590000A0043757272656E742061737369676ED9
:10F5A0006D656E743A20004572726F723A20456E36
:10F5B00061626C6520616E6420706C756720696E95
:10F5C000204750532066697273740D0A00456E61BE
:10F5D000626C696E67204750532070617373746862
:10F5E000726F7567682E2E2E0D0A00456E61626C73
:10F5F00065642066656174757265733A20004176B2
:10F6000061696C61626C65206665617475726573B1
:10F610003A2000496E76616C696420666561747594
:10F620007265206E616D652E2E2E0D0A0044697381
:10F6300061626C65642000456E61626C65642000E7
:10F640000D0A4C656176696E6720434C49206D6FE9
:10F6500064652E2E2E0D0A00526573657474696EF2
:10F660006720746F2064656661756C74732E2E2E2E
:10F670000043757272656E74206D697865723A2008
:10F6800025730D0A00417661696C61626C65206DBD
:10F6900069786572733A2000496E76616C696420FE
:10F6A0006D6978657220747970652E2E2E0D0A00B2
:10F6B0004D697865722073657420746F2025730D11
:10F6C0000A0043757272656E742070726F66696CA1
:10F6D000653A2025640D0A0055736167653A0D0A85
:10F6E0006D6F746F7220696E646578205B76616CF3
:10F6F00075655D202D2073686F77205B6F722073B6
:10F7000065745D206D6F746F722076616C75650D28
:10F710000A004E6F2073756368206D6F746F722CD2
:10F72000207573652061206E756D626572205B3097
:10F730002C2025645D0D0A004D6F746F72202564C6
:10F74000206973207365742061742025640D0A009C
:10F75000496E76616C6964206D6F746F722076619A
:10F760006C75652C20313030302E2E323030300D1B
:10F770000A0053657474696E67206D6F746F722030
:10F78000256420746F2025640D0A0061757820259A
:10F79000752025750D0A00496E76616C69642046F6
:10F7A00065617475726520696E6465783A206D755F
:10F7B0007374206265203C2025750D0A00202564A5
:10F7C0002025640043757272656E742073657474CD
:10F7D000696E67733A200D0A0025732073657420E3
:10F7E000746F20004552523A2056616C7565206155
:10F7F000737369676E6D656E74206F7574206F66C4
:10F800002072616E67650D0A004552523A20556EAE
:10F810006B6E6F776E207661726961626C65206EC7
:10F82000616D650D0A0043757272656E7420436FD9
:10F830006E6669673A20436F7079206576657279E4
:10F840007468696E672062656C6F772068657265A1
:10F850002E2E2E0D0A006D697865722025730D0A13
:10F8600000636D697820256400636D6978202564E4
:10F8700020302030203020300D0A0066656174751C
:10F880007265202D25730D0A0066656174757265B9
:10F890002025730D0A006D61702025730D0A007319
:10F8A0006574202573203D20004E4709004F4B0909
:10F8B00000437573746F6D206D697865723A200D21
:10F8C0000A4D6F746F720954687209526F6C6C093B
:10F8D0005069746368095961770D0A002325643AF9
:10F8E00009002573090053616E69747920636865A6
:10F8F000636B3A09007265736574006C6F61640034
:10F900004C6F61646564202573206D69782E2E2EFE
:10F910000D0A0057726F6E67206E756D62657220FA
:10F920006F6620617267756D656E74732C206E65ED
:10F93000656473206964782074687220726F6C6CDF
:10F94000207069746368207961770D0A004D6F74C7
:10F950006F72206E756D626572206D7573742062B2
:10F9600065206265747765656E203120616E642064
:10F9700025640D0A000D0A456E746572696E672074
:10F98000434C49204D6F64652C20747970652027A5
:10F99000657869742720746F2072657475726E2C97
:10F9A000206F72202768656C70270D0A000D0A23EE
:10F9B00020000D1B5B4B001B5B324A1B5B313B3154
:10F9C00048004552523A20556E6B6E6F776E206339
:10F9D0006F6D6D616E642C20747279202768656C80
:10F9E000702700082008006C6F6F7074696D6500E7
:10F9F000656D665F61766F6964616E6365006D69F0
:10FA0000647263006D696E7468726F74746C650003
:10FA10006D61787468726F74746C65006D696E6383
:10FA20006F6D6D616E64006D696E636865636B0018
:10FA30006D6178636865636B006465616462616EC3
:10FA40006433645F6C6F77006465616462616E64E7
:10FA500033645F68696768006E65757472616C33E2
:10FA600064006465616462616E6433645F746872CB
:10FA70006F74746C65006D6F746F725F70776D5F1B
:10FA80007261746500736572766F5F70776D5F7217
:10FA90006174650072657461726465645F61726D42
:10FAA00000666C6170735F73706565640066697889
:10FAB000656477696E675F616C74686F6C645F64BE
:10FAC0006972007265626F6F745F6368617261630F
:10FAD00074657200736F667473657269616C5F62DE
:10FAE0006175647261746500736F667473657269C1
:10FAF000616C5F315F696E76657274656400736F07
:10FB0000667473657269616C5F325F696E76657287
:10FB1000746564006770735F7479706500677073F3
:10FB20005F62617564726174650073657269616CAE
:10FB300072785F747970650074656C656D65747258
:10FB4000795F70726F76696465720074656C656D5B
:10FB5000657472795F706F72740074656C656D6541
:10FB60007472795F73776974636800766261747325
:10FB700063616C6500766261746D617863656C6C5D
:10FB8000766F6C7461676500766261746D696E632F
:10FB9000656C6C766F6C7461676500706F77657209
:10FBA0005F6164635F6368616E6E656C00616C6960
:10FBB000676E5F6779726F00616C69676E5F616322
:10FBC0006300616C69676E5F6D616700616C696796
:10FBD0006E5F626F6172645F726F6C6C00616C6902
:10FBE000676E5F626F6172645F7069746368006101
:10FBF0006C69676E5F626F6172645F7961770079CB
:10FC000061775F636F6E74726F6C5F646972656356
:10FC100074696F6E006163635F68617264776172BB
:10FC200065006D61785F616E676C655F696E636CBE
:10FC3000696E6174696F6E006D6F726F6E5F74686C
:10FC4000726573686F6C64006779726F5F6C706661
:10FC5000006779726F5F636D70665F666163746F72
:10FC600072006779726F5F636D70666D5F66616366
:10FC7000746F72007069645F636F6E74726F6C6C26
:10FC80006572007961776465616462616E640061C8
:10FC90006C745F686F6C645F7468726F74746C65A9
:10FCA0005F6E65757472616C00616C745F686F6C17
:10FCB000645F666173745F6368616E676500746832
:10FCC000726F74746C655F636F7272656374696F71
:10FCD0006E5F76616C7565007468726F74746C65C4
:10FCE0005F636F7272656374696F6E5F616E676C7C
:10FCF000650072635F726174650072635F6578703E
:10FD00006F007468725F6D6964007468725F657813
:10FD1000706F00726F6C6C5F70697463685F7261A2
:10FD200074650079617772617465007470617261E5
:10FD30007465007470615F627265616B706F696E8B
:10FD400074006661696C736166655F64656C617996
:10FD5000006661696C736166655F6F66665F6465A6
:10FD60006C6179006661696C736166655F74687265
:10FD70006F74746C65006661696C736166655F645D
:10FD800065746563745F7468726573686F6C640032
:10FD9000727373695F6175785F6368616E6E656CBD
:10FDA000007961775F646972656374696F6E00746E
:10FDB00072695F756E61726D65645F736572766F8F
:10FDC0000067696D62616C5F666C61677300616397
:10FDD000635F6C70665F666163746F72006163631A
:10FDE00078795F6465616462616E64006163637AFF
:10FDF0005F6465616462616E64006163635F756E18
:10FE000061726D656463616C006163635F747269E4
:10FE10006D5F7069746368006163635F7472696DBC
:10FE20005F726F6C6C006261726F5F7461625F73AE
:10FE3000697A65006261726F5F6E6F6973655F6C8E
:10FE40007066006261726F5F63665F76656C006208
:10FE500061726F5F63665F616C74006D61675F64A0
:10FE600065636C696E6174696F6E006770735F7053
:10FE70006F735F70006770735F706F735F690067A7
:10FE800070735F706F735F64006770735F706F7320
:10FE9000725F70006770735F706F73725F69006785
:10FEA00070735F706F73725F64006770735F6E6111
:10FEB000765F70006770735F6E61765F6900677070
:10FEC000735F6E61765F64006770735F77705F72F7
:10FED0006164697573006E61765F636F6E74726FD3
:10FEE0006C735F68656164696E67006E61765F73ED
:10FEF000706565645F6D696E006E61765F737065D5
:10FF000065645F6D6178006E61765F736C65775FC5
:10FF10007261746500705F706974636800695F7016
:10FF20006974636800705F726F6C6C00695F726FF8
:10FF30006C6C00705F79617700695F796177007040
:10FF40005F616C7400695F616C7400645F616C7404
:10FF500000705F6C6576656C00695F6C6576656CDA
:10FF600000645F6C6576656C00705F76656C006937
:10FF70005F76656C00645F76656C0061757800661D
:10FF80006561747572655F6E616D65206175786617
:10FF90006C6167206F7220626C616E6B20666F729D
:10FFA000206C69737400636D6978006465736967B8
:10FFB0006E20637573746F6D206D6978657200646F
:10FFC000656661756C747300726573657420746F17
:10FFD0002064656661756C747320616E642072655F
:10FFE000626F6F740064756D70007072696E74205A
:10FFF000636F6E666967757261626C6520736574A4
:020000040801F1
:1000000074696E677320696E20612070617374611A
:10001000626C6520666F726D006578697400666554
:100020006174757265006C697374206F72202D762F
:10003000616C206F722076616C0067707370617301
:10004000737468726F756768007061737374687237
:100050006F7567682067707320746F2073657269AD
:10006000616C0068656C70006D6170006D6170702E
:10007000696E67206F66207263206368616E6E65CB
:100080006C206F72646572006D69786572206E61B4
:100090006D65206F72206C697374006D6F746F7280
:1000A000006765742F736574206D6F746F72206FB5
:1000B00075747075742076616C75650070726F660A
:1000C000696C6500696E64657820283020746F2043
:1000D00032290073617665007361766520616E6414
:1000E000207265626F6F74006E616D653D76616C44
:1000F0007565206F7220626C616E6B206F72202AB2
:1001000020666F72206C6973740073686F77207358
:10011000797374656D20737461747573007665729C
:1001200073696F6E004759524F004143430042418B
:10013000524F00534F4E41520047505300475053C7
:100140002B4D4147004144584C333435004D5055F8
:1001500036303530004D4D413834357800424D4110
:10016000323830004E6F6E6500545249005155418F
:1001700044500051554144580042490047494D42BE
:10018000414C005936004845583600464C59494EB6
:10019000475F57494E470059340048455836580084
:1001A0004F43544F5838004F43544F464C415450DE
:1001B000004F43544F464C41545800414952504C13
:1001C000414E450048454C495F3132305F43435012
:1001D0004D0048454C495F39305F4445470056540F
:1001E00041494C340048455836480050504D5F5402
:1001F0004F5F534552564F004455414C434F505466
:1002000045520053494E474C45434F5054455200C8
:10021000435553544F4D0050504D005642415400E9
:10022000494E464C494748545F4143435F43414C24
:100230000053455249414C5258004D4F544F525F64
:1002400053544F5000534552564F5F54494C54003D
:10025000534F465453455249414C004C45445F521C
:10026000494E47004641494C534146450054454C90
:10027000454D4554525900504F5745524D455445F0
:100280005200564152494F003344000025010108F5
:100290002A0101082E01010841010108330101086A
:1002A000390101083D01010800000000E7F90008DC
:1002B00002000000041800200000000028230000B5
:1002C000F0F90008000000000618002000000000FF
:1002D00001000000FEF90008020000000A190020D9
:1002E000B0040000A406000004FA000802000000A8
:1002F000C818002000000000D007000010FA000815
:1003000002000000CA18002000000000D007000012
:100310001CFA000802000000CC18002000000000B9
:10032000D007000027FA0008020000000C19002086
:1003300000000000D007000030FA000802000000B2
:100340000E19002000000000D007000039FA000854
:1003500002000000CE18002000000000D0070000BE
:1003600048FA000802000000D01800200000000039
:10037000D007000058FA000802000000D218002040
:1003800000000000D007000062FA00080200000030
:10039000D418002000000000D007000076FA000802
:1003A00002000000D618002032000000007D00008E
:1003B00085FA000802000000D81800203200000072
:1003C000F201000094FA000800000000101900205B
:1003D0000000000001000000A1FA00080000000079
:1003E000111900200000000064000000ADFA0008B0
:1003F0000100000012190020FFFFFFFF01000000B4
:10040000C3FA00080000000022190020300000009C
:100410007E000000D8FA000804000000181900202F
:10042000B004000000C20100D4FA0008040000007B
:100430001C190020B0040000004B0000E8FA00087E
:100440000000000020190020000000000100000052
:10045000FEFA000800000000211900200000000042
:100460000100000014FB0008000000001419002027
:1004700000000000040000001DFB00080100000057
:100480001519002000000000040000002AFB0008ED
:100490000000000008190020000000000300000018
:1004A00038FB0008000000002419002000000000B4
:1004B000010000004BFB000800000000251900208F
:1004C00000000000020000005AFB000800000000CD
:1004D0002619002000000000010000006BFB00084E
:1004E00000000000FC1800200A000000C800000006
:1004F00075FB000800000000FD1800200A00000045
:100500003200000088FB000800000000FE180020F8
:100510000A000000320000009BFB00080000000001
:10052000FF1800200000000009000000ADFB0008DB
:1005300000000000DA1800200000000008000000A1
:10054000B8FB000800000000DB18002000000000DD
:1005500008000000C2FB000800000000DC180020BA
:100560000000000008000000CCFB000803000000B1
:10057000DE1800204CFFFFFF68010000DDFB0008D3
:1005800003000000E01800204CFFFFFF680100009E
:10059000EFFB000803000000E21800204CFFFFFF03
:1005A00068010000FFFB000801000000E4180020C3
:1005B000FFFFFFFF0100000015FC00080000000025
:1005C000E5180020000000000500000022FC0008E3
:1005D00002000000EE180020640000008403000008
:1005E00038FC000800000000EC18002000000000AB
:1005F0008000000048FC000802000000E61800200F
:10060000000000000001000051FC00080200000092
:10061000E818002064000000E803000062FC000805
:1006200002000000EA18002064000000E803000057
:1006300074FC0008000000002C17002000000000DF
:1006400001000000E3FD00080000000098170020F2
:10065000000000002000000083FC000800000000F3
:100660009917002000000000640000008FFC0008C3
:10067000000000009A17002001000000FA000000AE
:10068000A9FC0008000000009B17002000000000EB
:1006900001000000BEFC0008000000009E170020C2
:1006A0000000000096000000D8FC000802000000D6
:1006B0009C1700200100000084030000F2FC0008E9
:1006C000000000004B17002000000000FA000000AE
:1006D000FAFC0008000000004C1700200000000099
:1006E0006400000002FD0008000000004D1700201B
:1006F00000000000640000000AFD00080000000087
:100700004E170020000000006400000013FD0008E8
:10071000000000004F1700200000000064000000EF
:1007200023FD00080000000050170020000000001A
:10073000640000002BFD000800000000511700209D
:10074000000000006400000033FD0008020000000B
:1007500052170020E8030000D007000042FD000807
:1007600000000000E017002000000000C8000000AA
:1007700051FD000800000000E1170020000000000B
:10078000C800000064FD000802000000E21700201D
:10079000E8030000D007000076FD0008020000001A
:1007A000E417002064000000D007000090FD00085E
:1007B00001000000131900200000000004000000E8
:1007C000A1FD000801000000E6170020FFFFFFFF69
:1007D00001000000AFFD000801000000E717002045
:1007E0000000000001000000C1FD00080000000042
:1007F000E817002000000000FF000000CEFD000808
:10080000000000005A17002000000000FA0000005D
:10081000DDFD0008000000005C1700200000000063
:1008200064000000ECFD0008000000005B170020E1
:100830000000000064000000FAFD00080000000055
:100840006C170020000000000100000009FE0008F5
:100850000300000058170020D4FEFFFF2C01000009
:1008600018FE00080300000056170020D4FEFFFF0A
:100870002C01000026FE0008000000005D1700208B
:10088000000000003000000034FE000805000000F9
:1008900060170020000000000100000043FE000877
:1008A00005000000641700200000000001000000A7
:1008B0004FFE00080500000068170020000000003F
:1008C000010000005BFE0008030000005417002038
:1008D000B0B9FFFF504600006BFE000800000000AA
:1008E0003117002000000000C800000075FE00085D
:1008F000000000003B17002000000000C8000000BE
:100900007FFE0008000000004517002000000000E6
:10091000C800000089FE0008000000003217002017
:1009200000000000C800000094FE00080000000065
:100930003C17002000000000C80000009FFE0008D7
:10094000000000004617002000000000C800000062
:10095000AAFE00080000000033170020000000007D
:10096000C8000000B4FE0008000000003D17002091
:1009700000000000C8000000BEFE000800000000EB
:100980004717002000000000C8000000C8FE000853
:1009900002000000EA17002000000000D00700005D
:1009A000D6FE000800000000EE1700200000000046
:1009B00001000000EBFE000802000000F01700201C
:1009C0000A000000D0070000F9FE00080200000045
:1009D000F21700200A000000D007000007FF0008FF
:1009E00000000000ED17002000000000640000007F
:1009F00015FF0008000000002E1700200000000076
:100A0000C80000001DFF000800000000381700208B
:100A100000000000C8000000E7FB00080000000024
:100A20004217002000000000C800000025FF000859
:100A3000000000002D17002000000000C80000008A
:100A40002CFF000800000000371700200000000005
:100A5000C8000000D6FB000800000000411700207D
:100A600000000000C800000033FF00080000000084
:100A70002F17002000000000C800000039FF000808
:100A8000000000003917002000000000C80000002E
:100A9000F9FB0008000000004317002000000000E0
:100AA000C80000003FFF00080000000030170020D1
:100AB00000000000C800000045FF00080000000022
:100AC0003A17002000000000C80000004BFF00089B
:100AD000000000004417002000000000C8000000D3
:100AE00051FF000800000000341700200000000043
:100AF000C800000059FF0008000000003E17002059
:100B000000000000C800000061FF000800000000B5
:100B10004817002000000000C800000069FF00081E
:100B2000000000003617002000000000C800000090
:100B30006FFF0008000000004017002000000000C8
:100B4000C800000075FF0008000000004A170020E0
:100B500000000000C8000000524F4C4C3B5049546C
:100B600043483B5941573B414C543B506F733B50BA
:100B70006F73523B4E6176523B4C4556454C3B4D54
:100B800041473B56454C3B0041524D3B00414E478F
:100B90004C453B00484F52495A4F4E3B0042415250
:100BA0004F3B00564152494F3B004D41473B0048A7
:100BB000454144465245453B004845414441444A2D
:100BC0003B0043414D535441423B0043414D54523D
:100BD00049473B0047505320484F4D453B00475045
:100BE0005320484F4C443B005041535354485255B6
:100BF0003B004245455045523B004C45444D415811
:100C00003B004C45444C4F573B004C4C49474854E3
:100C1000533B0043414C49423B00474F5645524EDF
:100C20004F523B004F53442053573B0054454C45D3
:100C30004D455452593B00000000004B000000CBD2
:100C400061636F73660000000000000073717274CE
:100C500066000000000FC93F000F494000CB9640DE
:100C6000000FC9400053FB4000CB164100ED2F415F
:100C7000000F49410031624100537B41003A8A41F3
:100C800000CB9641005CA34100EDAF41007EBC412A
:100C9000000FC94100A0D5410031E24100C2EE4140
:100CA0000053FB4100F20342003A0A420083104223
:100CB00000CB164200141D42005C234200A52942CD
:100CC00000ED2F4200363642007E3C4200C74242D1
:100CD000000F4942A2000000F9000000830000005C
:100CE0006E0000004E0000004400000015000000EF
:100CF00029000000FC000000270000005700000051
:100D0000D1000000F500000034000000DD0000000C
:100D1000C0000000DB000000620000009500000041
:100D2000990000003C00000043000000900000001B
:100D300041000000FE0000005100000063000000C0
:100D4000AB000000DE000000BB000000C50000009A
:100D500061000000B7000000240000006E000000E9
:100D60003A000000420000004D000000D2000000E8
:100D7000E000000006000000490000002E00000016
:100D8000EA00000009000000D1000000920000000D
:100D90001C000000FE0000001D000000EB00000031
:100DA0001C000000B100000029000000A7000000A6
:100DB0003E000000E8000000820000003500000056
:100DC000F50000002E000000BB0000004400000001
:100DD00084000000E90000009C000000700000009A
:100DE00026000000B40000005F0000007E0000004C
:100DF000410000003900000091000000D600000012
:100E0000390000008300000053000000390000009A
:100E1000F40000009C000000840000005F0000005F
:100E20008B000000BD000000F90000002800000059
:100E30003B0000001F000000F800000097000000C9
:100E4000FF000000DE000000050000009800000028
:100E50000F000000EF0000002F0000001100000054
:100E60008B0000005A0000000A0000006D00000026
:100E70001F0000006D000000360000007E00000032
:100E8000CF00000027000000CB0000000900000098
:100E9000B70000004F000000460000003F000000C7
:100EA000660000009E0000005F000000EA000000F5
:100EB0002D0000007500000027000000BA000000AF
:100EC000C7000000EB000000E5000000F10000009A
:100ED0007B0000003D00000007000000390000001A
:100EE000F70000008A00000052000000920000009D
:100EF000EA0000006B000000FB0000005F00000043
:100F0000B10000001F0000008D0000005D00000027
:100F10000800000056000000030000003000000040
:100F200046000000FC0000007B0000006B00000099
:100F3000AB000000F0000000CF000000BC0000008B
:100F4000200000009A000000F400000036000000BD
:100F50001D000000A9000000E30000009100000057
:100F6000610000005E000000E60000001B000000C1
:100F700008000000650000009900000085000000E6
:100F80005F00000014000000A000000068000000E6
:100F9000400000008D000000FF000000D8000000AD
:100FA000800000004D0000007300000027000000DA
:100FB00031000000060000000600000015000000DF
:100FC00056000000CA00000073000000A8000000E6
:100FD000C900000060000000E20000007B0000008B
:100FE000C00000008C0000006B0000000400000046
:100FF00007000000090000000000C93F0000F039B0
:101000000000DA370000A2330000842E0000502BCD
:101010000000C2270000D0220000C41F0000C61B31
:10102000000044176937AC3168212233B40F143300
:101030006821A2333863ED3EDA0F493F5E987B3F6B
:10104000DA0FC93F0020202020202020202028283F
:101050002828282020202020202020202020202078
:1010600020202020208810101010101010101010B8
:1010700010101010100404040404040404040410E8
:101080001010101010104141414141410101010176
:101090000101010101010101010101010101010140
:1010A000101010101010424242424242020202024C
:1010B0000202020202020202020202020202020210
:1010C00010101010200000000000000000000000C0
:1010D0000000000000000000000000000000000010
:1010E0000000000000000000000000000000000000
:1010F00000000000000000000000000000000000F0
:1011000000000000000000000000000000000000DF
:1011100000000000000000000000000000000000CF
:1011200000000000000000000000000000000000BF
:1011300000000000000000000000000000000000AF
:1011400000000000000000004300000070010020CB
:10115000F8B500BFF8BC08BC9E467047F8B500BFA4
:08116000F8BC08BC9E46704774
:081168001DE800083501000834
:041170001101000861
:101174000303D90303010100413600080001000004
:101184000000803F0000000000000000DC05DC05DA
:10119400DC05DC05DC05DC05DC05DC050000803F46
:1011A40000000000880B010800000000010000009E
:1011B4008D0B01080100000002000000940B0108DF
:1011C40002000000030000009D0B01080300000062
:1011D40004000000A30B0108040000000500000047
:1011E400AA0B01080500000006000000AF0B01086F
:1011F4000600000007000000B90B0108070000000A
:1012040008000000C20B01080800000009000000EB
:10121400CB0B0108090000000A000000D40B0108F0
:101224000A0000000B000000DE0B01080B000000A8
:101234000C000000E80B01080C0000000D00000089
:10124400F20B01080D0000000E000000FA0B01086B
:101254000E0000000F000000020C01080F00000047
:10126400100000000A0C010810000000110000002A
:10127400130C010811000000120000001A0C0108F0
:101284001200000013000000240C010813000000E9
:10129400140000002C0C01081400000015000000CC
:1012A40000000000FF00000000000000000000003B
:1012B400010203040607080900127A0000A24A0486
:1012C40002040608000000000102030401020304F2
:1012D400060708090100000044100108000000008E
:1012E400000000005C040020C40400202C05002041
:1012F40000000000000000000000000000000000EA
:1013040000000000000000000000000000000000D9
:101314000000000048110108000000000000000067
:1013240000000000000000000000000000000000B9
:1013340000000000000000000000000000000000A9
:101344000000000000000000000000000000000099
:101354000000000000000000000000000000000089
:101364000000000000000000000000000000000079
:101374000000000000000000000000000000000069
:101384000000000000000000010000000000000058
:101394000E33CDAB34126DE6ECDE05000B0000001D
:1013A4000000000000000000000000000000000039
:1013B4000000000000000000000000000000000029
:1013C4000000000000000000000000000000000019
:1013D4000000000000000000000000000000000009
:0C17040000000000000000007001002048
:0400000508000000EF
:00000001FF
